:020000040800F2
:100000003087002029030008958A0008696E0008DF
:1000100001890008A52700081D9D000800000000B8
:10002000000000000000000000000000690200085D
:10003000532A000800000000C5020008FD910008D6
:100040004303000843030008430300084303000878
:100050004303000843030008552A0008430300082F
:10006000430300085F2A0008692A000843030008C8
:10007000D528000843030008430300084303000891
:10008000430300084303000843030008C92700088E
:10009000A9270008B927000843030008732A0008AD
:1000A0004303000843030008430300084303000818
:1000B0004303000843030008430300087D6E000863
:1000C0006D6E000843030008430300084303000863
:1000D000430300084303000843030008ED9C0008A5
:1000E00043030008430300084303000843030008D8
:1000F00043030008430300084303000843030008C8
:1001000043030008430300084303000843030008B7
:10011000430300084303000843030008D992000882
:10012000430300084303000829290008392900086F
:10013000430300084303000843030008F9270008AD
:10014000D9270008E92700084303000843030008F3
:100150004303000843030008430300084303000867
:100160004303000843030008430300084303000857
:100170004303000843030008430300080000000095
:10018000430300084303000800F002F800F05CF8A5
:100190000AA090E8000C82448344AAF10107DA45E2
:1001A00001D100F051F8AFF2090EBAE80F0013F0D8
:1001B000010F18BFFB1A43F00103184764ED00005C
:1001C00084ED00000A444FF0000C10F8013B13F0DE
:1001D000070408BF10F8014B1D1108BF10F8015BA0
:1001E000641E05D010F8016B641E01F8016BF9D193
:1001F00013F0080F1EBF10F8014BAD1C0C1B09D1EA
:100200006D1E58BF01F801CBFAD505E014F8016B5B
:1002100001F8016B6D1EF9D59142D6D370470000ED
:100220000023002400250026103A28BF78C1FBD8FF
:10023000520728BF30C148BF0B6070471FB50EF092
:100240004EFD1FBD10B510BD00F0E4F91146FFF7DB
:10025000F5FF0AF077FD00F002FA03B4FFF7F2FFB2
:1002600003BC00F005FA00002C4B19680868B0E8E0
:10027000F04F80F30988BFF36F8F4FF0000080F3D9
:10028000118870470000000008480068006880F38B
:1002900008884FF0000080F3148862B661B6BFF39F
:1002A0004F8FBFF36F8F00DF00BF00BF08ED00E08E
:1002B000DFF80C00016841F470010160704700BF75
:1002C00088ED00E0EFF30980BFF36F8F134B1A68DE
:1002D0001EF0100F08BF20ED108A20E9F04F1060CB
:1002E00009B44FF0500080F31188BFF34F8FBFF374
:1002F0006F8F0CF003FC4FF0000080F3118809BCF5
:1003000019680868B0E8F04F1EF0100F08BFB0EC95
:10031000108A80F30988BFF36F8F704718000020A0
:10032000EFF30580704700000948804709480047FF
:10033000FEE7FEE7FEE7FEE7FEE7FEE7FEE7FEE795
:10034000FEE7FEE704480549054A064B70470000F2
:10035000C592000889010008308100203087002004
:10036000308300203083002053EA020C00F06980C3
:100370002DE9F04B4FF00006002B1FBFB3FA83F5B9
:1003800003FA05F424FA05F65E4012BF1643B2FAEA
:1003900082F502FA05F4C5F120051EBF22FA05FC1C
:1003A00044EA0C04203556EA044C4FEA144418BFC2
:1003B000641C4FF000084FF00009904271EB030CF1
:1003C00039D3002919BFB1FA81F701FA07F6B0FA5B
:1003D00080F700FA07F6C7F120071EBF20FA07FCD6
:1003E00046EA0C062037B6FBF4FCA7EB0507103FE6
:1003F00007F01F0BCBF120060CFA0BFB2CFA06F6CC
:1004000044BFB3460026202FA4BF5E464FF0000B2A
:100410005BEA060C08BF4FF0010B19EB0B09ABFBB5
:10042000027C48EB0608C01B06FB02CC0BFB03CC8E
:1004300071EB0C01C1E70B46024641464846BDE858
:10044000F08B13B54FF000004FF00001AFF30080C8
:10045000BDE81C407047032A40F2308010F0030CC6
:1004600000F0158011F8013BBCF1020F624498BF07
:1004700011F801CB00F8013B38BF11F8013BA2F1A4
:10048000040298BF00F801CB38BF00F8013B11F01F
:10049000030300F02580083AC0F0088051F8043BBF
:1004A000083A51F804CBA0E80810F5E7121D5CBF2C
:1004B00051F8043B40F8043BAFF30080D20724BF5F
:1004C00011F8013B11F801CB48BF11F8012B24BFF3
:1004D00000F8013B00F801CB48BF00F8012B704742
:1004E00010B5203AC0F00B80B1E81850203AA0E8CF
:1004F0001850B1E81850A0E81850BFF4F5AF5FEA03
:10050000027C24BFB1E81850A0E8185044BF18C9B5
:1005100018C0BDE810405FEA827C24BF51F8043B5C
:1005200040F8043B08BF7047D20728BF31F8023BB0
:1005300048BF11F8012B28BF20F8023B48BF00F844
:10054000012B704702F0FF0343EA032242EA024212
:1005500000F037B84FF0000200B5134694469646B7
:10056000203922BFA0E80C50A0E80C50B1F12001C6
:10057000BFF4F7AF090728BFA0E80C5048BF0CC074
:100580005DF804EB890028BF40F8042B08BF7047D2
:1005900048BF20F8022B11F0804F18BF00F8012B44
:1005A000704770477047704710B500F02BF800682F
:1005B00010BD10B5044600F025F8046010BD4FF0E2
:1005C00000020429C0F0128010F0030C3FF4C4AF05
:1005D000CCF1040CBCF1020F18BF00F8012BA8BF2E
:1005E00020F8022BA1EB0C01FFF7B6BF5FEAC17C3C
:1005F00024BF00F8012B00F8012B48BF00F8012BA5
:100600007047000000487047CC80002000487047C9
:10061000CC8000207546FFF7F9FFAE46050069461D
:10062000534620F00700854618B020B5FFF78AFE34
:10063000BDE820404FF000064FF000074FF00008E3
:100640004FF0000B21F00701AC46ACE8C009ACE864
:10065000C009ACE8C009ACE8C0098D46704710B5C8
:100660000446AFF300802046BDE81040FFF7F5BD1B
:1006700001491820ABBEFEE72600020070470000CB
:1006800030B52DED068B81B005460C462DB94FF0E7
:10069000FF3001B0BDEC068B30BD14B94FF0FF3018
:1006A000F7E794ED000AD4ED010A20EE200AD4ED1C
:1006B000020A94ED031A00EE810AF0EE000A60EEE1
:1006C000208A94ED010A20EE000AD4ED020A94ED8E
:1006D000021A00EE810AF7EE000AB0EE001AB0EE40
:1006E000609A01EE409AF0EE490AB0EE680A09F00D
:1006F0006FFE85ED010A94ED000AD4ED020A20EEAA
:10070000200AD4ED030A94ED011A00EEC10AF0EEBE
:10071000000A20EE208AB0EEC80AF7EE000AB4EE16
:10072000E00AF1EE10FA0FDB9FED200A8DED000AD2
:1007300018EE100A0246009961F31E0200929DED28
:10074000000A85ED020A05E0B0EE480A09F03CFB1C
:1007500085ED020A94ED000AD4ED030A20EE200A8A
:10076000D4ED010A94ED021A00EE810AF0EE000ABF
:1007700060EE209A94ED020A20EE000AD4ED030AFE
:1007800094ED031A00EE810AF7EE000AB0EE001AAB
:10079000B0EE60AA01EE40AAF0EE4A0AB0EE690A95
:1007A00009F016FE85ED000A002072E7DB0FC93F55
:1007B00070B52DED0A8B04460D46F0EE408A24B943
:1007C0004FF0FF30BDEC0A8B70BDB7EE000AC0EEF3
:1007D000280AC4ED040AB7EE000A84ED000A9FED72
:1007E0006D0A84ED010A9FED6B0A84ED020A9FED0C
:1007F000690A84ED030A002D7DD095ED000A10EE04
:10080000101A08460EF094F941EC1B0B95ED010A05
:1008100010EE101A08460EF08BF941EC1C0BB0EEEE
:100820004B1AF0EE6B1AB0EE4C0AF0EE6C0A09F0BF
:10083000CFFCB0EE40AAF0EE60AA51EC1A0B0DF01E
:1008400075FC41EC190B0DF07DFC08EE100A95EDDE
:10085000000AB5EEC00AF1EE10FA1ED195ED010ABC
:10086000B5EEC00AF1EE10FA17D195ED020AB5EE19
:10087000C00AF1EE10FA10D19FED470A84ED000A8C
:100880009FED460A84ED010A9FED450A84ED020AB8
:100890009FED440A84ED030A78E09FED430AB4EE2D
:1008A000C08AF1EE10FA04D3B5EEC08AF1EE10FA68
:1008B00010DD9FED3E0A84ED000A9FED3D0A84EDB8
:1008C000010A9FED3C0A84ED020A9FED3B0A84ED8C
:1008D000030A5BE09FED390AB4EEC08AF1EE10FA2C
:1008E00006D39FED310AB4EEC08AF1EE10FA12DDA4
:1008F0009FED290A00E04AE084ED000A9FED270AF7
:1009000084ED010A9FED260A84ED020A9FED250A77
:1009100084ED030A3AE09FED2A0AB4EEC08AF1EEB4
:1009200010FA06D39FED250AB4EEC08AF1EE10FA54
:1009300010DD9FED190A84ED000A9FED180A84ED81
:10094000010A9FED170A84ED020A9FED160A84ED55
:10095000030A1BE09FED1A0AB4EEC08AF1EE10FA0A
:1009600004D3B5EEC08AF1EE10FA0FDD9FED0A0A4E
:1009700084ED000A9FED090A84ED010A9FED080A43
:1009800084ED020A9FED070A84ED030A00BF0020F0
:1009900018E7000000000000C5064D3F2D4A0D3C41
:1009A00056A439BBAD47193FDB0FC93F6E597F3F96
:1009B0000C53B039AB88BBBB8595973DDB0F4940E5
:1009C0000000B44200210160416081607047000076
:1009D000F0B52DED108B9DB004460D4616461F4612
:1009E0002CB94FF0FF301DB0BDEC108BF0BD15B928
:1009F0004FF0FF30F7E716B94FF0FF30F3E79FED08
:100A0000FE0AFE4880ED000A2FB9324629462046EC
:100A100000F07EFCE7E797ED00BA97ED019AD7ED7D
:100A2000029AB5EEC0BAF1EE10FA0FD1B5EEC09A47
:100A3000F1EE10FA0AD1F5EEC09AF1EE10FA05D1F6
:100A400032462946204600F063FCCCE7D5ED00EAAB
:100A5000D5ED01DA95ED02FA96ED000A8DED030A67
:100A600096ED010A8DED020A96ED020A8DED010A5E
:100A700094ED010AF1EE400A9DED030A20EE800A92
:100A800094ED021ADDED020A01EE600A94ED031AFC
:100A9000DDED010A01EE600AF6EE000A20EE200A02
:100AA0008DED190AD4ED000A9DED030A20EE800AAF
:100AB00094ED021ADDED010A01EE200A94ED031A0D
:100AC000DDED020A01EE600AF6EE000A20EE200AD1
:100AD0008DED180AD4ED000A9DED020A20EE800A81
:100AE00094ED011ADDED010A01EE600A94ED031A9E
:100AF000DDED030A01EE200AF6EE000A20EE200AE0
:100B00008DED170AD4ED000A9DED010A20EE800A52
:100B100094ED011ADDED020A01EE200A94ED021AAD
:100B2000DDED030A01EE600AF6EE000A20EE200A6F
:100B30008DED160AF5EEC0EAF1EE10FA09D1F5EEE8
:100B4000C0DAF1EE10FA04D1B5EEC0FAF1EE10FA07
:100B50007ED06EEEAE0A4DEEAD0A4FEE0F0AB0EE4D
:100B6000600A07F0BDF8B0EE40AA2EEE8A0AF0EE59
:100B700040EA2DEE8A0AF0EE40DA2FEE0A0AB0EED5
:100B800040FA6BEE0B0A49EE090A49EEA90AB0EEEB
:100B9000600A07F0A5F8B0EE40AA2BEE0A0AB0EE04
:100BA00040BA29EE0A0AB0EE409A29EE8A0AF0EE1F
:100BB000409A94ED000AF0EE000A20EE200A20EEA2
:100BC0000B0A8DED130A94ED000AF0EE000A20EEF8
:100BD000200A20EE090A8DED120A94ED000AF0EECB
:100BE000000A20EE200A20EE290A8DED110A94ED6C
:100BF000010AF0EE000A20EE200A20EE0B0A8DED2D
:100C0000100A94ED000AF0EE000A20EE200A8DEDA5
:100C10000D0A94ED010AF0EE000A20EE200A8DED97
:100C20000C0A94ED020AF0EE000A20EE200A8DED87
:100C30000B0A94ED030AF0EE000A20EE200A8DED77
:100C40000A0A94ED000AF0EE000A20EE200A00E005
:100C5000FDE2D4ED020A20EE200A8DED090A94EDA2
:100C6000020AF0EE000A20EE200AD4ED030A20EE7C
:100C7000200A8DED080A94ED000A20EE000A8DEDA1
:100C8000070A94ED000AD4ED010A60EE20CA94ED43
:100C9000000AD4ED020A20EE20DA94ED000AD4ED29
:100CA000030A20EE200A8DED060A94ED010A20EEDB
:100CB00000CA94ED010AD4ED020A20EE200A8DED5F
:100CC000050A94ED010AD4ED030A60EE20BA94ED12
:100CD000020A60EE00AA94ED020AD4ED030A20EEA7
:100CE000200A8DED040A94ED030A20EE00EA9DED42
:100CF000070A6BEE000A94ED031A9DED120A40EE0E
:100D0000410A94ED021A9DED110A40EE010AB0EE7F
:100D1000600A0BEE0C0ADDED0C0A60EE890A94ED18
:100D2000021A00EE810ADDED0C0A60EEA90A94EDCC
:100D3000031A00EE810A0BEE6A0A0BEE4E0A8DEDE5
:100D4000150AD4ED030A9DED130A20EE800ADDEDAD
:100D5000070A09EE200A94ED011ADDED110A00EEF2
:100D6000C10A94ED021ADDED100A00EE810A09EEC7
:100D70004C0A09EE2A0ADDED0B0A60EEA90A94ED91
:100D8000031A00EE810A09EE4E0A8DED140ADDED1C
:100D9000150A20EEA01ADDED140A00EEA01AB0EE3E
:100DA000410A06F09DFFF7EE000A80EE808AD4ED3E
:100DB000020A9DED130AB1EE400A60EE800A94ED3E
:100DC000011A9DED120A40EE010A9DED070A49EE57
:100DD000800A94ED031A9DED100A40EE010A49EED7
:100DE000CC0A9DED0B0A20EE091AD4ED031AB0EEE1
:100DF000600A01EE210A03E09EEF273DB0000020CB
:100E000009EEEA0AF0EE408A49EE8E8AB0EE000A58
:100E100068EE000ACDED0F0AB0EE000A28EE800A57
:100E20008DED0E0A9DED090AF0EE000A10EEAB0AF8
:100E300070EE6E0A9DED0B0AB1EE400A20EE801AAC
:100E40009DED080AF0EE000A00EEAC0A70EE6D1A95
:100E5000DDED0C0AB0EE410A00EEA10AF6EE000A42
:100E600070EEEA0A70EECE0A60EE880A3BEECD1A0A
:100E700048EE810A70EECB0A94ED021A21EE281A90
:100E800001EE600AD4ED030AB1EE481A60EE811A51
:100E9000D4ED010A48EEA01ADDED050A9DED061A13
:100EA00070EEC10A20EE881ADDED040A7CEEA00A7D
:100EB00008EEA01A71EE490A01EEA00A7DEE2B0A97
:100EC00060EE880AB6EE001A31EE4C1A31EE6A1A5C
:100ED00048EE810A70EEE90A94ED021A21EE081A32
:100EE00001EE200A8DED1C0A9DED090AF0EE000AC4
:100EF00010EEAB0A70EE6E0A9DED0A0A60EE800AF3
:100F00009DED080AB0EE001A01EE2C0A30EE6D1AC3
:100F10009DED0D0A40EE010AB7EE000AB0EE001A90
:100F200001EE4C0AB0EE001A01EE6A0A30EE4F1ADA
:100F300094ED010AF1EE001A60EE211AB0EE600A9B
:100F400001EEC10AF6EE000A70EEEA0A70EECE0A71
:100F500060EE880A3BEECD1A48EE810A70EECB0AAD
:100F600094ED031A21EE281A01EE200AD4ED020AAC
:100F700060EE881AD4ED000A48EEA01ADDED050AED
:100F80009DED061A70EEC10A20EE881ADDED040A06
:100F90007CEEA00A08EEA01A71EE490A01EEA00A42
:100FA000D4ED030A20EE881AD4ED011ADDED0E0A05
:100FB00000EEE11A7DEE2B0A60EE880AF6EE001ACA
:100FC00071EECC1A71EEEA1A48EEA10A70EEE90A47
:100FD00001EE200AF0EE40FA9DED090AF0EE000A5B
:100FE00010EEAB0A70EE6E0A9DED0D0AB1EE400AEE
:100FF00060EE800A9DED080AB0EE001A01EE2C0AA0
:1010000030EE6D1A9DED0A0A40EE010AB7EE000AB5
:10101000B0EE001A01EE4C0AB0EE001A01EE6A0AB8
:1010200030EE4F1A94ED020AF1EE001A60EE211A2A
:10103000B0EE600A01EEC10A94ED021ADDED0F0A6E
:10104000F1EE600A61EE200A94ED001A48EEC10A42
:10105000B6EE001A31EE6A1A31EE4E1A21EE081A77
:101060007BEECD1A08EEA11A31EE4B1A00EE810A82
:10107000D4ED010A60EE881AD4ED030A48EEA01AF6
:10108000DDED050A9DED061A70EEC10A20EE881A04
:10109000DDED040A7CEEA00A08EEA01A71EE490A02
:1010A00001EEA00AD4ED000A20EE881AD4ED021A4F
:1010B000DDED0E0A00EEE11A7DEE2B0A60EE880AE5
:1010C000F6EE001A71EECC1A71EEEA1A48EEA10A99
:1010D00070EEE90A01EE200A8DED1B0A9DED090A6A
:1010E000F0EE000A10EEAB0A70EE6E0A9DED0C0AEF
:1010F00060EE800A9DED080AB0EE001A01EE2C0A9F
:1011000070EE6D1A9DED0B1AB0EE600A01EE210A29
:1011100094ED031ADDED0F0AF1EE600A61EE200A8C
:1011200094ED011A48EE810AB6EE001A31EE6A1A01
:1011300031EE4E1A21EE081A7BEECD1A08EEA11AF6
:1011400031EE4B1A00EE810AD4ED000AB1EE481AD6
:1011500020EE811AD4ED020A08EEA01ADDED050A90
:10116000DDED061A70EEE10A60EE881ADDED040A84
:101170007CEEA00A48EEA01A71EEC90A01EE200A20
:101180007DEE2B0A60EE880AB6EE001A31EE4C1A9C
:1011900031EE6A1A48EE810A70EEE90A94ED011AFE
:1011A00021EE081A01EE200A8DED1A0ADDED1C0A67
:1011B00060EEA00A4FEEAF0A9DED1B1A41EE010A48
:1011C0009DED1A1A41EE010AB0EE600A06F088FDA4
:1011D000B0EE40AA9DED1C0A20EE0A0A8DED1C0A15
:1011E0002FEE8A0AF0EE40FA9DED1B0A20EE0A0A65
:1011F0008DED1B0A9DED1A0A20EE0A0A8DED1A0AE2
:101200009DED190A414890ED001ADDED1C0A01EE32
:10121000600A8DED190A9DED180AD0ED000A00EE66
:10122000EF0A8DED180A9DED170A90ED001ADDED1D
:101230001B0A01EE600A8DED170A9DED160A90ED6E
:10124000001ADDED1A0A01EE600A8DED160AD4EDE2
:10125000000A94ED041A9DED190A40EE010AC4ED4E
:10126000000AD4ED010A94ED041A9DED180A40EE2F
:10127000010AC4ED010AD4ED020A94ED041A9DEDB1
:10128000170A40EE010AC4ED020AD4ED030A94EDF8
:10129000041A9DED160A40EE010AC4ED030AD4EDCE
:1012A000000A60EEA00A94ED011AD4ED011A41EE95
:1012B000210A94ED021AD4ED021A41EE210A94EDAE
:1012C000031AD4ED031A41EE210AB0EE600A06F0CB
:1012D00007FDB0EE40AA94ED000A20EE0A0A84ED64
:1012E000000A94ED010A20EE0A0A84ED010A94ED49
:1012F000020A20EE0A0A84ED020A94ED030A20EEA7
:101300000A0A84ED030A0020FFF76DBBB00000203D
:1013100070B52DED108B8CB004460D4616462CB9D9
:101320004FF0FF300CB0BDEC108B70BD15B94FF015
:10133000FF30F7E716B94FF0FF30F3E79FEDF30A00
:10134000F34880ED000A95ED009AD5ED018AD5EDC0
:10135000029A96ED00AAD6ED01AA96ED02BA94ED96
:10136000010AB1EE400A20EE0A0AD4ED020A00EEAC
:10137000EA0AD4ED030A00EECB0AF6EE000A20EEEC
:10138000200A8DED0B0A94ED000A20EE0A0AD4ED36
:10139000020A00EE8B0AD4ED030A00EEEA0AF6EE2A
:1013A000000A20EE200A8DED0A0A94ED000A20EED4
:1013B0002A0AD4ED010A00EECB0AD4ED030A00EEAE
:1013C0008A0AF6EE000A20EE200A8DED090A94ED55
:1013D000000A20EE0B0AD4ED010A00EEAA0AD4EDB1
:1013E000020A00EECA0AF6EE000A20EE200A8DED8F
:1013F000080AB5EEC09AF1EE10FA09D1F5EEC08AEE
:10140000F1EE10FA04D1F5EEC09AF1EE10FA7CD0AC
:1014100069EE090A48EEA80A49EEA90AB0EE600A88
:1014200006F05EFCB0EE408A29EE080AB0EE409A63
:1014300028EE880AF0EE408A29EE880AF0EE409AFB
:1014400094ED000AF0EE000A20EE200A8DED070A66
:1014500094ED010AF0EE000A20EE200A8DED060A56
:1014600094ED020AF0EE000A20EE200A8DED050A46
:1014700094ED030AF0EE000A60EE20FA94ED000A03
:10148000F1EE000A20EE200A8DED040A94ED010A27
:10149000F1EE000A20EE20EA94ED020AF1EE000AD5
:1014A00060EE20EA94ED010AF2EE000A20EE200A36
:1014B0008DED030A94ED020AF2EE000A20EE200AF6
:1014C0008DED020A94ED000A20EE000A8DED010A6E
:1014D00094ED010A60EE00BA94ED020A20EE00CA13
:1014E00094ED030A20EE000A8DED000A9DED040A3A
:1014F00020EE0C0ADDED050A00EE890ADDED040A96
:1015000000EEAB0ADDED060A00E0A0E000EEE80A1E
:10151000B0EE40FA9DED000A2EEE000A0FEEC90A69
:10152000DDED010AB1EE001A60EE810A94ED011AB8
:1015300000EE810ADDED070A00EEE80A70EE4E0AC1
:101540009DED030A40EE2B0A9DED030A40EE0C0AC6
:101550004EEE290AF0EE60CA9DED010AF1EE000A96
:1015600020EE200AD4ED020A20EE200ADDED070A63
:1015700000EE890ADDED000A0EEEA00A0FEEE80A81
:1015800030EE6E0ADDED020A00EEAB0ADDED020A76
:1015900000EE8C0A0EEEA90AB0EE40DAB1EE000AB7
:1015A0002BEE800AD4ED030A20EE200ADDED060AB8
:1015B00000EEC90AF1EE000A6CEE200A94ED031A5F
:1015C00000EE810ADDED050A00EEE80AF0EE40DAF1
:1015D0006FEE0F0A4CEEAC0A4DEE0D0A4DEEAD0A61
:1015E000B0EE600A06F07CFBB0EE408A2FEE080AEF
:1015F000B0EE40FA2CEE880AF0EE40CA2DEE080A52
:10160000B0EE40DA2DEE880AF0EE40DA9DED0B0ADE
:101610003F48D0ED000A00EECF0A8DED0B0A9DED9C
:101620000A0AD0ED000A00EEEC0A8DED0A0A9DEDE3
:10163000090AD0ED000A00EECD0A8DED090A9DEDF4
:10164000080AD0ED000A00EEED0A8DED080AD4ED8F
:10165000000A94ED041A9DED0B0A40EE010AC4ED58
:10166000000AD4ED010A94ED041A9DED0A0A40EE39
:10167000010AC4ED010AD4ED020A94ED041A9DEDAD
:10168000090A40EE010AC4ED020AD4ED030A94ED02
:10169000041A9DED080A40EE010AC4ED030AD4EDD8
:1016A000000A60EEA00A94ED011AD4ED011A41EE91
:1016B000210A94ED021AD4ED021A41EE210A94EDAA
:1016C000031AD4ED031A41EE210AB0EE600A06F0C7
:1016D00007FBB0EE408A94ED000A20EE080A84ED84
:1016E000000A94ED010A20EE080A84ED010A94ED47
:1016F000020A20EE080A84ED020A94ED030A20EEA5
:10170000080A84ED030A00200CE60000022B073DC6
:10171000B0000020B0EE401AB1EE600AB4EEC01A7C
:10172000F1EE10FA02D2B1EE600A7047B4EEE01AA0
:10173000F1EE10FA02DDB0EE600AF6E7B0EE410A13
:10174000F3E7000010B504210248006809F096FD97
:1017500010BD0000C000002010B51323034A122161
:10176000002000F0D5F9002010BD0000507C0020C2
:1017700010B54FF0FF320121084609F0BFFD10BD42
:101780009FED010A704700000000C84310B5082112
:101790000248006809F072FD10BD0000C000002082
:1017A00010B50623034A0221012000F0B1F9002000
:1017B00010BD0000577C002010B54FF0FF32012112
:1017C000022009F09BFD10BD70B504460D4614B90A
:1017D0006FF0010070BD15B96FF00100FAE74448E1
:1017E000007810B16FF00200F4E709F0E0FD414924
:1017F000086010B96FF00100ECE7E562B6227E21C7
:10180000002000F0EBF9B6221421012000F0E6F9E7
:101810001E2000F01FFF1E21002000F0A5F900216E
:10182000084600F0A1F91E2802D06FF00300D1E7AE
:101830000021012000F098F90F2802D06FF003007A
:10184000C8E7032000F09AFD042000F097FD2A4A23
:101850000121002000F0C6FE2849032000F0E4FD2D
:101860002749042000F0E0FDAA224021002000F0DA
:10187000B5F901224121002000F0B0F908225321DE
:10188000002000F0ABF904225821002000F0A6F956
:1018900004227D21002000F0A1F9322000F0DAFEC0
:1018A00001220F21104600F099F903221021012096
:1018B00000F094F900221621012000F08FF9012296
:1018C0001821104600F08AF980221521012000F02D
:1018D00085F90A2000F0BEFE0120054908700320AA
:1018E00000F06CFD042000F069FD002072E70000AC
:1018F000C4000020C0000020C51A000845170008D9
:101900008D1700080EB5014611B96FF001000EBD2C
:101910002B48B0F8010002902948B0F8030001906C
:101920002748B0F805000090BDF9080000EE100A45
:10193000B8EEC00A81ED040ABDF9040000EE100AF9
:10194000B8EEC00A81ED050ABDF9000000EE100AEC
:10195000B8EEC00A81ED060A91ED040ADFED190A1E
:1019600080EE201A81ED041A91ED050ADFED150ACB
:1019700080EE201A81ED051A91ED060ADFED110ABD
:1019800080EE201A81ED061A0D48407CC0000C4BF9
:101990009B7C40EA6312B2F5806F02DBA2F5006027
:1019A00002B200EE102AF8EEC00AB4EE001AB3EE4E
:1019B000070A00EE810A81ED0A0A0020A7E700006D
:1019C000507C002000A0AA450EB5014611B96FF069
:1019D00001000EBD3848B0F8070002903648B0F854
:1019E000090001903448B0F80B000090BDF90800E0
:1019F00000EE100AB8EEC00A81ED070ABDF9040036
:101A000000EE100AB8EEC00A81ED080ABDF9000028
:101A100000EE100AB8EEC00A81ED090A91ED070A3E
:101A2000DFED260A80EE201A81ED071A91ED080AF3
:101A3000DFED220A80EE201A81ED081A91ED090AE5
:101A4000DFED1E0A80EE201A81ED091A91ED070ADA
:101A5000DFED1B0A20EE200A81ED070A91ED080A4E
:101A6000DFED170A20EE200A81ED080A91ED090A40
:101A7000DFED130A20EE200A81ED090A91ED070A35
:101A8000C86AD0ED000A30EE600A81ED070A91EDD8
:101A9000080AC86AD0ED010A30EE600A81ED080A32
:101AA00091ED090AC86AD0ED020A30EE600A81EDB4
:101AB000090A6FF001008CE7507C00206F1203428E
:101AC00035FA8E3C10B5012000F098FC40B9012198
:101AD000084600F0CDFC01210848006809F0CEFB63
:101AE000022000F08BFC40B90121022000F0C0FC74
:101AF00002210248006809F0C1FB10BDC0000020AF
:101B000010B54FF0FF3201210C2009F0F7FB10BD9A
:101B10002DE9F04105460E4614461F460CB9BDE8B6
:101B2000F08115B1012D0AD104E00021012000F05F
:101B30009FFC04E00021022000F09AFC00BF00BFDF
:101B400046F080000749087000230122184600F083
:101B500057FD01233A462146002000F019FD00BF41
:101B6000DDE70000BC00002070B504460D460120F2
:101B700000F070FD14B1012C0AD104E00021012015
:101B800000F076FC04E00021022000F071FC00BFB0
:101B900000BF45F08000104908700023012218465C
:101BA00000F02EFD002302220B49184600F0F0FC45
:101BB00014B1012C0ED106E00121084600F058FCBA
:101BC0000548407870BD0121022000F051FC024818
:101BD0000078F7E700BFF5E7BC00002070B50446C9
:101BE0000E46154606F07F001549087008464570F8
:101BF000012000F02FFD14B1012C0AD104E00021D6
:101C0000012000F035FC04E00021022000F030FC4F
:101C100000BF00BF002302220949184600F0F0FC73
:101C200014B1012C0AD104E00121084600F020FC87
:101C300004E00121022000F01BFC00BF00BF70BDCA
:101C4000BC0000202DE9F04107468846164606B93B
:101C50000A2664212348006809F05EFA18B16FF083
:101C60000400BDE8F081204805680DE02878B842FE
:101C700009D16868404506D11A48006809F0D6FACB
:101C80004FF0FF30EDE72D69002DEFD1142000F06B
:101C900005FC04462CB91348006809F0C7FAA81ED1
:101CA000DFE700221C21304609F092F9A060A0680D
:101CB00048B9204600F05CFB0A48006809F0B6FA13
:101CC0004FF0FF30CDE72770C4F804802673064834
:101CD00000682061044804600248006809F0A6FA20
:101CE0000020BEE7A4000020A000002070470000F4
:101CF00002460B460748016808E00878904204D184
:101D00004868984201D18868704709690029F4D170
:101D10000020F9E7A00000200146C868022806D18B
:101D20008868042801D1032070470220FCE78868F6
:101D3000042801D10120F7E70020F5E70146022938
:101D400001DB0020704711B1012904D101E00348F3
:101D5000F8E70348F6E70020F4E70000200200203F
:101D6000480200202DE9F047074688461446994668
:101D70001648007818B96FF00200BDE8F08714B972
:101D80006FF00100F9E764211148006809F0C4F917
:101D900010B16FF00400F0E741463846FFF7A8FFA6
:101DA00005460B48006809F041FA15B96FF00300C9
:101DB000E3E74B4600222146284609F0C9F80646CB
:101DC0000EB90020D9E74FF0FF30D6E7A800002079
:101DD000A400002010B58AB03F48007818B16FF019
:101DE00002000AB010BD68213C48FEF7B3FB002496
:101DF00003E0E0B200F03AFA641C022CF9DB384848
:101E000038490860002009F0B8F9374908600846E9
:101E1000006810B94FF0FF30E3E701202E49087049
:101E200028216846FEF796FB00200590009001905F
:101E30000690012007900020029003900120089056
:101E40000E200990002004906946284801F0DAF934
:101E5000264801F0C5FE264A0621002000F064F85D
:101E6000244A0021084600F05FF8224A01210020A0
:101E700000F05AF81F4A0221002000F055F8032113
:101E80001A4801F005F90E200590012004906946DA
:101E9000194801F0B7F9184801F0A2FE174A0821C5
:101EA000012000F041F8134A0021012000F03CF825
:101EB000104A0121084600F037F80E4A022101209D
:101EC00000F032F811210C4801F0E2F8012002493B
:101ED0000870002085E70000A8000020EC720020B8
:101EE000ED1C0008AC000020A4000020200200200F
:101EF000991F000815220008480200204920000808
:101F000070B504460D460748006828B129462046AA
:101F1000044A1268904770BD29462046FFF7E6FE46
:101F2000F9E70000AC00002010B503460F48007828
:101F300010B96FF0020010BD12B96FF00100FAE79E
:101F4000022B02DB4FF0FF30F5E70D2902DB4FF0EB
:101F5000FF30F0E703EB830000EBC300044C04EB1D
:101F6000800040F821200020E5E70000A8000020C4
:101F7000EC72002070B504460D4616460548007800
:101F800010B96FF0020070BD324629462046FFF7B7
:101F900059FEF8E7A80000202DE9F04391B0002495
:101FA0004DE0E0B2FFF7CAFE8046B8F1000F00D165
:101FB00044E03CE008AB0AAA0021404601F0E4F905
:101FC000002834D10C9808B90A9800E00B98814693
:101FD0000AA8FFF7A1FE054629464846FFF790FFED
:101FE0000646E0B23146FFF783FE0746F7B11C21F3
:101FF00001A8FEF7AFFA8DF80450CDF808900396CB
:102000000E98C0B28DF810000D9828B908A90DF1EE
:1020100011000E9AFEF71FFA02F072FA07900023E1
:102020001A4601A9384609F021F800BF00BF002177
:10203000404601F095F90028BCD100BF641C022C79
:10204000AFDB11B0BDE8F0832DE9F04391B000247F
:102050004DE0E0B2FFF772FE8046B8F1000F00D10C
:1020600044E03CE008AB0AAA0121404601F08CF9AB
:10207000002834D10C9808B90A9800E00B988146E2
:102080000AA8FFF749FE054629464846FFF738FFEC
:102090000646E0B23146FFF72BFE0746F7B11C219A
:1020A00001A8FEF757FA8DF80450CDF80890039672
:1020B0000E98C0B28DF810000D9828B908A90DF13E
:1020C00011000E9AFEF7C7F902F01AFA07900023E2
:1020D0001A4601A9384608F0C9FF00BF00BF012118
:1020E000404601F03DF90028BCD100BF641C022C21
:1020F000AFDB11B0BDE8F0832DE9F0478AB081462F
:102100000D4614461E46129F3948007820B96FF0DC
:1021100002000AB0BDE8F087B9F1020F02DB4FF010
:10212000FF30F6E736B9022D04D0032D02D06FF050
:102130000100EEE7082F02DD4FF0FF30E9E74846E7
:10214000FFF7FCFD8046B8F1000F02D16FF00100EF
:10215000DFE7202102A8FEF7FDF935B1012D09D0F6
:10216000022D0DD0032D17D110E002940020049011
:10217000059014E0039404200490002005900EE0E4
:102180000294002004900220059008E003940420AB
:1021900004900220059002E04FF0FF30B9E700BF45
:1021A000069700208DF81C0036B1002F04DD3A465A
:1021B000314608A8FEF74FF9404601F0AFF960B18B
:1021C00001AB08AA02A9404600F077FF8246BAF1A7
:1021D000000F01D100209CE700BF02A9484600F093
:1021E0009FF808B1002094E74FF0FF3091E700001E
:1021F000A800002038B505460C4614B96FF0010060
:1022000038BD20790090631D002128462268FFF721
:1022100073FFF5E770B58AB0002422E0E6B23046DD
:10222000FFF78CFD054605B91AE012E0284601F0DB
:1022300075F900B912E002A9304600F049F800B97A
:102240000CE001AB08AA02A9284600F036FF00B155
:1022500004E0304600F020F80028E7D000BF00BFBF
:10226000641C022CDADB0AB070BD0000022800DB1F
:102270007047002100EBC012064B03EBC202C2F80C
:10228000001400EBC01203EBC202C2F8041400BF3A
:10229000EEE70000547300200146022901DB012013
:1022A000704701EBC110094A02EBC000D0F80004EE
:1022B00001EBC112054B03EBC202D2F80424904299
:1022C00001D10120ECE70020EAE700005473002070
:1022D00070B505460E46022D00DA0EB9002070BD1D
:1022E00005EBC5100D4901EBC004D4F80004D4F887
:1022F0000414884201D10020F1E7D4F8040404EB6F
:10230000401120223046FEF7EBF8D4F80404401CBC
:1023100000F01F00C4F804040120E0E7547300201B
:102320002DE9F04105460F46022D00DA17B90020CD
:10233000BDE8F08105EBC5100C4901EBC004D4F8F1
:102340000004401C00F01F06D4F80404B04201D180
:102350000020EDE7D4F8001404EB411020223946A8
:10236000FEF7BEF8C4F800640120E1E754730020D2
:1023700010B5044620460AF0CBF810BD10B504464F
:1023800034B1032C08D0042C0AD0052C10D10BE05A
:10239000062002F0EBFC0EE00A2002F0E7FC0AE067
:1023A000172002F0E3FC06E0092002F0DFFC02E067
:1023B0004FF0FF3010BD00BF0020FBE710B5044612
:1023C00034B1032C08D0042C0AD0052C10D10BE01A
:1023D000062002F0E1FC0EE00A2002F0DDFC0AE03B
:1023E000172002F0D9FC06E0092002F0D5FC02E03B
:1023F0004FF0FF3010BD00BF0020FBE710B50446D2
:10240000072C01DB002010BD064A32F8341002EB25
:10241000C402506802F066F8012800D1F3E70020FA
:10242000F1E7000038ED000810B5024611B96FF071
:10243000010010BD072A02DB4FF0FF30F9E70A4820
:1024400030F83230002009E0012484401C401CB1E7
:10245000064C44F8201003E0441CE0B21028F3DBE3
:1024600000BF0020E5E7000038ED0008647B002095
:1024700070B504460D46072C02DB4FF0FF3070BDEF
:10248000054A32F8341002EBC40250682A4602F0C2
:1024900031F80020F3E7000038ED000810B50446DD
:1024A000204609F033FD10BD0146012902DB4FF043
:1024B000FF307047F7EE000AB4EEE00AF1EE10FAD2
:1024C00003DDF7EE000AB0EE600AB5EEC00AF1EEE9
:1024D00010FA03D2DFED1E0AB0EE600A1D4850F874
:1024E00031000068C36A581C00EE900AF8EE600ADA
:1024F00060EE200AFCEEE00A10EE902A154800EB90
:10250000C100808828B9134850F831000068426340
:102510001CE0104800EBC1008088042805D10D485C
:1025200050F831000068826310E00A4800EBC100F7
:102530008088082805D1074850F831000068C26338
:1025400004E0044850F83100006802640020B0E75D
:102550000000000070ED000810B50446012C02DBFD
:102560004FF0FF3010BD054A02EBC4029188034AC8
:1025700052F8340004F014F90020F3E770ED00087D
:10258000014609B9014870470020FCE71803002004
:102590002DE9F04105460F4690461E46022D03DB0D
:1025A0004FF0FF30BDE8F0812846FFF7E9FF044611
:1025B00014B94FF0FF30F5E74EB142463946204698
:1025C00003F006FA08B10120ECE70020EAE7142343
:1025D00042463946204603F039F908B10120E1E7C7
:1025E0000020DFE7034612B96FF00100704703488F
:1025F00000EB431040F821200020F7E7EC7B00209F
:102600002DE9F04105460F4690461E46022D03DB9C
:102610004FF0FF30BDE8F0812846FFF7B1FF0446D8
:1026200014B94FF0FF30F5E74EB142463946204627
:1026300003F048FD08B10120ECE70020EAE714238D
:1026400042463946204603F087FA08B10120E1E707
:102650000020DFE770B5044608F0F3FB4FF47A7111
:10266000B1FBF0F5B4FBF5F608F0C4FB022816D078
:1026700006DCB0F1FF3F0CD0C8B101281CD117E037
:10268000032808D0042807D06FF00041401A13D166
:1026900000E000BF00BF00BF4FF0FF3070BD0EB1C3
:1026A000314600E00121084608F07BFB04E000BF52
:1026B000204601F0E3FD00BF00BF0020EEE72DE95A
:1026C000F04108F0BEFB05460BF03EFA4FF47A717C
:1026D000B1FBF5F100FB01F64FF0E02087690BF04C
:1026E00033FA4FF47A71B1FBF5F100FB01F44FF0CE
:1026F000E020D0F81880A64214D14FF47A707843C5
:102700004FF0E0214969491CB0FBF1F004EB4401B2
:10271000C1EBC4114FF47A7202EBC101081A002117
:10272000BDE8F0814FF47A7008FB00F04FF0E02133
:102730004969491CB0FBF1F004EB4401C1EBC41141
:102740004FF47A7202EBC101081A0021E8E7000099
:1027500038B504462068006800F0100010281ED12B
:1027600000BF00200090206800680090206840684A
:10277000009000BF00BF204607F0E8F800EBC00063
:10278000074901EB8000006A48B1204607F0DEF8F7
:1027900000EBC000024901EB8000056AA84738BD84
:1027A0002C7C002000BFFEE710B5024800F0D1FEEF
:1027B00010BD00002002002010B5024800F0C9FE44
:1027C00010BD00002002002010B5024800F0C1FE3C
:1027D00010BD00002002002010B5024800F0B9FE34
:1027E00010BD00004802002010B5024800F0B1FE04
:1027F00010BD00004802002010B5024800F0A9FEFC
:1028000010BD000048020020014609B903207047AE
:10281000064A0868904201D10020F8E7044A086897
:10282000904201D10120F2E70320F0E7006400406C
:1028300000680040B0EE401AD0ED001A71EE811A27
:10284000B0EE610AF5EEC00AF1EE10FA12DDB4EE58
:10285000E00AF1EE10FA04DB70EE601AB0EE610AE5
:1028600008E0B5EEC00AF1EE10FA03D270EE201ABD
:10287000B0EE610A80ED000A7047F0EE401A31EECA
:10288000E02AB0EE420AB5EEC01AF1EE10FA1BDDF6
:10289000F0EE002A81EE223AB0EE432AB4EEC20AEC
:1028A000F1EE10FA04DD70EE412AB0EE620A0AE0A1
:1028B000F1EE422AB4EEE20AF1EE10FA03D270EE23
:1028C000012AB0EE620A00BF70470000004870475E
:1028D000D000002010B500F007F8024801F0EEFA31
:1028E00010BD0000A805002010B50C48006800F4D9
:1028F000006088B10A4800780F2803D0192006F03C
:1029000065FA03E00749064809F018FC03488068A7
:1029100040F400600149886010BD00000060024082
:102920007B7C0020637C002010B5024801F0C6FAD1
:1029300010BD0000C803002010B5024801F0BEFA27
:1029400010BD000028040020014608781038182324
:10295000B0FBF3F20848805CC865032A05D9086813
:102960006FF30900001D886503E008686FF3090034
:102970008865886D7047000018ED0008014600204A
:102980008A6A8B69CBB932B1012A0DD0022A03D0F1
:10299000032A10D10EE000BFCB6A03F08073B3F1BD
:1029A000807F00D1012007E0CB6AB3F1C07F00D166
:1029B000012001E000E000BF34E08B69B3F5005F67
:1029C0001AD132B1012A07D0022A03D0032A11D129
:1029D0000AE000BF01200EE0CB6A03F08073B3F180
:1029E000807F00D1012006E0CB6AB3F1C07F00D127
:1029F000012000E000BF15E032B1012A05D0022A13
:102A000004D0032A0CD103E000BF00BF012008E07E
:102A1000CB6A03F08073B3F1807F00D1012000E026
:102A200000BF00BF704730B50468246824F48024D8
:102A300005682C60046863608468402C04D10468D5
:102A4000A2600468E16003E00468A1600468E260D9
:102A500030BD704710B5012001F03CFC10BD10B531
:102A6000082001F037FC10BD10B5102001F032FC39
:102A700010BD10B5202001F02DFC10BD72B600BFB6
:102A8000FEE700002DE9F0412DED088B04460D46D0
:102A900004B12DB94FF0FF30BDEC088BBDE8F081DB
:102AA000FFF70DFED4E90023861A61EB03013046DF
:102AB0000CF09FF800EE100ADFEDCD0A80EE201A30
:102AC00084ED021AFFF7FBFDC4E9000129782046D6
:102AD00000F05CFA95ED010AD4ED020A20EE208A9E
:102AE00095ED020AD4ED020A60EE20BA95ED010AD6
:102AF000D4ED020A60EE208A95ED020AD4ED020AB6
:102B000020EE209A207C20B101280DD002280AD185
:102B1000C3E09FEDB80A84ED9F0A9FEDB60A04F565
:102B20001F7084EDA00A60E194ED050A30EE280ADA
:102B300084ED050AE06890ED480AB5EEC00AF1EEB2
:102B400010FA1ADD94ED050AD4ED870AB4EEE00A16
:102B5000F1EE10FA03DD94ED870A84ED050A94ED99
:102B6000050AD4ED880AB4EEE00AF1EE10FA1DD29F
:102B700094ED880A84ED050A18E0DFED9F0AB0EEB7
:102B8000680A04F11400FFF755FE94ED050ADFED25
:102B90009B0AB4EEE00AF1EE10FA07DD94ED050AA7
:102BA000DFED950A30EE600A84ED050A94ED060A21
:102BB00030EE090A84ED060AE06890ED490AB5EEA8
:102BC000C00AF1EE10FA19DD94ED060AD4ED890A77
:102BD000B4EEE00AF1EE10FA03DD94ED890A84ED1B
:102BE000060A94ED060AD4ED8A0AB4EEE00AF1EE84
:102BF00010FA03D294ED8A0A84ED060A94ED021AC3
:102C0000F0EE411A94EDA41AF0EE410A94ED051A83
:102C1000B0EE410A9FED771A04F12C0005F03CFF5D
:102C2000F0EE409A94ED020AF0EE401A94EDA30AF9
:102C3000F0EE400A9FED6F1AB0EE690A04F16800E9
:102C400005F02AFF84ED9F0A94ED021AF0EE411A76
:102C500094EDA51AF0EE410A94ED061AB0EE410A81
:102C60009FED641A04F1A40005F016FFB0EE40AA2F
:102C700094ED020AF0EE401A94EDA10AF0EE400A3B
:102C80009FED5C1AB0EE4A0A04F1E00005F004FF83
:102C900004F51F7084EDA00AA7E094ED080A30EE59
:102CA000080A84ED080AE06890ED480AB5EEC00A0B
:102CB000F1EE10FA1ADD94ED080AD4ED8B0AB4EEA9
:102CC000E00AF1EE10FA03DD94ED8B0A84ED080AB8
:102CD00094ED080AD4ED8C0AB4EEE00AF1EE10FA95
:102CE0000CD294ED8C0A84ED080A07E0DFED420A6D
:102CF000B0EE480A04F12000FFF79CFD94ED090AAC
:102D000030EE090A84ED090AE06890ED490AB5EE53
:102D1000C00AF1EE10FA19DD94ED090AD4ED8D0A1E
:102D2000B4EEE00AF1EE10FA03DD94ED8D0A84EDC5
:102D3000090A94ED090AD4ED8E0AB4EEE00AF1EE28
:102D400010FA03D294ED8E0A84ED090A94ED021A6A
:102D5000F0EE411A94EDA71AF0EE410A94ED081A2C
:102D6000B0EE410A9FED231A04F5AC7005F094FE15
:102D7000F0EE40AA94ED020AF0EE401A94EDA80A93
:102D8000F0EE400A9FED1B1AB0EE6A0A04F58E7051
:102D900005F082FE84ED9F0A94ED021AF0EE411ACE
:102DA00094EDAB1AF0EE410A94ED091AB0EE410A27
:102DB0009FED101A04F5E87005F06EFEB0EE40BA13
:102DC00094ED020AF0EE401A94EDAC0AF0EE400ADF
:102DD0009FED081AB0EE4B0A04F5CA7005F05CFED0
:102DE00004F51F7084EDA00A00BF00BF00BF53E6CA
:102DF0000024744900000000DB0FC940DB0F49408C
:102E000070B52DED028B04460D46B0EE408A24B914
:102E10004FF0FF30BDEC028B70BDE56000202074E8
:102E2000E06800F13002B0EE480A012104F12C0004
:102E300005F004FFE06800F11002B0EE480A01213D
:102E400004F1680005F0FAFEE06800F17002B0EEEF
:102E5000480A012104F1A40005F0F0FEE06800F149
:102E60005002B0EE480A012104F1E00005F0E6FE50
:102E7000E06800F1B002B0EE480A012104F5AC7040
:102E800005F0DCFEE06800F19002B0EE480A012196
:102E900004F58E7005F0D2FEE06800F1F002B0EEAD
:102EA000480A012104F5E87005F0C8FEE06800F169
:102EB000D002B0EE480A012104F5CA7005F0BEFE4A
:102EC000E06890ED440AF0EE400AB0EE480A04F5DE
:102ED0000F7004F06DFFE06890ED440AF0EE400AD8
:102EE000B0EE480A04F5177004F062FFE06890ED58
:102EF0004C0A84ED890AE06890ED4D0A84ED8A0A57
:102F0000E06890ED4E0A84ED870AE06890ED4F0A84
:102F100084ED880AE06890ED500A84ED8D0AE0683F
:102F200090ED510A84ED8E0AE06890ED520A84ED2E
:102F30008B0AE06890ED530A84ED8C0AFEF74AFF95
:102F4000E16801F1080005F01BF9E06805F018F9E7
:102F500000205FE710B50446E06805F00BF8E16873
:102F600001F1080005F006F8D4ED9F0AB0EE600A02
:102F7000E16801F1080005F063F9D4EDA00AB0EEB4
:102F8000600AE06805F05CF910BD000070B5044609
:102F90000D4614B94FF0FF3070BD207CA84201D11E
:102FA0000020F9E704F12C0005F0AEFE04F1680002
:102FB00005F0AAFE04F1A40005F0A6FE04F1E0006D
:102FC00005F0A2FE9FED110A04F50F7004F07AFFE0
:102FD0009FED0E0A04F5177004F074FF04F114005D
:102FE000FDF7F0FC94EDA50A84ED060A94EDA40A21
:102FF00084ED050A94EDAB0A84ED090A94EDA70A65
:1030000084ED080A25740020C6E7000000000000D7
:103010002DE9F04104461CB94FF0FF30BDE8F081C6
:10302000E16801F1080005F064F9E06805F061F974
:10303000E16801F1080005F070F80646E06805F067
:103040006CF8054605B966B104F5217006F1080172
:103050008EC918308EC0283805F108018EC9283075
:103060008EC00020DAE730B5024612B94FF0FF30CB
:1030700030BD02F5207091E83800001D38C00C38D2
:10308000D1E90445CB68C0E90445C36000BFEFE760
:1030900010B5024692F82030012B01D0022B06D148
:1030A00010684069084314686061002010BD506AD0
:1030B00040F4802050620120F8E7F0B504460D4648
:1030C0001E4694F8207020688368A86800B900E064
:1030D00000BF012F01D0022F7DD103F0806030B9F5
:1030E00003F0006018B903F0805000287ED0C3F3CD
:1030F0000161012088403060A86860B9B5F800C05F
:10310000E86840EA4C5C206800F5C07000EB0110F4
:10311000C0F800C00FE0D5E901C040EACC00D5F806
:103120000CC040EA0C00D4F800C00CF5C07C0CEBDD
:10313000011CCCF80000D5F810C0206800F5C07064
:1031400000EB0110C0F804C0287D01280ED12068D2
:1031500000F5C07000EB0110406840F4807C2068EE
:1031600000F5C07000EB0110C0F804C0D079000673
:1031700092F806C040EA0C4092F805C040EA0C20E4
:1031800092F804C040EA0C00D4F800C00CF5C07CF2
:103190000CEB011CCCF80C00D078000692F802C0B1
:1031A00040EA0C4092F801C040EA0C2092F800C0BE
:1031B00040EA0C00D4F800C00CF5C07C0CEB011CFC
:1031C000CCF80800206800F5C07000EB0110006822
:1031D00040F0010C01E00FE008E0206800F5C0704D
:1031E00000EB0110C0F800C00020F0BD606A40F4A0
:1031F000001060620120F8E7606A40F4802060629D
:103200000120F2E7F0B504460A4694F82050012D5B
:1032100001D0022D7ED1424901F50071086840F0CD
:1032200001000860086820F47C5008600868566A4D
:1032300040EA06200860107D00F01F06012000FA19
:1032400006F3C8699843C861A1F50071D069C8B98F
:10325000D1F80C029843C1F80C02908880B296898C
:1032600040EA064601F51070576940F8376010884B
:1032700080B2168940EA064601F51070576900EBE6
:10328000C7004660D069012819D1D1F80C02184353
:10329000C1F80C02908880B2168840EA064601F513
:1032A0001070576940F83760908980B2168940EAFB
:1032B000064601F51070576900EBC700466090693B
:1032C00028B9D1F804029843C1F8040204E0D1F807
:1032D00004021843C1F80402106928B9D1F8140295
:1032E0009843C1F8140204E0D1F814021843C1F85D
:1032F0001402106A012804D1D1F81C021843C1F845
:103300001C02D1F8000220F00100C1F800020020E8
:10331000F0BDFFE7606A40F4802060620120F7E7BB
:103320000064004070B505462846FFF76DFA044674
:10333000032C11D004EB840000EBC400074901EB1F
:103340008000006B40B104EB840101EBC401034A2F
:1033500002EB8101086B804770BD0000EC72002019
:1033600010B50246002092F82030012B01D0022B2C
:1033700009D121B91468E46804F0030003E014687B
:10338000246904F0030010BD70B5044694F8205081
:10339000012D01D0022D7DD151B92068C06800F007
:1033A000030080B9606A40F400106062012070BDC3
:1033B0002068006900F0030028B9606A40F400103A
:1033C00060620120F3E7206800F5D87000EB01107F
:1033D000006800F004009060906840B9206800F533
:1033E000D87000EB01100068400D106007E0206805
:1033F00000F5D87000EB01100068C008506020682C
:1034000000F5D87000EB0110006800F00200D060F9
:10341000206800F5D87000EB0110406800F00F0044
:10342000082802D30820106108E0206800F5D87051
:1034300000EB0110406800F00F001061206800F5FB
:10344000D87000EB0110406800F47F40000A9061E2
:10345000206800F5D87000EB01104068000C506146
:10346000206800F5D87000EB0110806818702068A3
:1034700000F5D87000EB0110806800F47F40000A6E
:103480005870206800F5D87000EB0110806800F4D7
:103490007F0000E03CE0000C9870206800F5D870D8
:1034A00000EB01108068000ED870206800F5D8701D
:1034B00000EB0110C0681871206800F5D87000EBAF
:1034C0000110C06800F47F40000A5871206800F5C0
:1034D000D87000EB0110C06800F47F00000C9871F8
:1034E000206800F5D87000EB0110C068000ED8719C
:1034F00031B92068C06840F020002668F06005E01F
:103500002068006940F020002668306100204EE706
:10351000606A40F480206062012048E70146002094
:1035200091F82020012A01D0022A11D10B689B6852
:1035300003F0806303B1401C0B689B6803F00063D9
:1035400003B1401C0B689B6803F0805303B1401C1F
:1035500070472DE9F05F0446002520684669206821
:10356000D0F80490206887682068D0F80CA0206804
:10357000D0F810B02068D0F8188006F001000028BC
:1035800055D007F00100C0B101202168886007F024
:10359000020018B1204600F071FB0EE007F00400B5
:1035A00010B145F4006508E007F0080010B145F4DB
:1035B000805502E0204600F043FB07F48070C8B15C
:1035C0004FF480702168886007F4007018B12046BD
:1035D00000F08EFB0EE007F4806010B145F400555A
:1035E00008E007F4006010B145F4804502E0204691
:1035F00000F060FB07F48030C8B14FF480302168E0
:10360000886007F4003018B1204600F0ADFB0EE0F2
:1036100007F4802010B145F4004508E007F40020CD
:1036200010B145F4803502E0204600F07FFB06F043
:10363000080038B10AF0100020B145F400751020E0
:103640002168C86006F0040040B10AF0080028B103
:1036500008202168C860204600F02CFA06F002001D
:1036600038B12068C06800F0030010B1204600F0B7
:103670003FFA06F0400038B10BF0100020B145F4DD
:10368000806510202168086106F0200040B10BF031
:10369000080028B1082021680861204600F046FA99
:1036A00006F0100038B12068006900F0030010B186
:1036B000204600F059FA06F4003040B109F010003D
:1036C00028B1102021684860204600F06BFA06F40B
:1036D000803040B109F0080028B108202168486016
:1036E000204600F05FFB06F4004088B309F00400B8
:1036F00078B306F4807020B108F0010008B145F0FD
:10370000010506F4007020B108F0020008B145F090
:10371000020506F4806020B108F0040008B145F00D
:10372000040506F40060A0B108F0700088B108F04C
:103730007000402817D006DC10280BD020280CD0B1
:10374000302819D10CE0502810D0602814D110E096
:103750001DE019E045F008050FE045F010050CE00C
:1037600045F0200509E045F0400506E045F08005FC
:1037700003E045F4807500E000BF00BF2068806969
:1037800020F07000216888610420216848602DB114
:10379000606A284360622046FFF7C4FDBDE8F09FE1
:1037A00070B504460CB9012070BD94F8200010B922
:1037B000204600F0AFF82068006840F00100216862
:1037C000086000F09DFE05460DE000F099FE401BEC
:1037D0000A2808D9606A40F400306062052084F845
:1037E00020000120E0E72068406800F00100002888
:1037F000EBD02068006820F002002168086000F02B
:103800007FFE05460DE000F07BFE401B0A2808D92C
:10381000606A40F400306062052084F820000120D6
:10382000C2E72068406800F002000028EBD1207E4B
:10383000012806D12068006840F0800021680860F7
:1038400005E02068006820F0800021680860607E44
:10385000012806D12068006840F040002168086017
:1038600005E02068006820F0400021680860A07E24
:10387000012806D12068006840F020002168086017
:1038800005E02068006820F0200021680860E07EE4
:10389000012806D12068006820F010002168086027
:1038A00005E02068006840F0100021680860207F73
:1038B000012806D12068006840F0080021680860EF
:1038C00005E02068006820F0080021680860607F3B
:1038D000012806D12068006840F0040021680860D3
:1038E00005E02068006820F0040021680860D4E941
:1038F0000201084321690843616908436168491E60
:1039000008432168C86100206062012084F820001B
:10391000002049E710B586B00446142101A8FCF741
:1039200019FE5E492068884251D15D480068401CFC
:103930005B4908600846006801280FD100BF0020DD
:1039400000905848006840F00070564908600846EA
:10395000006800F00070009000BF00BF00BF0020B2
:10396000009050481038006840F008004D49103968
:1039700008600846006800F00800009000BF00BF23
:103980000320019002200290002003900320049065
:103990000920059001A9444800F0AAFC0022052155
:1039A000132001F00DFA132001F0F6F90022052191
:1039B000142001F005FA142001F0EEF9002205218F
:1039C000152001F0FDF9152001F0E6F964E0374912
:1039D0002068884260D100BF002000903148006814
:1039E00040F080602F4908600846006800F0806061
:1039F000009000BF00BF2A480068401C28490860AA
:103A00000846006801280FD100BF0020009025481B
:103A1000006840F00070234908600846006800F024
:103A20000070009000BF00BF00BF002000901D4844
:103A30001038006840F002001A4910390860084642
:103A4000006800F00200009000BF00BF60200190FD
:103A5000022002900020039003200490092005908A
:103A600001A9134800F044FC002205213F2001F089
:103A7000A7F93F2001F090F900220521402001F034
:103A80009FF9402001F088F900220521412001F032
:103A900097F9412001F080F906B010BD00640040A4
:103AA0000400002040380240000C02400068004042
:103AB0000004024070B505462846FEF7A5FE044600
:103AC000032C11D004EB840000EBC400074901EB88
:103AD0008000C06940B104EB840101EBC401034ADA
:103AE00002EB8101C869804770BD0000EC720020C4
:103AF00070B505462846FEF787FE0446032C11D014
:103B000004EB840000EBC400074901EB80008069EE
:103B100040B104EB840101EBC401034A02EB8101D3
:103B20008869804770BD0000EC72002070B50546C2
:103B30002846FEF769FE0446032C11D004EB8400EE
:103B400000EBC400074901EB8000406A40B104EB80
:103B5000840101EBC401034A02EB8101486A8047FA
:103B600070BD0000EC72002070B505462846FEF7D7
:103B70004BFE0446032C11D004EB840000EBC40080
:103B8000074901EB8000006A40B104EB840101EBBE
:103B9000C401034A02EB8101086A804770BD00003E
:103BA000EC72002070B505462846FEF72DFE04464F
:103BB000032C11D004EB840000EBC400074901EB97
:103BC0008000806A40B104EB840101EBC401034A28
:103BD00002EB8101886A804770BD0000EC72002012
:103BE00070B5044694F82000012822D1022084F800
:103BF00020002068006820F001002168086000F0C3
:103C00007FFC05460DE000F07BFC401B0A2808D92C
:103C1000606A40F400306062052084F820000120D2
:103C200070BD2068406800F001000028EBD16062A0
:103C3000F6E7606A40F4002060620120F0E70000CF
:103C400070B505462846FEF7DFFD0446032C11D06B
:103C500004EB840000EBC400074901EB8000C0685E
:103C600040B104EB840101EBC401034A02EB810182
:103C7000C868804770BD0000EC72002070B5054632
:103C80002846FEF7C1FD0446032C0FD004EB840048
:103C900000EBC400064951F8200038B104EB840160
:103CA00001EBC401024A52F82100804770BD0000B8
:103CB000EC72002070B505462846FEF7A5FD0446C7
:103CC000032C11D004EB840000EBC400074901EB86
:103CD0008000006940B104EB840101EBC401034A98
:103CE00002EB81010869804770BD0000EC72002082
:103CF00070B505462846FEF787FD0446032C11D013
:103D000004EB840000EBC400074901EB800040682D
:103D100040B104EB840101EBC401034A02EB8101D1
:103D20004868804770BD0000EC72002070B5054601
:103D30002846FEF769FD0446032C11D004EB8400ED
:103D400000EBC400074901EB8000406940B104EB7F
:103D5000840101EBC401034A02EB810148698047F9
:103D600070BD0000EC72002070B505462846FEF7D5
:103D70004BFD0446032C11D004EB840000EBC4007F
:103D8000074901EB8000806840B104EB840101EB3E
:103D9000C401034A02EB81018868804770BD0000BE
:103DA000EC72002070B505462846FEF72DFD04464E
:103DB000032C11D004EB840000EBC400074901EB95
:103DC0008000C06A40B104EB840101EBC401034AE6
:103DD00002EB8101C86A804770BD0000EC720020D0
:103DE00070B50446A56D00F08BFB064694F83500CF
:103DF000022808D08020606500BF002084F83400CD
:103E000000BF012070BD2068006820F01600216806
:103E100008602068406920F0800021684861206CBB
:103E200008B9A06C28B12068006820F0080021685B
:103E300008602068006820F001002168086010E038
:103E400000F05EFB801B05280BD920206065032055
:103E500084F8350000BF002084F8340000BF032040
:103E6000D0E72068006800F001000028E8D194F84D
:103E70005C103F208840A860012084F8350000BF16
:103E8000002084F8340000BF00BFBBE7014691F872
:103E90003500022803D080204865012070470520A6
:103EA00081F835000868006820F001000A68106099
:103EB0000020F3E7014691F835007047F8B5044655
:103EC000002000908C4800684FF41651B0FBF1F7C9
:103ED000A56D2E6894F85C1008208840304098B199
:103EE0002068006800F0040070B12068006820F0CD
:103EF00004002168086094F85C1008208840A860DD
:103F0000606D40F00100606594F85C10012088400D
:103F1000304068B12068406900F0800040B194F8FA
:103F20005C1001208840A860606D40F00200606570
:103F300094F85C1004208840304068B12068006824
:103F400000F0020040B194F85C1004208840A860A2
:103F5000606D40F00400606594F85C1010208840AB
:103F6000304078B32068006800F0080050B394F83F
:103F70005C1010208840A8602068006800F4802051
:103F800080B12068006800F4002028B9206CC8B116
:103F90002046216C884715E0A06C98B12046A16CA2
:103FA00088470FE02068006800F4807028B9206816
:103FB000006820F0080021680860206C10B12046DD
:103FC000216C884794F85C102020884030400028FD
:103FD00065D02068006800F0100000285FD094F8D9
:103FE0005C1020208840A86094F83500052828D16E
:103FF0002068006820F01600216808602068406989
:1040000020F0800021684861206C08B9A06C28B1BC
:104010002068006820F008002168086094F85C10AF
:104020003F208840A860012084F8350000BF0020B0
:1040300084F8340000BF206D10B12046216D884700
:10404000F8BD2068006800F4802080B12068006816
:1040500000F4002028B9606C10B12046616C8847DC
:104060001DE0E06BD8B12046E16B884717E020687F
:10407000006800F4807068B92068006820F01000C3
:1040800021680860012084F8350000BF002084F812
:10409000340000BFE06B10B12046E16B8847606DD3
:1040A00038B3606D00F00100F0B1052084F83500F0
:1040B0002068006820F001002168086000BF0098B7
:1040C000401C0090B84200D905E02068006800F06C
:1040D00001000028F3D100BF012084F8350000BFA3
:1040E000002084F8340000BFE06C10B12046E16C81
:1040F000884700BFA4E70000140000202DE9F0412C
:104100000446002500F0FCF9074614B90120BDE87B
:10411000F081606A00B100BF022084F8350000BF62
:10412000002084F8340000BF2068006820F00100FF
:10413000216808600AE000F0E3F9C01B052805D9F2
:1041400020206065032084F83500E0E720680068DF
:1041500000F001000028EED12068056821480540E4
:10416000D4E901010843E168084321690843616912
:104170000843A1690843E1690843216A08430543EC
:10418000606A042803D1D4E90B0108430543206881
:1041900005602068456925F00705606A0543606A87
:1041A00004280DD1A06A0543E06A48B12046FEF715
:1041B000E5FB28B140206065012084F83500A6E7C2
:1041C000206845612046FEF7BFFB064694F85C1068
:1041D0003F208840B06000206065012084F83500F1
:1041E000002094E73F8010F02DE9F04704460D468B
:1041F00016461F464FF00008D4F8589000BF94F8B8
:104200003400012802D10220BDE8F087012084F8A3
:10421000340000BF94F83500012825D1022084F82D
:104220003500002060653B46324629462046FEF7B1
:10423000FAFB94F85C103F208840C9F80800206819
:10424000006840F0160021680860206C28B12068E2
:10425000006840F00800216808602068006840F0AD
:1042600001002168086006E000BF002084F83400E7
:1042700000BF4FF002084046C6E7000070B5044694
:1042800000F03EF906462546681C10B10448007847
:10429000054400BF00F034F9801BA842FAD370BD7A
:1042A0001000002070B5054600240DE00120A0405C
:1042B000284038B1064850F8240018B1044951F894
:1042C00024008047601CC4B2102CEFDB70BD0000DE
:1042D000647B002010B5044604480068204020B1EB
:1042E000024804602046FFF7DDFF10BD143C01408A
:1042F000F8B502460B460025002400200021D6E038
:10430000012606FA01F51E6806EA0504AC4274D1DE
:104310001E7906F00306012E04D01E7906F003066E
:10432000022E13D190684F000326BE40B0434F00C9
:10433000DE68BE4030439060506801268E40B04336
:104340001E79C6F300168E40304350601E7906F089
:104350000306032E09D0D0684F000326BE40B043A9
:104360004F009E68BE403043D0601E7906F00306C1
:10437000022E13D1CF0802F1200656F827004E076F
:10438000F70E0F26BE40B0434F07FF0E1E69BE401A
:104390003043CF0802F1200646F8270010684F008E
:1043A0000326BE40B0431E7906F003064F00BE4010
:1043B000304310605E6806F44036002E76D000BFB1
:1043C000002600963C4E366846F480463A4F3E60E2
:1043D0003E46366806F48046009600BF00BF374E62
:1043E0008F0856F827008E07370F0F26BE40B043C0
:1043F000334EB24202D1002624E057E0314EB242A1
:1044000001D101261EE0304EB24201D1022619E050
:104410002E4EB24201D1032614E02D4EB24201D1FC
:1044200004260FE02B4EB24201D105260AE02A4EA7
:10443000B24201D1062605E0284EB24201D107263C
:1044400000E008268F073F0FBE4030431B4E8F0809
:1044500046F82700224E3068A0435E6806F48016B6
:1044600006B120431E4E3060361D3068A0435E68A2
:1044700006F4001606B12043194E361D3060184E62
:10448000361F3068A0435E6806F4003606B120434C
:10449000134E361F3060361F3068A0435E6806F446
:1044A000803606B120430E4E083E3060491C10296C
:1044B000FFF426AFF8BD0000443802400838014040
:1044C000000002400004024000080240000C0240CC
:1044D000001002400014024000180240001C02407C
:1044E000083C0140024613690B400BB1012000E07B
:1044F000002070470AB1816101E00B0483617047BD
:1045000001480068704700000800002070B50546AB
:10451000284602F04FFD0446032C0DD004EBC400E6
:10452000064901EB8000006A30B104EBC401034A84
:1045300002EB8101086A804770BD0000A47B002067
:1045400070472DE9F84F0446206847692068D0F885
:104550000480002594F83E90C7F3002040B1C8F3D2
:10456000002028B145F001056FF480702168486192
:10457000C7F3402040B1C8F3002028B145F0020540
:104580006FF4007021684861C7F3802070B3C8F3EE
:10459000002058B3CA46B4F82AB094F83D60206BA6
:1045A0000090BAF1200F0FD1BBF1000F0CD1212EDA
:1045B00006D0292E04D0282E06D10098212803D118
:1045C000204603F04BFA11E06FF4806021684861E7
:1045D00045F00405B9F1100F02D0B9F1400F05D133
:1045E0002068006840F4007021680860C7F3C020AC
:1045F00040B1C8F3002028B145F008056FF4006011
:10460000216848612DB1206C28432064204602F0C7
:10461000E5FCBDE8F88F2DE9F04705464FF00009AD
:1046200028684668D5F82CA095F83E7095F83D802E
:10463000102F01D0402F75D12868D0F81890286825
:10464000446904F0010060B9BAF52A0F02D0BAF14A
:104650002A4F01D1012000E00020012801D1BDE84E
:10466000F08704F0010048B1C6F3402030B128467D
:1046700002F00CFC284603F0A6F8B7E0C4F3C00033
:1046800030B1C6F3402018B1284602F053FFADE028
:10469000C4F3400030B1C6F3402018B1284602F000
:1046A0005EFFA3E0C9F3800040B32868406800F4CF
:1046B0000060B0F5006FE0D0C4F3C01048B1C6F39D
:1046C000802030B1C4F3800018B9284602F0C6FE3D
:1046D0008CE0C4F380000028CFD0C6F3402000282F
:1046E000CBD0B8F1210F03D1284602F067FE7DE060
:1046F000402F7BD1284603F0B5F877E02868406862
:1047000000F40060B0F5006F70D0C4F3801050B1B9
:10471000C6F3802038B1C4F3800020B9284602F0E7
:10472000CBFD63E00BE0C4F3800000285ED0C6F34D
:10473000402000285AD0284602F026FD56E0286C7A
:1047400010B12868446904E02868D0F818902868F7
:104750004469C4F3400060B1C6F3402048B1286CFE
:1047600010B12868D0F818904946284603F03DF962
:104770003CE0C4F3001030B1C6F3402018B1284625
:1047800003F0C0F932E0B8F1210F02D0B8F1290FDF
:1047900016D1C4F3C01048B1C6F3802030B1C4F3C1
:1047A000800018B9284603F0FDF81FE0C4F380002C
:1047B000E0B1C6F34020C8B1284603F0E6F815E0A2
:1047C000C4F3801048B1C6F3802030B1C4F3800038
:1047D00018B9284603F0B6F808E0C4F3800028B101
:1047E000C6F3402010B1284603F09FF800BF36E71B
:1047F00070B50546284602F0DDFB0446032C0DD0BB
:1048000004EBC400064901EB8000C06930B104EB41
:10481000C401034A02EB8101C869804770BD0000F2
:10482000A47B002070B504460CB9012070BD94F83B
:104830003D0028B9002084F83C00204600F05AF9D9
:10484000242084F83D002068006820F001002168E1
:1048500008602068006840F4004021680860206813
:10486000006820F400402168086000F0C3FB0546A2
:104870005C496068884206D85B48854201D20120C5
:1048800007E0002005E05948854201D2012000E000
:104890000020012800D1C9E75548B5FBF0F6206893
:1048A000406820F03F003043216848604D4960680F
:1048B000884201D8701C07E04FF4967070434FF4A3
:1048C0007A71B0FBF1F0401C2168096A21F03F01C8
:1048D00008432168086243496068884214D8681E0A
:1048E00061684900B0FBF1F0401CC0F30B000428E4
:1048F00001D204203DE0681E61684900B0FBF1F080
:10490000401CC0F30B0034E0A06838B9681E616831
:1049100001EB4101B0FBF1F0401C0AE0681E616848
:1049200001EBC10202EB0111B0FBF1F0401C40F4BD
:104930008040C0F30B0008B901201AE0A06848B914
:10494000681E616801EB4101B0FBF1F0401CC0F34F
:104950000B000CE0681E616801EBC10202EB011163
:10496000B0FBF1F0401CC0F30B0040F4804040F479
:1049700000402168C9694CF6FF72914308432168E1
:10498000C861D4E9070108432168096821F0C00122
:10499000084321680860D4E9031008432168896846
:1049A00048F2FF329143084321688860D4E9050149
:1049B00008432168C96821F0FF0108432168C860E5
:1049C0002068006840F00100216808600020206431
:1049D000202084F83D000020206384F83E0000BFC2
:1049E00024E70000A086010080841E0000093D002D
:1049F00040420F0070B50546284602F0DBFA044637
:104A0000032C0DD004EBC400064901EB80000069C3
:104A100030B104EBC401034A02EB8101086980470D
:104A200070BD0000A47B002070B50546284602F04A
:104A3000C1FA0446032C0DD004EBC400064901EB77
:104A40008000406830B104EBC401034A02EB8101ED
:104A50004868804770BD0000A47B002070B5054603
:104A6000284602F0A7FA0446032C0BD004EBC4003E
:104A7000054951F8200028B104EBC401024A52F85C
:104A80002100804770BD0000A47B002070B5054662
:104A9000284602F08FFA0446032C0DD004EBC40024
:104AA000064901EB8000806930B104EBC401034A80
:104AB00002EB81018869804770BD0000A47B002063
:104AC00070B50546284602F075FA0446032C0DD051
:104AD00004EBC400064901EB8000406930B104EBEF
:104AE000C401034A02EB81014869804770BD0000A0
:104AF000A47B002010B586B00446142101A8FBF762
:104B000029FD3E492068884241D100BF0020009025
:104B10003B48006840F002003949086008460068D8
:104B200000F00200009000BF00BF4FF44070019001
:104B3000122002900020039003200490042005908E
:104B400001A93048FFF7D4FB00BF002000902C489B
:104B50001030006840F40010294910310860084600
:104B6000006800F40010009000BF00BF0022052183
:104B70001F2000F025F91F2000F00EF9002205216A
:104B8000202000F01DF9202000F006F933E01E4936
:104B9000206888422FD100BF00200090184800688C
:104BA00040F02000164908600846006800F0200028
:104BB000009000BF00BF032001901220029000204F
:104BC0000390032004900420059001A90F48FFF7EB
:104BD0008FFB00BF0020009009481030006840F4AF
:104BE00080000749103108600846006800F4800022
:104BF000009000BF00BF06B010BD00000054004090
:104C000030380240000402400058004000140240C6
:104C100070B50546284602F0CDF90446032C0DD0A8
:104C200004EBC400064901EB8000C06830B104EB1E
:104C3000C401034A02EB8101C868804770BD0000CF
:104C4000A47B002070B50546284602F0B3F904465F
:104C5000032C0DD004EBC400064901EB80008068F2
:104C600030B104EBC401034A02EB8101886880473C
:104C700070BD0000A47B0020034800680349097848
:104C80000844014908607047080000201000002017
:104C900010B50D48006840F400700B4908600846E4
:104CA000006840F4806008600846006840F4807046
:104CB0000860032000F0C2F80F2000F007F800F0B1
:104CC0002BF8002010BD0000003C024070B50446E7
:104CD0000E4800784FF47A71B1FBF0F00C49096886
:104CE000B1FBF0F5284601F0D5FA08B1012070BDFE
:104CF000102C07D200222146501E00F061F8054812
:104D0000046001E00120F2E70020F0E7100000203D
:104D1000140000200C00002008B500BF0020009007
:104D20001148006840F480400F4908600846006858
:104D300000F48040009000BF00BF00BF0020009042
:104D4000081F006840F08050091F0860084600688E
:104D500000F08050009000BF00BF00220F21901E85
:104D600000F02EF808BD00004438024010B501469E
:104D7000084600280BDB00F01F0301229A40054B78
:104D8000440943F82420BFF34F8FBFF36F8F00BF58
:104D900010BD000080E100E00146084600280DDB60
:104DA00000BF00BF00F01F0301229A4043099B008F
:104DB00003F1E023C3F8002100BF00BF00BF70472C
:104DC0002DE9F05F80460D461646002704F0DCFF13
:104DD000074639462A46334601F00700C0F1070A64
:104DE000BAF1040F02D94FF0040A01E0C0F1070A3A
:104DF000D14600F1040ABAF1070F02D24FF0000ABF
:104E000001E0A0F1030AD4464FF0010A0AFA09FAB8
:104E1000AAF1010A0AEA020A0AFA0CFA4FF0010B97
:104E20000BFA0CFBABF1010B0BEA030B4AEA0B0488
:104E30002146404604F0B0FFBDE8F09F00BF00F0FF
:104E40000702064B19684FF6FF031940044B0B434A
:104E500043EA0221014B196000BF70470CED00E0EE
:104E60000000FA0570B504460D460CB9012070BD6E
:104E70005848006800F00700A84209D255490D7053
:104E80000846006800F00700A84201D00120EEE7C4
:104E9000207800F0020002281DD1207800F00400E4
:104EA000042805D14C48006840F4E0504A490860A5
:104EB000207800F00800082805D14748006840F431
:104EC0006040454908604448006820F0F000A1684F
:104ED000084341490860207800F00100A8B36068E9
:104EE000012807D13C4808380068C0F34040B8B9F1
:104EF0000120BCE76068022802D06068032807D15F
:104F0000354808380068C0F3406048B90120AEE772
:104F1000314808380068C0F3400008B90120A6E70E
:104F20002D48006820F00300616808432A490860A2
:104F3000FFF7E6FA064609E0FFF7E2FA801B41F2C6
:104F40008831884202D9032091E707E022480068AF
:104F500000F00C006168B0EB810FEDD11D480068D6
:104F600000F00700A84209D91A490D7008460068E8
:104F700000F00700A84201D0012078E7207800F077
:104F80000400042807D11448006820F4E050E168C8
:104F9000084311490860207800F00800082808D16B
:104FA0000D48006820F46040216940EAC1000A49C8
:104FB000086000F03FF808490968C1F30311074A87
:104FC000515CC8400649086006480068FFF77EFE4D
:104FD00000204CE7003C02400838024020ED000869
:104FE000140000200C0000200148006870470000F9
:104FF0001400002000B5FFF7F7FF04490968C1F36A
:105000008221034A515CC84000BD000008380240BC
:1050100030ED000800B5FFF7E7FF04490968C1F368
:105020004231034A515CC84000BD000008380240CC
:1050300030ED00082DE9F047002400250026A146A8
:105040002548006800F00C0020B1042805D008288D
:105050003AD105E0DFF8849039E0DFF8849036E05B
:105060001D48001F006800F03F041B48001F006837
:1050700000F4800078B11A481749091F0968C1F384
:105080008811A0FB01700146224600233846FBF739
:105090006BF905460EE011480F49091F0968C1F375
:1050A0008811A0FB01700146224600233846FBF719
:1050B0005BF905460848001F0068C0F30140401C2A
:1050C0004600B5FBF6F902E0DFF8109000BF00BF24
:1050D0004846BDE8F0870000083802400024F4008C
:1050E000001BB700F8B504460CB90120F8BD2078C4
:1050F00000F00100002874D0F948006800F00C00AE
:1051000004280DD0F648006800F00C00082813D1E0
:10511000F348001F006800F48000B0F5800F0BD149
:10512000EF4808380068C0F34040002859D0606854
:10513000002856D10120D9E700BF6068B0F5803F54
:1051400008D1E7480838006840F48030E44908395D
:1051500008601EE06068B0F5A02F0DD1E048083867
:10516000006840F48020DE4908390860084600687D
:1051700040F4803008600CE0D9480838006820F41A
:105180008030D749083908600846006820F480203C
:10519000086000BF606890B1FFF7B2F9054606E00D
:1051A000FFF7AEF9401B642801D903209EE7CC48E5
:1051B00008380068C0F340400028F1D011E0FFF744
:1051C0009FF9054606E0FFF79BF9401B642801D9CB
:1051D00003208BE7C24808380068C0F3404000282D
:1051E000F1D1207800F0020002285FD1BC480068AD
:1051F00000F00C0058B1BA48006800F00C00082814
:105200001CD1B748001F006800F48000B0B9B44852
:1052100008380068C0F3400020B1E068012801D0E0
:10522000012063E7AE480838006820F0F8002169E3
:1052300040EAC100AA490839086037E0E06800B3D5
:105240000120A8490860FFF75BF9054606E0FFF773
:1052500057F9401B022801D9032047E7A048083826
:105260000068C0F340000028F1D09D48083800686D
:1052700020F0F800216940EAC10099490839086026
:1052800014E0002097490860FFF73AF9054606E068
:10529000FFF736F9401B022801D9032026E7904882
:1052A00008380068C0F340000028F1D1207800F0F1
:1052B000080008282CD16069A8B101208A4908603B
:1052C000FFF71EF9054606E0FFF71AF9401B022812
:1052D00001D903200AE782486C300068C0F340001F
:1052E0000028F1D014E000207F490860FFF708F99A
:1052F000054606E0FFF704F9401B022801D9032008
:10530000F4E677486C300068C0F340000028F1D123
:10531000207800F00400042870D10027704838304D
:10532000006800F0805090B900BF002000906C48E9
:105330003830006840F080506949383108600846CC
:10534000006800F08050009000BF00BF0127674850
:10535000006800F48070B0B96448006840F4807060
:1053600062490860FFF7CCF8054606E0FFF7C8F889
:10537000401B022801D90320B8E65C48006800F40D
:1053800080700028F2D000BFA068012808D15448DE
:105390006830006840F001005149683108601DE044
:1053A000A06805280DD14E486830006840F0040020
:1053B0004B49683108600846006840F00100086009
:1053C0000CE047486830006820F00100444968312B
:1053D00008600846006820F00400086000BFA0686C
:1053E000A8B1FFF78DF8054609E0FFF789F8401BE3
:1053F00041F28831884202D9032077E626E0384816
:1054000068300068C0F340000028EED013E0FFF7DA
:1054100077F8054608E0FFF773F8401B41F2883142
:10542000884201D9032061E62D4868300068C0F346
:1054300040000028EFD1012F07D1294838300068FB
:1054400020F0805026493831086000BFA06900284C
:1054500045D02348006800F00C0008285DD0A06902
:10546000022845D100201F490866FFF749F8054684
:1054700006E0FFF745F8401B022801D9032035E676
:10548000174808380068C0F340600028F1D1D4E91B
:1054900007010843616A40EA81110122A06AC2EB58
:1054A000500041EA00412C20005D41EA00600C49B7
:1054B000091F086001200B490866FFF721F805461F
:1054C00006E0FFF71DF8401B022801D903200DE676
:1054D000034808380068C0F340600028F1D049E074
:1054E0000838024000004742800E474200700040EA
:1054F000002021490866FFF703F8054606E0FEF79D
:10550000FFFF401B022801D90320EFE51B4800687C
:10551000C0F340600028F2D12CE0A069012800D13E
:10552000E4E51648001D0668A069012820D006F4AD
:105530008001E06981421BD106F03F01206A81426F
:1055400016D147F6C0703040616AB0EB811F0FD1B1
:1055500006F440310122A06AC2EB5000B1EB004FCB
:1055600006D106F070612C20005DB1EB006F01D018
:105570000120BBE50020B9E50000474200380240A9
:1055800070B50446204603F0B9FD0546032D0FD043
:10559000204603F0B3FD074901EB4010806938B1A4
:1055A000204603F0ABFD034901EB40108669B0478C
:1055B00070BD0000EC7B002010B504460CB9012042
:1055C00010BD606A38B96068B0F5827F00D105E02F
:1055D0000021E16102E00021216161610021A162FD
:1055E00094F8510028B9002084F85000204600F0BB
:1055F00047F8022084F851002068006820F040003D
:1056000021680860A08800F48270218901F40441B7
:105610000843A18901F400610843217C01F00201E3
:105620000843217D01F001010843218B01F4007141
:105630000843217F01F0380108432021095D01F072
:1056400080010843218D01F400510843216808605E
:105650000421A06901EA104094F8241001F010011F
:105660000843216848602068C06920F40060216810
:10567000C86100206065012084F8510000209FE788
:1056800010B586B00446142101A8FAF763FF6649F5
:10569000206888427ED100BF0020009063480068E7
:1056A00040F48050614908600846006800F480506A
:1056B000009000BF00BF00BF002000905B4814387E
:1056C000006840F002005949143908600846006833
:1056D00000F00200009000BF00BF00BF002000905B
:1056E0000846006840F0010008600846006800F0C5
:1056F0000100009000BF00BF18200190022002901E
:1057000001200390032004900520059001A948483A
:10571000FEF7EEFD80200190022002900120039010
:10572000032004900520059001A94248FEF7E0FD02
:105730004148424908604FF0C060486000213F483E
:105740008160C1604FF4806101610021416181612C
:10575000C1614FF44031016200214162FEF7CEFC8D
:1057600008B1FDF78BF900BF3448E064846300BFE3
:1057700031481830324908604FF0C060486040211D
:105780002F4881600021C1604FF4806101610021D8
:10579000416100E010E08161C1614FF400310162BC
:1057A00000214162FEF7AAFC08B1FDF767F900BFCE
:1057B0002348A064846335E022492068884231D1BF
:1057C00000BF002000901948001F006840F480408E
:1057D0001649091F08600846006800F480400090E0
:1057E00000BF00BF00BF00200090104814380068C0
:1057F00040F480700D49143908600846006800F4D0
:105800008070009000BF00BF0E2001900220029027
:1058100001200390032004900520059001A90A4867
:10582000FEF766FD06B010BD00300140443802406E
:10583000000402400000024040640240C80300200F
:105840002804002000380040002002402DE9F843E1
:105850000446884616461D4694F85100012802D099
:105860000220BDE8F883B8F1000F00D00EB9012086
:10587000F7E76068B0F5827F0CD1A06850B90420CA
:1058800084F851003346424641462046009500F0D8
:1058900042FAE6E7FEF734FE074600BF94F85000F0
:1058A000012801D10220DCE7012084F8500000BF6C
:1058B000042084F8510000206065C4F83880A68771
:1058C000E6872063A086E08620646064A068B0F567
:1058D000004F0BD12068006820F04000216808606C
:1058E0002068006820F48040216808602068006813
:1058F00000F04000402805D02068006840F04000DB
:1059000021680860E06830BB21E02068806800F012
:10591000010050B12068007BA16B0870A06B401C97
:10592000A063E08F401EE08711E0FEF7E9FDC01B99
:10593000A84201D3681C00B94DB9012084F8510078
:1059400000BF002084F8500000BF032089E7E08FEB
:105950000028DAD125E021E02068806800F001000D
:1059600050B12068C068A16B0880A06B801CA06348
:10597000E08F401EE08711E0FEF7C2FDC01BA84289
:1059800001D3681C00B94DB9012084F8510000BF53
:10599000002084F8500000BF032062E7E08F002859
:1059A000DAD13A462946204603F019FB08B12020F7
:1059B0006065012084F8510000BF002084F8500089
:1059C00000BF606D08B101204BE7002049E70000EF
:1059D0002DE9F04104460E46154694F85100012881
:1059E00002D00220BDE8F08106B10DB90120F9E72F
:1059F000A06868B96068B0F5827F09D1042084F896
:105A000051002B4632463146204600F0A9FAE9E71C
:105A100000BF94F85000012801D10220E2E70120E4
:105A200084F8500000BF042084F851000020606515
:105A3000A663A587E58720646064A086E086A068E9
:105A4000B0F5004F0BD12068006820F040002168BD
:105A500008602068006820F48040216808601F48C2
:105A6000E16C08641E48E16CC8631E48E16CC864C0
:105A70000020E16C0865E38F276807F10C01A26B39
:105A8000E06CFEF7B1FB50B1606D40F01000606556
:105A900000BF002084F8500000BF0120A2E720686A
:105AA000006800F04000402805D02068006840F001
:105AB00040002168086000BF002084F8500000BF4B
:105AC0002068406840F020002168486020684068F5
:105AD00040F0010021684860002083E7518E0008F3
:105AE0007B8E0008298E000870B50446204603F01E
:105AF00005FB0546032D0FD0204603F0FFFA0749AA
:105B000001EB4010406838B1204603F0F7FA034932
:105B100001EB40104668B04770BD0000EC7B0020F0
:105B200070B50446204603F0E9FA0546032D0FD070
:105B3000204603F0E3FA074901EB4010006938B151
:105B4000204603F0DBFA034901EB40100669B04739
:105B500070BD0000EC7B00202DE9F84304460F46A1
:105B600016461D46FEF7CCFC8046B14694F851001F
:105B7000012802D00220BDE8F88307B10EB9012048
:105B8000F9E700BF94F85000012801D10220F2E7A4
:105B9000012084F8500000BF032084F85100002049
:105BA00060652763A686E686A063A087E0876064B9
:105BB0002064A068B0F5004F0BD12068006820F089
:105BC0004000216808602068006840F48040216837
:105BD00008602068006800F04000402805D0206878
:105BE000006840F0400021680860E068B0F5006F90
:105BF00037D1606810B1B9F1010F09D1206B00886D
:105C00002168C860206B801C2063E08E401EE08607
:105C100023E02068806800F0020002280AD1206B8F
:105C200000882168C860206B801C2063E08E401EC5
:105C3000E08612E0FEF764FCA0EB0800A84201D366
:105C4000681C00B94DB9012084F8510000BF002044
:105C500084F8500000BF03208DE7E08E0028D8D1E3
:105C600036E0606810B1B9F1010F09D1206B0078FE
:105C700021680873206B401C2063E08E401EE08684
:105C800023E02068806800F0020002280AD1206B1F
:105C9000007821680873206B401C2063E08E401E52
:105CA000E08612E0FEF72CFCA0EB0800A84201D32E
:105CB000681C00B94DB9012084F8510000BF0020D4
:105CC00084F8500000BF032055E7E08E0028D8D1AB
:105CD00042462946204603F0CDF908B120206065F0
:105CE000A06850B900BF002000902068C0680090F4
:105CF00020688068009000BF00BF012084F8510038
:105D000000BF002084F8500000BF606D08B1012082
:105D100031E700202FE72DE9FE4F04460F4690465D
:105D20001D460C9E01200190FEF7EAFB814694F887
:105D300051B060680290AA46BBF1010F0BD00298E7
:105D4000B0F5827F04D1A06810B9BBF1040F02D076
:105D50000220BDE8FE8F1FB1B8F1000F00D00DB9D1
:105D60000120F6E700BF94F85000012801D102207D
:105D7000EFE7012084F8500000BF94F85100042898
:105D800002D0052084F8510000206065C4F83880F6
:105D9000E587A5872763E586A5862064606420687B
:105DA000006800F04000402805D02068006840F0FE
:105DB000400021680860E068B0F5006F52D160686B
:105DC00010B1BAF1010F09D1206B00882168C860B9
:105DD000206B801C2063E08E401EE0863BE0206844
:105DE000806800F00200022810D1E08E70B10198A6
:105DF00001280BD1206B00882168C860206B801CB3
:105E00002063E08E401EE0860020019020688068BC
:105E100000F0010068B1E08F58B12068C068A16B44
:105E20000880A06B801CA063E08F401EE0870120EB
:105E30000190FEF765FBA0EB0900B0420BD3701C8C
:105E400048B1012084F8510000BF002084F85000C0
:105E500000BF03207DE7E08E0028C0D1E08F00283E
:105E6000BDD152E0606810B1BAF1010F09D1206BC9
:105E7000007821680873206B401C2063E08E401E70
:105E8000E0863CE02068806800F00200022810D123
:105E9000E08E70B1019801280BD1206B0078216849
:105EA0000873206B401C2063E08E401EE0860020BB
:105EB00001902068806800F0010068B1E08F58B15F
:105EC0002068C068A16B0870A06B401CA063E08FC5
:105ED000401EE08701200190FEF712FBA0EB0900B5
:105EE000B04201D3701C00B94EB9012084F85100B2
:105EF00000BF002084F8500000BF032029E7E08E97
:105F00000028BFD1E08F0028BCD14A463146204648
:105F100003F0B0F840B12020606500BF002084F895
:105F2000500000BF012014E7A06850B900BF002056
:105F300000902068C068009020688068009000BFD2
:105F400000BF012084F8510000BF002084F85000F9
:105F500000BF606D08B10120FBE60020F9E60000FB
:105F60002DE9F04704460E4617461D4694F8518029
:105F7000D4F80490B8F1010F0AD0B9F5827F04D1AA
:105F8000A06810B9B8F1040F02D00220BDE8F08774
:105F90000EB107B10DB90120F8E700BF94F8500029
:105FA000012801D10220F1E7012084F8500000BF50
:105FB00094F85100042802D0052084F851000020F4
:105FC00060652663A586E586A763A587E5872064C7
:105FD000606494F85100042806D13548E16C0864E7
:105FE0003448E16CC86305E03348E16C0864334829
:105FF000E16CC8633248E16CC8640020E16C08655C
:10600000E38FD4F800C00CF10C01A26BE06CFEF73A
:10601000EBF850B1606D40F01000606500BF0020EB
:1060200084F8500000BF0120B0E72068406840F0CD
:106030000100216848600020A16C0864A16CC8635D
:10604000A16CC864A16C0865E38ED4F800C00CF1A3
:106050000C02216BA06CFEF7C7F850B1606D40F0E8
:106060001000606500BF002084F8500000BF0120D0
:106070008CE72068006800F04000402805D02068C8
:10608000006840F040002168086000BF002084F8EC
:10609000500000BF2068406840F020002168486040
:1060A0002068406840F002002168486000206DE7E9
:1060B000518E00087B8E00086D8E0008778F0008D7
:1060C000298E00082DE9F04104460E46154694F845
:1060D0005100012802D00220BDE8F08106B10DB9BF
:1060E0000120F9E700BF94F85000012801D10220F7
:1060F000F2E7012084F8500000BF032084F851002B
:10610000002060652663A586E586A0636064206440
:10611000A087E087A068B0F5004F0BD12068006829
:1061200020F04000216808602068006840F480404A
:10613000216808601F48A16C08641F48A16CC863EF
:106140001E48A16CC8640020A16C0865E38E276816
:1061500007F10C02216BA06CFEF746F850B1606DA0
:1061600040F01000606500BF002084F8500000BFC0
:106170000120B1E72068006800F04000402805D009
:106180002068006840F040002168086000BF0020DF
:1061900084F8500000BF2068406840F0200021686B
:1061A00048602068406840F0020021684860002094
:1061B00092E700005F8E0008F78E0008298E000825
:1061C00070B50546284602F099FF0446032C09D015
:1061D000054800EB4410006820B1034901EB44116D
:1061E0000868804770BD0000EC7B002070B5044655
:1061F000204602F083FF0546032D0FD0204602F013
:106200007DFF074901EB4010C06838B1204602F01D
:1062100075FF034901EB4010C668B04770BD000030
:10622000EC7B002070B50446204602F067FF05466F
:10623000032D0FD0204602F061FF074901EB40100B
:10624000806838B1204602F059FF034901EB401045
:106250008668B04770BD0000EC7B002070B5044636
:10626000204602F04BFF0546032D0FD0204602F0DA
:1062700045FF074901EB4010406938B1204602F064
:106280003DFF034901EB40104669B04770BD000077
:10629000EC7B002070B504462546681EB0F1807F77
:1062A00001D301200FE0681E4FF0E02148610F216B
:1062B0004FF0FF3003F070FD00204FF0E0218861C7
:1062C00007200861002070BD7047704730B5024656
:1062D0000B4600BF92F83C00012801D1022030BDDE
:1062E000012082F83C0000BF022082F83D001068C7
:1062F00044681068816824F07004186804431068CA
:106300004460184D1068A8421BD01068B0F1804F4F
:1063100017D0154D1068A84213D0144D1068A8422C
:106320000FD0134D1068A8420BD0124D1068A84230
:1063300007D0114D1068A84203D0104D1068A84234
:1063400005D121F080015868014310688160012067
:1063500082F83D0000BF002082F83C0000BF00BF73
:10636000BDE70000000001400004004000080040BC
:10637000000C0040000401400040014000180040B3
:1063800010B504460CB9012010BD94F83D0028B9A1
:10639000002084F83C00204600F026F8022084F813
:1063A0003D00211D206802F09FFF012084F8460077
:1063B00000BF84F83E0001213F20015540200155D7
:1063C0004120015500BF00BF012084F84200432056
:1063D0000155442001554520015500BF012084F896
:1063E0003D000020D0E7000038B504461949206878
:1063F000884218D100BF002000901748006840F084
:106400002000154908600846006800F02000009050
:1064100000BF00BF002205213720FEF7D1FC372046
:10642000FEF7BAFC15E00D492068884211D100BF83
:10643000002000900848001D006840F40030064924
:10644000091D08600846006800F40030009000BF95
:1064500000BF38BD001400404038024000440140F5
:10646000704770B504462068C5682068066906F064
:106470000200022819D105F00200022815D1401FA0
:1064800021680861012020772068806900F00300FE
:1064900018B12046FFF7E4FF05E0204600F0C8F8F9
:1064A000204600F07CF90020207706F00400042844
:1064B00019D105F00400042815D1C04321680861F2
:1064C000022020772068806900F4407018B12046CF
:1064D000FFF7C6FF05E0204600F0AAF8204600F0CE
:1064E0005EF90020207706F00800082819D105F091
:1064F0000800082815D1C0432168086104202077CE
:106500002068C06900F0030018B12046FFF7A8FF1B
:1065100005E0204600F08CF8204600F040F900200D
:10652000207706F01000102819D105F0100010286F
:1065300015D1C04321680861082020772068C06910
:1065400000F4407018B12046FFF78AFF05E02046AE
:1065500000F06EF8204600F022F90020207706F0C7
:10656000010048B105F0010030B16FF00100216871
:106570000861204600F09AF906F08000802809D1D1
:1065800005F08000802805D1C043216808612046BD
:10659000FFF79AFE06F04000402809D105F04000C0
:1065A000402805D1C04321680861204600F07FF9EA
:1065B00006F02000202809D105F02000202805D170
:1065C000C043216808612046FFF77FFE70BD0000D0
:1065D00010B586B00446142101A8F9F7BBFF114994
:1065E000206888421CD100BF002000900E4800683F
:1065F00040F020000C4908600846006800F02000C8
:10660000009000BF00BF40200190022002900020B7
:10661000039004900320059001A90448FDF768FE4B
:1066200006B010BD00440140303802400014024062
:1066300070472DE9F04104460D461646002700BF7D
:1066400094F83C00012802D10220BDE8F08101202D
:1066500084F83C0000BF36B1042E1BD0082E31D088
:106660000C2E5ED145E02946206802F0BFFE20686E
:10667000806940F00800216888612068806920F006
:1066800004002168886120688069296908432168BD
:10669000886148E02946206802F0E0FE20688069B1
:1066A00040F40060216888612068806920F480607F
:1066B0002168886120688069296940EA0120216891
:1066C000886130E02946206802F006FF2068C06932
:1066D00040F008002168C8612068C06920F004000B
:1066E0002168C8612068C069296908432168C861B8
:1066F00019E02946206802F02BFF2068C06940F4A9
:1067000000602168C8612068C06920F48060216849
:10671000C8612068C069296940EA01202168C86110
:1067200001E0012700BF00BF00BF002084F83C004B
:1067300000BF384689E710B504460CB9012010BDEA
:1067400094F83D0028B9002084F83C00204600F071
:1067500025F8022084F83D00211D206802F0C4FDC8
:10676000012084F8460000BF84F83E0001213F204C
:106770000155402001554120015500BF00BF0120B7
:1067800084F842004320015544200155452001551D
:1067900000BF012084F83D000020D0E7704770471B
:1067A00070B504460D4615B994F83E000BE0042D73
:1067B00002D13F20005D06E0082D02D14020005D9F
:1067C00001E04120005D012801D0012070BD1DB90C
:1067D000022084F83E000EE0042D03D102213F2068
:1067E000015508E0082D03D102214020015502E0A7
:1067F00002214120015501222946206802F0E4FDD2
:1068000023492068884203D022492068884201D168
:10681000012000E0002028B12068406C40F40040D6
:10682000216848641A49206888421BD02068B0F16A
:10683000804F17D018492068884213D01749206824
:1068400088420FD01649206888420BD01149206831
:10685000884207D013492068884203D01249206833
:1068600088420CD12068806800F00706062E0CD004
:106870002068006840F001002168086005E0206899
:10688000006840F001002168086000209EE70000D9
:1068900000000140000401400004004000080040E6
:1068A000000C004000400140001800407047704755
:1068B0007047000070B50546284603F047F80446C7
:1068C000022C0DD004EBC400064901EB80000069E6
:1068D00030B104EBC401034A02EB8101086980472F
:1068E00070BD00002C7C00202DE9F84F0446206884
:1068F00005682068C668206847694FF00009CA46E5
:1069000005F00F09B9F1000F0AD105F0200038B1E8
:1069100006F0200020B1204603F024F8BDE8F88FEF
:10692000B9F1000F7CD007F0010018B906F490709F
:10693000002875D005F0010030B106F4807018B160
:10694000606C40F00100606405F0040030B107F0B5
:10695000010018B1606C40F00200606405F00200B4
:1069600030B107F0010018B1606C40F004006064C1
:1069700005F0080048B106F0200010B907F001004A
:1069800018B1606C40F008006064606C002846D06C
:1069900005F0200028B106F0200010B1204602F0DA
:1069A000E1FF20684069C0F3801A606C00F00800C5
:1069B00010B9BAF1000F2DD0204602F080FF2068F8
:1069C000406900F04000402820D100BF00BF21688E
:1069D000143151E8001F21F040002168143141E8D2
:1069E0000002002AF3D100BFE06B50B17F48E16B99
:1069F0000865E06BFDF74AFA88B1E06B016D8847E6
:106A00000DE02046FFF756FF09E009E02046FFF7BA
:106A100051FF04E02046FFF74DFF002060647DE752
:106A2000206B012878D105F01000002874D006F002
:106A300010000028FAD000BF0020009020680068F5
:106A4000009020684068009000BF00BF2068406947
:106A500000F04000402870D1E06B006840681FFAE9
:106A600080F8B8F1000F58D0A08D404555DDA4F84E
:106A70002E80E06BC069B0F5807F43D000BF00BFBF
:106A800021680C3151E8001F21F4807021680C311D
:106A900041E80002002AF3D100BF00BF00BF216817
:106AA000143151E8001F21F001002168143141E840
:106AB0000002002AF3D100BF00BF00BF21681431DB
:106AC00051E8001F21F040002168143141E8000224
:106AD000002AF3D100BF202084F842000020206368
:106AE00000BF00BF21680C3151E8001F21F01000E9
:106AF00021680C3141E80002002AF3D100BFE06BAD
:106B0000FDF76EF902206063A08DE28D801A81B2DC
:106B10002046FFF7CDFE0EE052E0A08D40450AD1A1
:106B2000E06BC069B0F5807F05D102206063A18D64
:106B30002046FFF7BDFEF1E6FFE7A08DE18D401A8C
:106B40001FFA80F8E08DD0B3B8F1000F37D000BF46
:106B500000BF21680C3151E8001F21F490702168BA
:106B60000C3141E80002002AF3D100BF00BF00BF92
:106B70002168143151E8001F21F00100216814310F
:106B800041E80002002AF3D100BF202084F842002F
:106B90000020206300BF00BF21680C3151E8001FB6
:106BA00021F0100021680C3141E80002002AF3D1E5
:106BB00000BF0220606341462046FFF779FEADE644
:106BC00005F0800030B106F0800018B1204603F0D7
:106BD0005DF8A3E605F0400030B106F0400018B1C2
:106BE000204602F0A2FE99E600BF97E6AD980008A5
:106BF00010B504460CB9012010BDA06900B100E039
:106C000000BF94F8410028B9002084F840002046D5
:106C100000F02AF8242084F841002068C06820F49D
:106C200000502168C860204602F01AFF2068006901
:106C300020F49040216808612068406920F02A0013
:106C4000216848612068C06840F400502168C8602D
:106C500000206064202084F8410084F84200002075
:106C6000606300BFC8E7000010B586B00446142179
:106C700001A8F9F76FFC5A49206888424ED100BF3D
:106C8000002000905748006840F010005549086007
:106C90000846006800F01000009000BF00BF00BF71
:106CA000002000904F481438006840F002004D4921
:106CB000143908600846006800F00200009000BF28
:106CC00000BF00BF002000900846006840F00100AF
:106CD00008600846006800F00100009000BF00BF97
:106CE0008020019002200290002003900320049055
:106CF0000720059001A93C48FDF7FAFA4FF400700F
:106D000001900220029000200390032004900720AD
:106D1000059001A93548FDF7EBFA5EE0344920689B
:106D200088425AD100BF002000902E48001F006802
:106D300040F480202B49091F08600846006800F4D1
:106D40008020009000BF00BF00BF002000902548B9
:106D50001438006840F004002249143908600846DD
:106D6000006800F00400009000BF00BF4FF44060D6
:106D7000019002200290002003900320049007203D
:106D8000059001A91B48FDF7B3FA1B481B49086091
:106D90004FF000604860002118488160C1604FF4E6
:106DA000806101610021416181614FF48071C161A5
:106DB000002101624162FDF7A1F908B1FBF75EFE17
:106DC00000BF0E48E063846300BF00220521272036
:106DD000FDF7F6FF2720FDF7DFFF06B010BD00002E
:106DE000001001404438024000040240000002400C
:106DF000004800400008024028600240A80500202A
:106E000070B50546284602F0A1FD0446022C0DD0BF
:106E100004EBC400064901EB8000C06830B104EB0C
:106E2000C401034A02EB8101C868804770BD0000BD
:106E30002C7C002070B50546284602F087FD0446EC
:106E4000022C0DD004EBC400064901EB8000406821
:106E500030B104EBC401034A02EB8101486880476A
:106E600070BD00002C7C002000BFFEE710B502487A
:106E7000FDF767FB10BD00007002002010B502484E
:106E8000FDF7C9FB10BD000070020020C16AB1F51A
:106E90002A0F02D10121C16205E0C16AB1F12A4F76
:106EA00001D10821C1627047F8B505460020009065
:106EB000AC6B94F83D60394800681921B0FBF1F0E3
:106EC0004FF47A71B0FBF1F0C0EBC00000EB800032
:106ED000009000BF009820B9206C40F02000206492
:106EE00009E00098401E00902068006800F40070DF
:106EF000B0F5007FEED000BF606B10B10020616B79
:106F0000C863A06B10B10020A16BC8632068006843
:106F100020F480602168086000206085606B10B1FB
:106F20000020616B0865A06B10B10020A16B0865A3
:106F30002068006820F001002168086094F83D0096
:106F400060280AD1202084F83D00002084F83E000B
:106F500020642046FDF7DAFA1EE006F02800282813
:106F600011D12068006840F00100216808602068A5
:106F7000006840F4806021680860002020632820B9
:106F800084F83D0005E0202084F83D00002084F8CE
:106F90003E002046FDF72CFCF8BD00001400002048
:106FA00001684969C1F3C01111B100210268116182
:106FB000704700000146074A0868904201D100204E
:106FC0007047054A0868904201D10120F8E7032084
:106FD000F6E7000000540040005800402DE9F04161
:106FE000044694F83D6094F83E70102F01D0402F75
:106FF00007D1222E05D12068006820F400602168A6
:10700000086006F02800282805D1002020632820E9
:1070100084F83D0010E02068406800F40060B0F59E
:10702000006F07D0602E05D0202084F83D0000209E
:1070300084F83E00002020632068406800F400606F
:10704000B0F5006F40D12068406820F400602168EE
:107050004860606B90F83500012814D04848616B97
:107060000865606BFCF712FF00285BD020680068A1
:1070700020F0010021680860202084F83D00606B4A
:10708000016D88474EE03E48A16B0865A06BFCF798
:10709000FDFE002846D020684069C0F3801030B162
:1070A00020680069616A0870606A401C606220683C
:1070B000006820F0010021680860202084F83D006D
:1070C000A06B016D88472DE094F83D0060281AD12F
:1070D000202084F83D000020206420684069C0F32F
:1070E000801030B120680069616A0870606A401CD5
:1070F00060622068006820F0010021680860204676
:10710000FDF704FA0EE020684069C0F3801030B14A
:1071100020680069616A0870606A401C60622046ED
:10712000FDF766FB256C05F0010058B905F002007B
:10713000022807D005F00400042803D005F0080059
:10714000082805D12068406820F4E0602168486084
:1071500094F83D60206C00F0040004280ED1282E25
:107160000CD10848E06200202063202084F83D0014
:10717000002084F83E002046FDF73CFCBDE8F0818D
:10718000A96E00080000FFFF70B50446E56A608D37
:10719000042810D12068406820F48060216848608D
:1071A00020680069616A0870606A401C6062608DD6
:1071B000401E60857FE0608D03281AD120684068FA
:1071C00020F4806021684860042D07D0022D05D08E
:1071D0002068006820F480602168086020680069E9
:1071E000616A0870606A401C6062608D401E608544
:1071F00061E0608D022854D1012D01D0102D06D1FF
:107200002068006820F480602168086010E0042D88
:1072100001D0022D06D12068006840F4806021680A
:10722000086005E02068006840F40070216808608C
:1072300020680069616A0870606A401C6062608D45
:10724000401E608520680069616A0870606A401CA1
:107250006062608D401E60852068406820F4407048
:1072600021684860202084F83D0094F83E004028C2
:1072700007D1002084F83E0020632046FDF706FC7D
:1072800019E0002084F83E00082D01D0202D02D105
:107290000020206301E0122020632046FDF7C4FB9C
:1072A00009E020680069616A0870606A401C6062D9
:1072B000608D401E608570BD70B5044694F83D0039
:1072C00022287AD1E66A658D032D13D920680069DA
:1072D000616A0870606A401C6062608D401E608553
:1072E000608D032868D12068406820F480602168A0
:1072F000486061E0E06A022858D0012D01D0002DDD
:1073000054D1204600F0C4FCA0BB2068006820F4E3
:107310008060216808602068406820F4E06021688F
:10732000486020680069616A0870606A401C606299
:10733000608D401E6085202084F83D0094F83E005A
:10734000402807D1002084F83E0020632046FDF746
:107350009DFB31E0002084F83E00082E01D0202E55
:1073600002D10020206301E0122020632046FDF7B7
:107370005BFB21E0FFE72068406820F4E0602168C3
:10738000486020680069616A0870606A401C606239
:10739000608D401E6085202084F83D00002084F828
:1073A0003E002046FDF724FA06E006E0206840682B
:1073B00020F480602168486000BF70BD70B504464D
:1073C000E56A94F83D00212847D1608D50B1606A8C
:1073D000007821680861606A401C6062608D401E10
:1073E00060853AE0082D16D0202D14D015F5803F89
:1073F00011D02068406820F4E060216848601120C6
:107400002063002084F83E00202084F83D002046C0
:10741000FDF724FB21E02068406820F4E06021684B
:1074200048602068006840F400702168086000200F
:107430002063202084F83D0094F83E00402806D1C7
:10744000002084F83E002046FDF73AFB05E00020CE
:1074500084F83E002046FDF701FB70BD2DE9F041A8
:10746000044694F83D5094F83E70E66A208DB0BB17
:10747000212D3CD1082E16D0202E14D016F5803F99
:1074800011D02068406820F4E06021684860112035
:107490002063002084F83E00202084F83D00204630
:1074A000FDF7DCFA44E02068406820F4E0602168E1
:1074B00048602068006840F400702168086000207F
:1074C0002063202084F83D0094F83E00402807D136
:1074D000002084F83E002046FDF7F2FA28E006E09E
:1074E000002084F83E002046FDF7B8FA20E0212D68
:1074F00003D0402F1CD1222D1AD1608D30B92068C5
:10750000406820F480602168486011E094F83E00F3
:10751000402803D1204600F0A5F909E0606A007810
:1075200021680861606A401C6062608D401E608551
:10753000BDE8F081416CC9B202681161416B11B1C3
:10754000416BC96B21B9816B41B1816BC96B29B1A9
:107550000168496841F4006102685160704738B5BC
:1075600090F83E20C16A036B90F83D40222C73D105
:10757000046D64B9402A0AD100BF00240094046855
:10758000646900940468A469009400BF1AE1046D62
:10759000C4B90469B4F5404F14D100BF002400946D
:1075A0000468646900940468A469009400BF00BF83
:1075B0000468246844F4807405682C60046D641CBD
:1075C0000465FFE0448D8CB900BF0024009404687A
:1075D000646900940468A469009400BF00BF046853
:1075E000246844F4007405682C60DDE0448D012CAF
:1075F00072D111F5803F30D10468246824F480648E
:1076000005682C600468646804F40064B4F5006FD5
:1076100010D10468246824F4806405682C6000BFDD
:10762000002400940468646900940468A4690094C8
:1076300000BFB9E000BF00240094046864690094AE
:107640000468A469009400BF00BF0468246844F47F
:10765000007405682C60A7E0A9E0082923D0202940
:1076600021D0122B01D101291DD104290AD00229D0
:1076700008D0102906D00468246824F480640568C2
:107680002C6005E00468246844F4806405682C607C
:1076900000BF002400940468646900940468A4692D
:1076A000009400BF80E00468246824F480640568C6
:1076B0002C6000BF0024009404686469009404688E
:1076C000A469009400BF00BF0468246844F40074F7
:1076D00005682C6068E0FFE7448D022C3BD104294B
:1076E00010D002290ED010290CD00468246824F48C
:1076F000806405682C600468246844F400640568AC
:107700002C6005E00468246844F4806405682C60FB
:107710000468646804F40064B4F5006F10D111F5D6
:10772000803F07D0012905D0082903D0102901D0B6
:10773000202905D10468646844F4805405686C60AD
:1077400000BF002400940468646900940468A4697C
:10775000009400BF28E00468246844F4806405684D
:107760002C600468646804F40064B4F5006F10D100
:1077700011F5803F07D0012905D0082903D0102931
:1077800001D0202905D10468646844F48054056858
:107790006C6000BF0024009404686469009404686D
:1077A000A469009400BF00BF002404650AE000BF84
:1077B000002400940468646900940468A469009437
:1077C00000BF00BF38BD90F83E1040290ED1016DBA
:1077D00029B9416C01F0FE010268116141E0416C80
:1077E000C9B241F00101026811613AE00169B1F5E5
:1077F000804F20D190F83D10212905D1416C01F036
:10780000FE010268116105E0416CC9B241F001015D
:1078100002681161416B11B1416BC96B21B9816B78
:10782000F9B1816BC96BE1B10168496841F400614C
:107830000268516015E0016D41B9416C01F440717D
:10784000F02242EAE111026811610AE0016D0129AA
:1078500007D1416C01F44071F12242EAE111026862
:107860001161704770B5044694F83D50206D98B989
:10787000E06C012807D1A06CC0B221680861206DBE
:10788000801C206550E0A06CC0F3072021680861CF
:10789000206D401C206547E0206D012807D1A06CB9
:1078A000C0B221680861206D401C20653CE0206D5D
:1078B000022836D1222D09D12068006840F480705A
:1078C00021680860206D401C20652DE0608D60B14E
:1078D000212D0AD1606A007821680861606A401C25
:1078E0006062608D401E60851EE0608DE0B9212DD4
:1078F0001AD12068406820F4E06021684860206860
:10790000006840F400702168086000202063202097
:1079100084F83D00002084F83E002046FDF7D0F8B2
:1079200002E02046FFF73CFB70BD418D49B1016884
:107930000969426A1170416A491C4162418D491EC0
:107940004185704770B5044694F83D50608DD8B1BC
:1079500020680069616A0870606A401C6062608D1E
:10796000401E6085608D78B92A2D0DD12068406851
:1079700020F480602168486022202063282084F859
:107980003D002046FDF744F970BD418D49B1416A83
:10799000097802681161416A491C4162418D491EA2
:1079A0004185704770B5044694F83D50608DD8B15C
:1079B000606A007821680861606A401C6062608DBE
:1079C000401E6085608D78B9292D0DD120684068F2
:1079D00020F480602168486021202063282084F8FA
:1079E0003D002046FDF72EF970BDF8B504460D4662
:1079F000002794F83D0000F0280028281CD12068BA
:107A0000406820F4806021684860C5F3800000B9B8
:107A10000127C5F3C01010B9A08986B201E0208B00
:107A200086B200BF002084F83C0000BF32463946D1
:107A30002046FCF785FD0FE000BF00200090206885
:107A40004069009020688069009000BF00BF00BFBF
:107A5000002084F83C0000BFF8BD000070B504466B
:107A600094F83D50E66A082E01D0202E1FD1282D13
:107A70001DD12348E0622068406820F4E06021685E
:107A800048606FF48060216848612068006820F4D5
:107A900080602168086000202063202084F83D0079
:107AA000002084F83E002046FCF7A4FF26E0212DAC
:107AB00020D11348E06221202063202084F83D007B
:107AC000002084F83E002068406820F4E0602168CF
:107AD00048606FF48060216848612068006820F485
:107AE0008060216808602046FFF75AFA2046FDF7BB
:107AF000A9F803E06FF480602168486170BD000060
:107B00000000FFFF38B5044694F83D5020684068F7
:107B100020F4E0602168486000BF002000902068E9
:107B2000406900902068006840F00100216808600A
:107B300000BF00BF2068006820F4806021680860F2
:107B40002068406800F40060B0F5006F42D1222D3B
:107B500001D02A2D1FD1A06B006840686085608D20
:107B600018B1206C40F0040020642068406820F4C4
:107B7000006021684860A06BFCF79CF9012829D0BF
:107B80004148A16B0865A06BFCF780F910B3A06BAE
:107B9000016D88471EE0606B006840686085608DFD
:107BA00018B1206C40F0040020642068406820F484
:107BB000006021684860606BFCF77CF9012809D0FF
:107BC0003148616B0865606BFCF760F910B1606B60
:107BD000016D8847608D18B320684069C0F380004C
:107BE00048B120680069616A0870606A401C606280
:107BF000608D401E608520684069C0F3801048B1E8
:107C000020680069616A0870606A401C6062608D6B
:107C1000401E6085608D18B1206C40F00400206427
:107C2000206C18B12046FFF7D9F92BE02A2D07D197
:107C300000202063282084F83D002046FCF7E8FF60
:107C400094F83D0028280DD11048E0620020206300
:107C5000202084F83D00002084F83E002046FCF7F8
:107C6000C9FE0FE0206B222801D0222D0AD100206E
:107C70002063202084F83D00002084F83E00204648
:107C8000FCF7C6FF38BD0000A96E00080000FFFF2A
:107C900008B5014600200090104800681922B0FB8A
:107CA000F2F04FF47A72B0FBF2F000EB800000903B
:107CB00000BF0098401E0090009828B9086C40F062
:107CC00020000864012008BD0868006800F4007006
:107CD000B0F5007FEDD00020F5E700001400002093
:107CE000F0EE400AF6EE001A60EEA11AB0EE611A4C
:107CF000B0EE600A10EE100A0C49A1EB600000EE35
:107D0000100A21EE002AF7EE081A42EE401A61EE40
:107D1000801AB0EE610A21EE002AF7EE081A42EE50
:107D2000401A61EE801AB0EE610A7047DF59375F82
:107D3000B0EE401A10B99FED1D0A704790ED062A6B
:107D4000D0ED012AB0EE410A02EE620A90ED072A58
:107D5000D0ED022AF0EE400A42EE620A10EE901ACE
:107D60004FF07F42B2EB410F01D1012200E000222F
:107D70000AB1F0EE410A90ED060A90ED042A20EED9
:107D8000020A90ED032A00EE820A90ED072AD0ED58
:107D9000052AF0EE401A42EE221A90ED060A80ED16
:107DA000070AC0ED060AB0EE610AC6E7000000004F
:107DB00010B52DED068B0446B0EE409AF0EE609AB9
:107DC00014B9BDEC068B10BDC4ED009A9FED3A0AC4
:107DD00084ED060A9FED380A84ED070A94ED000A47
:107DE000B5EEC00AF1EE10FA14D8B7EE000A84ED31
:107DF000030A9FED310A84ED040A9FED2F0A84EDFA
:107E0000050A9FED2D0A84ED010A9FED2B0A84EDF2
:107E1000020AD6E794ED000A89EE00AA9FED270A30
:107E2000C0EE0A0AF0EE60AAB0EE6A0A02F0F2FCB6
:107E3000B0EE408A9FED220A02F020FCF0EE000A2C
:107E400060EE200AB7EE000A00EE880AF0EE408AE3
:107E500048EE088A28EE080AC0EE280AC4ED030A94
:107E600094ED030AF0EE000A20EE200A84ED040AE5
:107E700094ED030A84ED050AB7EE000A18EE080A2D
:107E8000F0EE000A20EE200AC0EE280AC4ED010A36
:107E90009FED0B0A02F0F2FBF0EE000A60EE200A02
:107EA000B7EE000A00EEC80A08EE080AC0EE280A7B
:107EB000C4ED020A00BF84E700000000DB0F494068
:107EC000DB0F493F00B50346F0EE403A13B99FED92
:107ED000140A00BD93ED030AD3ED040A30EE200A24
:107EE000D3ED050A30EE200A83EE803A13EE100A35
:107EF000C0F3C751FF2901D0012100E0002121B1C9
:107F000083ED063A83ED073A03E0C3ED063AC3ED8D
:107F1000073AB0EE630A1846FFF70AFFD9E70000F8
:107F20000000000010B50446022C02DB4FF0FF30C9
:107F300010BD0F4850F8240008B10020F8E7482091
:107F4000FAF7ACFA0A4941F82400084650F8240030
:107F500010B94FF0FF30EBE7054951F824004821F4
:107F6000F8F7F8FA024850F8240004700020DFE720
:107F7000C80000202DE9FF41054625B96FF001003A
:107F800004B0BDE8F081287800F086F8064616B9FE
:107F90006FF00300F4E7B41C6F88A7F201200B28F0
:107FA0006BD2DFE800F0060708092526272845469A
:107FB000470000BF00BF00BF4FF4007000900820D2
:107FC0008DF80400002010E034F81010C1F30722EF
:107FD0000DF1050101F8102014F81020012101EB2A
:107FE00040030DF10501CA54401C0428ECDB47E0B6
:107FF00000BF00BF00BF40F2FF10009008208DF8C6
:108000000400042011E034F81010C1F30723011F0D
:108010000DF1050202F8113014F81020012303EBD2
:1080200041030DF10501CA54401C0828EBDB27E091
:1080300000BF00BF40F2FF20009008208DF8040030
:1080400000BF12E034F81010C1F30723A0F10801BB
:108050000DF1050202F8113014F81020012303EB92
:1080600041030DF10501CA54401C0B28EADB002135
:108070008DF80B108DF80C1002E04FF0FF307FE709
:1080800000BF28786946FAF7B5F808B9002077E705
:108090004FF0FF3074E700000146022901DB0020A9
:1080A0007047024850F82100FAE70000C80000209D
:1080B000014621B1012905D0022909D105E042F28A
:1080C000107070474FF48040FBE747F23050F8E7FC
:1080D0004FF0FF30F5E7024621B1012903D0022914
:1080E00016D10AE000BFB2F5007F05DDB2F5027FD0
:1080F00002DA501E40B270470BE0B2F5017F06DD98
:1081000040F20B20824202DA501E40B2F3E700E058
:1081100000BF00BF4FF0FF30EDE770B505460DB969
:10812000002070BD2878FFF7B7FF04460CB9002087
:10813000F7E700210AE004F1180252F8210020B10B
:1081400042886B889A4200D1EBE7491C94F84400BE
:108150008842F0DC0020E4E720B1012805D00228A5
:1081600009D105E09FED050A7047B3EE030AFBE76E
:10817000B7EE000AF8E7B7EE000AF5E70000104294
:1081800070B5054615B96FF0010070BD2878FFF78E
:10819000C9FE10B14FF0FF30F7E72878FFF77CFFFA
:1081A000044614B94FF0FF30EFE7002110E004F16E
:1081B000180050F8210050B104F1180050F82100C7
:1081C00040886A88904202D16FF00200DDE7491CC6
:1081D00094F844008842EADC94F844000B2802DB5F
:1081E0004FF0FF30D1E75020FAF758F9064616B99C
:1081F0004FF0FF30C9E72868306068687060282158
:1082000006F11800F8F7A6F96979282081556988E0
:1082100028780322F9F7AEFE28B13046FAF7A8F81D
:108220004FF0FF30B1E794F8441004F1180040F823
:10823000216094F84400401C84F844000020A4E726
:108240002DE9F0472DED028B0446B0EE408A2CB9A3
:108250006FF00100BDEC028BBDE8F0872078FFF7DE
:108260001BFF054615B96FF00300F3E7B7EE000AF0
:10827000B4EEC08AF1EE10FA03DDB7EE000AB0EEFC
:10828000408ABFEE000AB4EEC08AF1EE10FA03D2C3
:10829000BFEE000AB0EE408A607918B1B1EE480A2C
:1082A000B0EE408A2046FFF738FF074617B96FF057
:1082B0000300CFE721796088FFF70DFF0646002E07
:1082C00002DA4FF0FF30C5E705F102082079FFF729
:1082D000EFFE00EE100AB8EEC00A20EE080ABDEE6E
:1082E000C00A10EE100A0FFA80F928F81690002044
:1082F000B0E72DE9F04387B0054625B96FF00100DE
:1083000007B0BDE8F0832878FFF7C6FE064616B929
:108310006FF00300F4E74FF000093AE006F11800AF
:1083200050F8294094B36088698888422FD16988C1
:10833000287800236A46F9F715FDA8B1FAF7BFF9C6
:1083400007468846D4E90831FA1A68EB01004FF471
:108350007A7300219A1A814103D200202076001FEF
:10836000CEE74FF0FF30CBE701202076FAF7A7F9F0
:10837000C4E908016946204600F0C4FA04F1080186
:108380008EC904F12C008EC00020B9E7FFE709F187
:10839000010996F844004845C0DC6FF00300AFE7E0
:1083A00010B50F480F4908600320486000210D48B0
:1083B0008160C1604FF4102101614FF400114161EF
:1083C00000210176417681760121C1760021017775
:1083D0004177FBF7E5F908B1FAF750FB10BD000053
:1083E000006400402002002010B50F480F490860CB
:1083F0000320486000210D488160C1604FF41021C6
:1084000001614FF4001141610021017641768176CE
:108410000121C176002101774177FBF7C1F908B14D
:10842000FAF72CFB10BD0000006800404802002055
:1084300008B500BF002000901A48006840F4001002
:10844000184908600846006800F40010009000BF5A
:1084500000BF00BF002000900846006840F4800084
:1084600008600846006800F48000009000BF00BF6C
:10847000002207210C20FCF7A3FC0C20FCF78CFC4D
:10848000002205213A20FCF79BFC3A20FCF784FCF3
:10849000002205213B20FCF793FC3B20FCF77CFCF1
:1084A00008BD00003038024010B5064A00210648D9
:1084B00002F083FF05490860054A0021054802F0E3
:1084C0007CFF10BDF4EC0008ED91000800000020D6
:1084D00098ED0008A595000800B587B0142102A802
:1084E000F8F738F800BF002001907248006840F0AB
:1084F0000200704908600846006800F00200019020
:1085000000BF00BF00BF002001900846006840F097
:10851000010008600846006800F00100019000BFFB
:1085200000BF00BF002001900846006840F008002E
:1085300008600846006800F00800019000BF00BF16
:1085400000BF002001900846006840F00400086069
:108550000846006800F00400019000BF00BF00BFA3
:10856000002001900846006840F4807008600846CA
:10857000006800F48070019000BF00BF00BF0020C1
:1085800001900846006840F0200008600846006836
:1085900000F02000019000BF00BF00BF002001904C
:1085A0000846006840F0800008600846006800F057
:1085B0008000019000BF00BF00BF0020019008466E
:1085C000006840F0400008600846006800F0400085
:1085D000019000BF00BF002240213748FBF78AFF0F
:1085E000012210213548FBF785FF0122114634484E
:1085F000FBF780FF4020029001200390049005903B
:1086000002A92D48FBF774FE082002904FF40410D5
:1086100003900120049002A92748FBF769FE01207E
:1086200002904FF4041003900120049002A9234803
:10863000FBF75EFE1020029001200390049005904D
:1086400002A91E48FBF754FE302002904FF404109C
:1086500003900120049002A91A48FBF749FE01206B
:10866000029003900490059002A91548FBF740FE84
:10867000002205210620FCF7A3FB0620FCF78CFB5B
:10868000002205210920FCF79BFB0920FCF784FB55
:10869000002206210A20FCF793FB0A20FCF77CFB52
:1086A000002206211720FCF78BFB1720FCF774FB38
:1086B00007B000BD30380240001802400000024000
:1086C000000402400008024010B50B480B49086046
:1086D0000B484860002109488160C1604FF4804127
:1086E0000161002141618161C1610162FCF79AF879
:1086F00008B1FAF7C3F910BD005400407002002021
:10870000A086010010B50B480B4908600B48486073
:10871000002109488160C1604FF48041016100215E
:1087200041618161C1610162FCF77CF808B1FAF72F
:10873000A5F910BD00580040C4020020A086010029
:1087400010B50F480F4908604FF48270486000214F
:108750000C488160C160022101610121416149022F
:1087600081611821C16100210162416281620A2197
:10877000C162FCF721FF08B1FAF780F910BD0000D3
:10878000003001401803002010B50F480F49086061
:108790004FF48270486000210C4881604FF4006102
:1087A000C160022101610121416149028161002111
:1087B000C1610162416281620A21C162FCF7FCFE73
:1087C00008B1FAF75BF910BD0038004070030020D3
:1087D00000B587B01C216846F7F7BCFE154816495E
:1087E00008600020486000211348816041F2883110
:1087F000C160002101618161FDF7C2FD08B1FAF796
:108800003DF90D48FDF797FF08B1FAF737F96020F9
:1088100000900020019002900490002269460648D2
:10882000FDF707FF08B1FAF729F90348FDF7D0FE75
:1088300007B000BD00440140D00400201CB500205A
:10884000009001900E480F49086000204860002108
:108850000C48816040F2E731C16000218161FDF781
:108860008FFD08B1FAF70AF90020009001906946DF
:108870000448FDF72BFD08B1FAF700F91CBD000014
:10888000001400408804002010B50B480B49086014
:108890004FF4E1304860002108488160C160016107
:1088A0000C21416100218161C161FEF7A1F908B18C
:1088B000FAF7E4F810BD0000001001401805002090
:1088C00010B50C480C4908600C48486000210A4863
:1088D00081604FF40051C160C91001610C214161F8
:1088E00000218161C161FEF783F908B1FAF7C6F88A
:1088F00010BD00000048004060050020A086010077
:1089000000BFFEE72DE9F0412DED068B04460D4634
:10891000A87B697B40EA0126297CE87B41EA0020AC
:1089200000B209EE100AA97C687C41EA002007B277
:108930002079FFF7BDFB80462079FFF70DFCB0EEF4
:10894000408A00EE106AB8EE400A9FED4E1AC0EE63
:10895000010A9FED4D0A20EE800AF0EE408AB8EE43
:10896000C90AF0EE409A17FB08F000EE100AB8EEC4
:10897000C00ADFED460A80EE201AB0EE41AAA079C7
:1089800070B3B4F84010701AB0F5805F03DD616C0D
:10899000491E616405E010F5805F02DA616C491CD4
:1089A0006164A4F84060B0EE680AD4ED110AB8EE34
:1089B000E01ADFED351AF0EE400A41EE210A80EEB2
:1089C000881A84ED121AD4ED120AC4ED020AC9EE17
:1089D000880AC4ED030A6AEE080AC4ED040A0DE031
:1089E00000206064A4F840609FED290A84ED120A1B
:1089F000C4ED028AC4ED039A84ED04AA2820005D28
:108A0000A8B307E094ED020ADFED1F0A30EE200A5A
:108A100084ED020A94ED020AB5EEC00AF1EE10FAF6
:108A2000F0D307E094ED020ADFED170A30EE600A9A
:108A300084ED020A94ED020ADFED130AB4EEE00AB7
:108A4000F1EE10FAEEDA94ED020ADFED0F0A30EEE5
:108A5000C00A84ED020A94ED030AB1EE400A84EDE7
:108A6000030A94ED040AB1EE400A84ED040AE87C9E
:108A700000EE100AB8EE400A84ED050ABDEC068B44
:108A8000BDE8F08100000046DB0FC94000008046D1
:108A90000000000000BFFEE710B52DED0C8B044672
:108AA000B0EE40DAF0EE60AAB0EE41BAF0EE619AB4
:108AB0001DEE100A01F05FF970B11AEE900A01F094
:108AC0005AF948B11BEE100A01F055F920B119EE20
:108AD000900A01F050F920B994ED060ABDEC0C8B18
:108AE00010BD606890ED070AB0EE401AF0EE6A0A19
:108AF000B0EE4D0AF9F7C1FEF0EE40BA606890EDB5
:108B0000000A20EE2BCA606890ED000A60EE2ADAB7
:108B1000B0EE6D0A04F11C00FFF70AF9B0EE40AAAE
:108B20002078B0B1012802D0022815D10EE094EDD2
:108B3000020AF0EE400AB0EE690A01F047FED4EDF9
:108B4000050A7AEE600AC0EE808A05E0F0EE4B8AF4
:108B500002E0DFED388A00BF00BFC4ED04BA84ED47
:108B600005AA18EE900A01F006F918B99FED310A2E
:108B7000F0EE408A606890ED010A20EE0C0AD0ED1C
:108B8000030AB0EE408A08EEE08A94ED030AB0EEE4
:108B9000409A0CEE299A606890ED020A60EE09CACC
:108BA000606890ED020ADFED240AB4EEE00AF1EE0F
:108BB00010FA1CDD19EE100A01F0DDF8B8B138EE3C
:108BC0002C0AB0EEC00A6068D0ED050AB4EEE00AE7
:108BD000F1EE10FA0BD8B0EEC90A6068D0ED040AC5
:108BE000B4EEE00AF1EE10FA01D884ED039A38EE03
:108BF0002C0AB0EE408A18EE100A01F0BCF8B0B1B1
:108C0000606890ED050ADFED0C0AB4EEE00AF1EEC3
:108C100010FA0ADD606890ED050AF0EE400AB0EE49
:108C2000480AF8F777FDB0EE408A84ED068A94EDA5
:108C3000060A53E700000000BD37863570B52DEDFC
:108C4000028B04460E46F0EE408A154624B94FF0DA
:108C5000FF30BDEC028B70BD95ED010A10EE101ACD
:108C6000084601F088F810B94FF0FF30F1E795EDB4
:108C7000020A10EE101A084601F07DF810B94FF004
:108C8000FF30E6E795ED030A10EE101A084601F0F2
:108C900072F810B94FF0FF30DBE795ED040A10EEE3
:108CA000101A084601F067F810B94FF0FF30D0E70E
:108CB00095ED050A10EE101A084601F05CF810B99F
:108CC0004FF0FF30C5E76560B7EE000A80EE288AF6
:108CD00018EE100A01F04FF810B184ED028A02E09C
:108CE0004FF0FF30B5E7606890ED060AF0EE400AFD
:108CF000B0EE680A04F11C00FFF75AF8267020460F
:108D000000F002F80020A4E710B5044614B94FF0B3
:108D1000FF3010BD9FED0B0A84ED030A9FED090A99
:108D200084ED040A9FED070A84ED050A9FED050A0C
:108D300084ED060A9FED030A04F11C00FFF7C2F858
:108D40000020E6E7000000001C4A1268526942F069
:108D500040021A4B1B685A61194A926A42F010028B
:108D6000174B9A62174A1268126822F00102154BDB
:108D70001B681A6007E0134A1268126822F00102A9
:108D8000104B1B681A600F4A1268126802F0010249
:108D9000002AF0D10C4A0B4B1B689A60094A1268F2
:108DA000D060084A12685160064A1268126842F0A0
:108DB0000102044B1B681A60704700006005002028
:108DC00000600240A80500200448004010B5044699
:108DD00013480068C06820F4005011490968C86051
:108DE00010480068006820F001000E49096808601A
:108DF0000C4800684460032003F0C5FA0948006885
:108E0000006840F0010007490968086004480068EC
:108E1000C06840F4005002490968C86010BD0000F5
:108E200060050020A805002070B50546AC6B2068E1
:108E3000406820F0030021684860606D40F0100039
:108E40006065012084F851002046FCF799FB70BD55
:108E500070B50446A56B2846FCF762FE70BD70B580
:108E60000446A56B2846FDF7C1F970BD70B50446F0
:108E7000A56B2846FDF7F2F970BD70B50546AC6BE1
:108E8000FBF73EFB06462868006800F48070B0F5EA
:108E9000807F2BD02068406820F020002168486047
:108EA000A06850B96068B0F5827F06D1206840683C
:108EB00020F003002168486005E02068406820F049
:108EC00001002168486032466421204600F087F89E
:108ED00008B1202060650020E087012084F851005F
:108EE000606D18B12046FCF74BFB70BD2046FCF7C7
:108EF000FBFD00BFF9E7F8B50546AC6BFBF700FBDF
:108F000006462868006800F48070B0F5807F2DD098
:108F10002068406820F02000216848602068406890
:108F200020F002002168486032466421204600F0AB
:108F3000A1F818B1606D40F020006065A06850B9DC
:108F400000BF002000902068C06800902068806802
:108F5000009000BF00BF0020E086012084F851008F
:108F6000606D18B12046FCF70BFBF8BD2046FDF7FD
:108F700027F900BFF9E770B50546AC6BFBF7C0FAFF
:108F800006462868006800F48070B0F5807F21D024
:108F90002068406820F02000216848603246642143
:108FA000204600F067F818B1606D40F02000606561
:108FB0002068406820F00300216848600020E086B7
:108FC000E087012084F85100606D18B12046FCF75D
:108FD000D7FA70BD2046FDF725F900BFF9E7F8B5CF
:108FE00004460E4615466068B0F5827F0DD1A06834
:108FF000B0F5004F03D0A068B0F5806F05D12068B0
:10900000006820F04000216808606068B0F5827F49
:109010001FD1A068B0F5806F0DD0334600228021AB
:109020002046009500F076F808B3606D40F020000F
:1090300060650320F8BD33460022012120460095DB
:1090400000F068F898B1606D40F020006065032082
:10905000F0E73346002201212046009500F05AF83F
:1090600028B1606D40F0200060650320E2E7002039
:10907000E0E700007CB504460E4615463346012263
:1090800002212046009500F045F828B1606D40F0BF
:109090002000606503207CBD164800681821B0FBE5
:1090A000F1F01549B0FBF1F04FF47A7148430190AB
:1090B0006068B0F5827F0DD13346002280212046C2
:1090C000009500F027F898B1606D40F020006065D1
:1090D0000320E0E700BF019800B908E00198401EB6
:1090E000019020688068C0F3C0100028F3D100BF51
:1090F0000020D0E71400002040420F000146044A3F
:109100000868904201D1002070470320FCE700006E
:10911000003001402DE9F84F04460D4690461E46AA
:10912000DDF82890FBF7ECF9A0EB0900371AFBF704
:10913000E7F982462C480068C0F3CB3078430090B2
:1091400046E0701C002843D0FBF7DAF9A0EB0A00D8
:10915000B84200D2A7BB2068406820F0E000216838
:1091600048606068B0F5827F0DD1A068B0F5004F0F
:1091700003D0A068B0F5806F05D12068006820F0AA
:10918000400021680860A06AB0F5005F0DD100BF03
:109190002068006820F4005021680860206800689A
:1091A00040F400502168086000BF012084F851009D
:1091B00000BF002084F8500000BF0320BDE8F88FF6
:1091C000FFE7009808B9002702E00098401E0090D1
:1091D000206880682840A84201D1012000E00020DA
:1091E0004045AED10020E9E71400002070B50546E7
:1091F00002F0DDF8044602F03CF970BD10B5FBF753
:109200003BFD04F091FC012801D003F0ADFD10BD41
:1092100000B593B0302107A8F7F79CF9142102A8F4
:10922000F7F798F900BF002001902448006840F04B
:109230008050224908600846006800F08050019084
:1092400000BF00BF00BF002001901D48006840F42F
:1092500080401B4908600846006800F48040019087
:1092600000BF00BF012007900004089002200D906D
:1092700041050E9106210F91A82110910221119113
:109280000421129107A8FBF72DFF08B1F9F7F6FBAF
:109290000F20029002200390002004904FF4A05071
:1092A00005904FF480500690052102A8FBF7DAFDE7
:1092B00008B1F9F7E3FB13B000BD000040380240ED
:1092C000007000400348006840F4700001490860E5
:1092D0007047000088ED00E010B50248FDF7C1F8C6
:1092E00010BD00008804002010B502682B4B984286
:1092F0000ED0B0F1804F0BD0294B984208D0294BAB
:10930000984205D0284B984202D0284B984203D16E
:1093100022F070024B681A43204B984220D0B0F1E3
:10932000804F1DD01E4B98421AD01E4B984217D02A
:109330001D4B984214D01D4B984211D01C4B9842A3
:109340000ED01C4B98420BD01B4B984208D01B4BA5
:10935000984205D01A4B984202D01A4B984203D13A
:1093600022F44072CB681A4322F080034C6943EA2E
:1093700004028B68C3620B688362084B984202D078
:109380000A4B984201D10B690363036843F004035D
:10939000036001234361026010BD00000000014032
:1093A0000004004000080040000C004000040140A0
:1093B00000400140004401400048014000180040C6
:1093C000001C00400020004030B501F01F050124C2
:1093D00004FA05F3046A9C430462046A01F01F0561
:1093E00002FA05F52C43046230BD000030B5026A74
:1093F000056A25F0010505624368846924F070045C
:1094000024F003040D682C4322F002028D682A43E5
:10941000104DA84200D103E00F4DA84206D100BF75
:1094200022F00802CD682A4322F00402094DA84226
:1094300002D0094DA84207D123F4807323F40073AE
:109440004D692B438D692B43436084614D684563AF
:10945000026230BD000001400004014030B5026AE4
:10946000056A25F0100505624368846924F4E04428
:1094700024F440740D6844EA052422F020028D682B
:1094800042EA0512124DA84200D103E0114DA84254
:1094900007D100BF22F08002CD6842EA051222F017
:1094A00040020B4DA84202D00A4DA84209D123F434
:1094B000806323F400634D6943EA85038D6943EAC1
:1094C0008503436084614D688563026230BD00009E
:1094D000000001400004014030B5026A056A25F42D
:1094E000807505624368C46924F0700424F00304A5
:1094F0000D682C4322F400728D6842EA0522124D59
:10950000A84200D103E0114DA84207D100BF22F4C8
:109510000062CD6842EA052222F480620A4DA84228
:1095200002D00A4DA84209D123F4805323F40053FA
:109530004D6943EA05138D6943EA05134360C4612D
:109540004D68C563026230BD000001400004014067
:1095500030B5036A056A25F4805505624468C2691E
:1095600022F4E04222F440720D6842EA052223F41C
:1095700000538D6843EA0533084DA84202D0084DD8
:10958000A84204D124F480444D6944EA851444601F
:10959000C2614D680564036230BD000000000140F7
:1095A0000004014070B5054601F064FC1D4A00212D
:1095B0001D4801F002FF1D4908601D4A00211D4899
:1095C00001F0FBFE194948601B4A00211B4801F0CD
:1095D000F4FE1649886000220A21022001F0F8FCFE
:1095E0001249C86000223021022001F0F1FC0F492D
:1095F000486100220C21022001F0EAFC01460B48E0
:10960000816100221821022001F0E2FC0146074896
:10961000C16101F07BFC01F0CAFE044601F029FFA4
:1096200070BD0000BCED0008419600087C80002061
:10963000E0ED00088597000804EE00082D9800086A
:109640002DED048B01F0FDFB064605F069F841ECB9
:10965000190B9FED3F0B53EC102B04F059FE41EC1E
:10966000180B05F019F80546002001F09AFB01F0EF
:10967000DBFB044638493948F8F7A6F83748F8F7CD
:109680007FF8B0EE408A36493648F7F791F833480C
:10969000F8F776F8F7EE000A80EE801AB0EE418A0D
:1096A000314AB0EE480A00213048FFF7C7FA0020DF
:1096B000F8F752FF4BE02C44F8F722FAF8F74CF891
:1096C000F8F756F8F8F76CF8F8F776F801F0D2FBEF
:1096D0002248F8F717F92148F8F776F9204B1F4A86
:1096E0001C32A2F10C011F48F7F772F91D492048FE
:1096F000F6F7C6FF01F00AFC184890ED0A0AF0EEF2
:10970000400ADFED1C1A9FED1B1A9FED1B0A17483C
:10971000FFF7C2F9B0EE408A0020F8F7C5FE1748FF
:10972000134B0ECB0C300EC018380C4B1C330ECB29
:109730000EC01349486901F0DBFC114900231A46A9
:1097400048690E4901F092FC204601F039FBB2E76E
:109750000000000000407F40687D0020987C0020D1
:10976000FC7C0020E87C002078ED0008147D0020BF
:10977000087D00200000000000002042507D0020F5
:109780007C8000202DED048B01F05BFB064604F08D
:10979000C7FF41EC190B9FED1E0B53EC102B04F08F
:1097A000B7FD41EC180B04F077FF0546002001F0EF
:1097B000F8FA01F039FB0446F9F788F806469FED00
:1097C000160A31461548F9F71BFB20E02C441449D2
:1097D00000231A464869134901F0BAFB18B9114928
:1097E0000E48F9F740FC0E4900231A4688690E49D5
:1097F00001F0AEFB0948F9F70BFC0B490748F9F7F4
:1098000041F90648F9F7A6FB204601F0D9FADDE751
:109810000000000000407F400000FA43987D0020D7
:109820007C80002058800020708000202DED048B6B
:1098300001F007FB064604F073FF41EC190B9FEDA6
:10984000150B53EC102B04F063FD41EC180B04F0E6
:1098500023FF0546002001F0A4FA01F0E5FA0446D2
:1098600001F000FA02F062FC13E02C440B4A0C49B0
:109870000C4802F017FC0C49886901F039FC0A49D0
:1098800000231A468869074901F0F0FB204601F0E1
:1098900097FAEAE70000000000407F40807D00204A
:1098A000637C0020747D00207C80002070B504461D
:1098B000A56B0020E8852846FCF7FCFF70BD00BFC3
:1098C00000BF02680C3252E8002F22F49071026847
:1098D0000C3242E80013002BF3D100BF00BF00BFE1
:1098E0000268143252E8002F22F00101026814329B
:1098F00042E80013002BF3D100BF016B01290ED108
:1099000000BF00BF02680C3252E8002F22F01001A5
:1099100002680C3242E80013002BF3D100BF202173
:1099200080F8421000210163704710B5044620689A
:10993000C06820F040002168C860202084F8410001
:109940002046FDF777FA002010BD00000146044ACA
:109950000868904201D1002070470220FCE7000017
:1099600000480040F8B504460025002694F842005F
:10997000222873D1A068B0F5805F0BD1206948B967
:10998000A66A20684068C0F308003080A06A801C86
:10999000A06214E0A56AA068B0F5805F03D0A0685B
:1099A00028B9206918B920684068287004E0206848
:1099B000406800F07F002870A06A401CA062E08D23
:1099C000401E80B2E085002846D12068C06820F0A3
:1099D00020002168C8602068C06820F48070216879
:1099E000C8602068406920F001002168486120209B
:1099F00084F8420000206063206B012826D10020FB
:109A0000206300BF00BF21680C3151E8001F21F026
:109A1000100021680C3141E80002002AF3D100BF98
:109A20002068006800F0100010280AD100BF002054
:109A3000009020680068009020684068009000BF97
:109A400000BFA18D2046FCF733FF02E02046FDF762
:109A5000D7F90020F8BD01E00020FBE70220F9E77C
:109A60002DE9F84F04462068006920F44050E16871
:109A70000843216808612169A068084361690843B7
:109A8000E169084300902068C06849F20C6188438E
:109A9000009908432168C8602068406920F440703C
:109AA000A16908432168486176492068884203D04B
:109AB00075492068884203D1FBF7ACFA814602E081
:109AC000FBF798FA8146E069B0F5004F6CD10220AF
:109AD0006168A0FB015003461920A9FB00700146F4
:109AE0002A463846F6F740FC6421B0FBF1F04FEA15
:109AF000001A02206168A0FB01510B461920A9FB46
:109B000000712A463846F6F72FFC8346022061682A
:109B1000A0FB015003461920A9FB00712A463846D4
:109B2000F6F722FC6421B0FBF1F000EBC00101EB81
:109B30000010ABEB8000322101EBC0006421B0FBD0
:109B4000F1F000F0F8000AEB400A02206168A0FB87
:109B5000015003461920A9FB007001462A463846E9
:109B6000F6F702FC834602206168A0FB0150034621
:109B70001920A9FB00712A463846F6F7F5FB642147
:109B8000B0FBF1F000EBC00101EB0010ABEB80008B
:109B9000322101EBC0006421B0FBF1F000F00700BE
:109BA0005044216888606AE004206168A0FB01508D
:109BB00003461920A9FB007001462A463846F6F7ED
:109BC000D3FB824604206168A0FB015003461920A4
:109BD000A9FB007001462A463846F6F7C5FB64210A
:109BE000B0FBF1F000EBC00101EB0010AAEB80002C
:109BF000322101EB00106421B0FBF1F000F0F00A1B
:109C000004206168A0FB017003461920A9FB0051E4
:109C10003A462846F6F7A8FB6421B0FBF1F00AEBC0
:109C2000001A04206168A0FB01510B461920A9FB12
:109C300000712A463846F6F797FB83460420616890
:109C4000A0FB015003461920A9FB007001462A46DB
:109C50003846F6F789FB6421B0FBF1F000EBC00158
:109C600001EB0010ABEB8000322101EB001064210E
:109C7000B0FBF1F000F00F00504421688860BDE8AF
:109C8000F88F00000010014000140140014691F8D7
:109C90004100212828D18868B0F5805F0BD1086980
:109CA00048B90A6A1088C0F308000B685860086A4F
:109CB000801C086205E00B6A581C086218780B6863
:109CC0005860C88C401E80B2C88458B90868C06803
:109CD00020F080000B68D8600868C06840F0400041
:109CE0000B68D860002070470220FCE710B500F038
:109CF00009F80348FCF7F8FD0148F8F729FD10BD05
:109D0000600500200448006800F0200018B10248F7
:109D100000680149086070470048004000BFFEE746
:109D200003B401984100009850EAC12018BF0420F4
:109D30004A0D18BF40F0010040F2FF72B2EB515FD4
:109D400008BF40F00200012808BF052002B070479C
:109D50004100080218BF04200A0E18BF40F001009D
:109D60004FF07F4232EA010108BF40F002000128B3
:109D700008BF052070470146C1F3C750FF2801D036
:109D8000012070470020FCE702480068C0F3022071
:109D9000704700000CED00E010B5002804DB0A0756
:109DA000130E054A135406E00A07140E034A00F086
:109DB0000F031B1FD45410BD00E400E018ED00E0B9
:109DC000EFF305807047000010B54FF00E402DED09
:109DD000028BB0EE408A18EE104A00EB4400B0F15E
:109DE000506F4AD84FF0FC40B0EB440F22D2B0EE97
:109DF000C80AF7EE000A30EEC00AF6EE000A60EE7E
:109E0000208A18EE900A02F09FFA01EE100A14F070
:109E1000004F1DBFDFED2D0A9FED2D0AB1EE411A57
:109E2000DFED2C0A08BF9FED2C0AF8EE001A21EE98
:109E3000218A05E0DFED290A68EE088AB0EE600AA3
:109E40009FED271ADFED271A30EE080A48EE811A37
:109E50009FED251A08EEA11ADFED241A48EE811AAB
:109E60009FED231A08EEA11A68EE281ABDEC028BAA
:109E700001EE810A30EE200A10BD4FF0E440B0EB55
:109E8000440F0CD918EE100AFFF762FF042808BF30
:109E900000F02CFEB0EE480ABDEC028B10BD4FF076
:109EA0007F40B0EB440F07D2B0EE480ABDEC028B06
:109EB000BDE8104000F00CBE0120F6F77AFBBDECC7
:109EC000028BBDE8104000F009BE00000000C9BFD1
:109ED00022AAFDB90000C93F22AAFD3900000000F6
:109EE00024FE1C3DC78AD83C1E67383D1B93993D14
:109EF000AFAA2A3E0000000070B59B482DED020B72
:109F00002DED068B079D25F00044A04218DC9748F4
:109F1000844202DC0AD1069840B19DED060BBDECEF
:109F2000068B02B0BDE8704000F0AEBD002DCCBF86
:109F30009FED8F0B9FED900BBDEC068B02B070BDBB
:109F40008F48A04215DD8F48A042D8BF4FF0FF34A4
:109F500058DD9DED060B51EC100BFFF7E1FE0428D8
:109F600008BF00F0A5FD9DED060BBDEC068B02B011
:109F700070BD9DED060B51EC100B00F0D5FECDE948
:109F8000060181489FED828BA0423CDD8248A042C1
:109F90001FDD00249FED82AB9DED060B53EC1A2BC9
:109FA00051EC100B04F000F99DED060B41EC190B80
:109FB00053EC1A2B51EC100B04F0C6FB53EC182B8E
:109FC00004F0CCFC53EC192B04F0A2F9CDE9060106
:109FD00049E09DED060B012453EC182B51EC100BBE
:109FE00004F0E2F89DED060B41EC190B53EC182B35
:109FF00051EC100B04F0B2FC53EC192B04F088F96F
:10A00000CDE906012FE06848A0421FDD02249FED44
:10A01000689B9DED060B53EC192B51EC100B04F0D3
:10A0200093FB53EC182B04F0BFF89DED060B41ECAD
:10A03000180B53EC192B51EC100B04F08FFC53EC64
:10A04000182B04F065F9CDE906010CE09DED060B37
:10A05000032453EC102B9FED580B51EC100B04F024
:10A0600057F9CDE906019DED060B53EC102B51EC91
:10A07000100B04F069FB41EC180B53EC182B04F0A7
:10A0800063FB41EC190B4E480621B0EE490AF0EE95
:10A09000690A784400F07CFC53EC182B51EC100B4F
:10A0A00004F052FB41EC180B4648B0EE490AF0EEC2
:10A0B000690A0521784400F06BFC53EC192B51EC34
:10A0C000100B04F041FB41EC100B51EC180B53EC5E
:10A0D000102B002C0EDA04F067F89DED061B53ECF4
:10A0E000112B04F031FB9DED061B53EC112B04F0FA
:10A0F00029FC35E004F058F89DED061B53EC112BBC
:10A1000004F022FB41EC100B2F48784400EBC40014
:10A1100090ED001B51EC100B53EC112B04F01EFCC6
:10A120009DED061B53EC112B04F018FC41EC100BB9
:10A130002648784400EBC40090ED001B51EC100B56
:10A1400053EC112B04F0FEFB41EC100B002DA2BFD1
:10A15000BDEC068B02B070BD51EC100B03F0E6FFB6
:10A1600041EC100B01E70000000010440000F07FFC
:10A17000182D4454FB21F93F182D4454FB21F9BFFD
:10A180000000DC3F0000203E0000F33F0000000024
:10A19000000000000000F03F0000E63F000000006B
:10A1A00000000000000000400080034000000000AC
:10A1B000000000000000F83F000000000000F0BFB9
:10A1C000FA4D0000B04D00003A4D0000F24C000086
:10A1D00070B56F4E2DED040B2DED048B82B0DDF8C4
:10A1E00024C0DDE907235C422CF000411C4341EA16
:10A1F000D474069D22F00040B44205D86C422C4332
:10A2000040EAD474B4420BD99DED081B9DED060BBA
:10A2100002B0BDEC048B04B0BDE8704000F03EBC61
:10A22000ACF14054A4F17F641C430BD0022404EA37
:10A23000AC7444EAD27405439FED578B9FED582BC5
:10A2400007D015E09DED060B51EC100B00F000FD62
:10A2500042E0002C11BF012C9DED060B02B0BDECBD
:10A26000048B04BF04B070BD022C38D0032C3BD04B
:10A270000B439FED4D1B9FED4E0B0AD0B14218D101
:10A28000B04209D121F0804120F08040099107902F
:10A290000FE0002A15DA10E0474B7B44002C08BF82
:10A2A00093ED000B0DD0012C10D0022C17D0032CF5
:10A2B0001AD0B0421DD1002A03DAB0EE410AF0EE06
:10A2C000610A02B0BDEC048B04B070BD93ED000BCD
:10A2D00051EC100B03F02AFF41EC100BF1E7B0EE4C
:10A2E000480AF0EE680AECE7B0EE420AF0EE620AC5
:10A2F000E7E7401A00159FED329B3C28C8BF8DED63
:10A30000000B17DCBCF1000FBCBF10F13C0F8DED52
:10A31000009B0FDB9DED080B53EC102B9DED060B06
:10A3200051EC100B03F0F4FF00F0FEFC00F090FC89
:10A33000CDE90001B4B1012C10D0022C9FED220B0D
:10A3400053EC102B9DED000B51EC100B19D004F0C9
:10A3500005FB53EC182B04F001FBBDE7019880F0DE
:10A36000004001909DED000B53EC192B51EC100BAC
:10A3700004F026F904BF0220F6F71BF99DED000B4F
:10A380009FE704F0EBFA53EC182B04F0DBFAA3E799
:10A390000000F07F00000000182D4454FB2109400C
:10A3A000182D4454FB2109C0182D4454FB21F9BF3A
:10A3B000182D4454FB21F93F224C000000000000FE
:10A3C0000000000000000000075C143326A6A13C3A
:10A3D00070B54FF068422DED048BF0EE408A18EE18
:10A3E000900AB0EE608A18EE101A02EB4003B3F147
:10A3F000654F3CBF02EB4102B2F1654F7DD200BF19
:10A40000C0F3C753C1F3C7529A1A1B2A09DD10F0D3
:10A41000004F14BF9FED830A9FED830ABDEC048BB0
:10A4200070BD12F11A0F36DA11F0004F09D010F09A
:10A43000004F0CBF9FED7D0A9FED7D0ABDEC048BA4
:10A4400070BD88EE889A19EE100AFFF781FC042887
:10A4500008BF00F04BFB18EE900AFFF779FC0546A9
:10A4600018EE100AFFF774FC044619EE100AFFF705
:10A470006FFC042D18BF052D08D1042C18BF052C26
:10A4800004D1002804BF0220F6F793F8B0EE490A81
:10A49000BDEC048B70BD4200B2EB410F3AD910F015
:10A4A000004F19BFDFED630A9FED630ADFED630A1A
:10A4B0009FED630AB0EE481A0A46B1EE688A80F052
:10A4C0000041F0EE418A10460A1A5200B2F1807F34
:10A4D00034D2484010F0004FDFED5A1A9FED5A2A4F
:10A4E0001DBFBEEE001A70EEE10A30EE420AB6EE73
:10A4F000001A08BF70EEA10A00E040E008BF30EE8D
:10A50000020AB0EE682A01EE482A08EE818AC2EEFD
:10A51000081A15E011F0004F04BF9FED4C0AF0EE51
:10A52000400AD1D010F0004F19BFDFED490A9FED6E
:10A53000490ADFED490A9FED490AC5E7C8EE881AC6
:10A5400021EEA11A9FED462ADFED462A41EE022AAE
:10A550009FED452A01EE222ADFED442A41EE022A30
:10A560009FED432ABDEC048B01EE222A21EE811AD5
:10A5700001EE020A30EE210A30EE200A70BD4FF0E3
:10A580007F42B2EB400F28BFB2EB410F09D2F0EE91
:10A59000480AB0EE680ABDEC048BBDE8704000F0DC
:10A5A0009ABA40EA01035B0008BF41F0FF410BD0BB
:10A5B000B2EB400F08BFB2EB410F08D120F0804052
:10A5C00008EE900A21F0804108EE101A18E7B2EB6D
:10A5D000400F12BF5FEA410340F0FF4001F000412D
:10A5E0003FF40EAFB2EB410F12BF5FEA400200F042
:10A5F000004041F0FF413FF403AF4A0092EA4003BC
:10A600003FF5FEAE002AACBF9FED1A0A9FED1A0A75
:10A6100068EE808A28EE008A18EE900A18EE101A6A
:10A62000EEE60000DB0FC9BFDB0FC93FDB0F49407F
:10A63000DB0F49C00000C9BF22AAFDB90000C93F15
:10A6400022AAFD390060ED3EC30ACE3700000000AB
:10A65000000049C022AA7DBA0000494022AA7D3AE2
:10A660002DAD65BD8FB8D53D0FB511BE61C84C3E4F
:10A67000A8AAAABE0000804F0000802F10EE101A7A
:10A6800008B5444A6846B2EB410F28D94FF0E6407E
:10A69000B0EB410F94BF00204FF0FF3000900098C6
:10A6A000002861DB60EE000A10F0010F45D010F0C9
:10A6B000020FDFED391A9FED391A00EEE11ADFEDD6
:10A6C000381A40EE811A21EEA01AF0EE400A40EE50
:10A6D000010A08BFF1EE600AB0EE600A08BD314B16
:10A6E00021F0004293423CD911F0004FDFED2E0AD9
:10A6F00020EE201ADFED2D0A19BF31EE601A71EE3F
:10A70000200A31EE201A71EE600ABDEEE01A11EE59
:10A71000100A9FED271A00F0030000EEC10A9FED1A
:10A72000251A009000EEC10A9FED231A00EEC10A1F
:10A730009FED221A00EEC10AB1E79FED211A9FEDAD
:10A74000210A10F0020F00EE810A9FED1F1A00EEA1
:10A75000801AB7EE000A00EE810A18BFB1EE400A77
:10A7600008BD00F0CBF99AE710EE100A4000B0F1F6
:10A770007F4F3CBFB7EE000A08BD07D14FF0010084
:10A78000F5F717FFBDE8084000F0A8B9BDE808409C
:10A7900000F09EB9B61F927E336D4C39DA82083CC8
:10A7A000A0AA2ABE490E494683F9223F0000004B69
:10A7B0000000C93F00A0FD390020A2331A61342CEB
:10A7C000B93AB2BACA9F2A3DDDFFFFBE10B52DEDE2
:10A7D000028BB0EE608AF0EE408A18EE101A18EE86
:10A7E000900A04F0DDF900F07040B0F1005F0CD089
:10A7F00018EE100A20F00040C0F1FF40C00F02BF69
:10A80000B0EE480ABDEC028B10BDB0EE680ABDEC9C
:10A81000028B10BD00B510EE101A2DED028B81B029
:10A820004D4A6846B2EB410F3CD94FF0E640B0EBE1
:10A83000410F94BF00204FF0FF3000900098B0EE21
:10A84000408A00285FDB28EE080ADFED440A9FED0E
:10A85000441A00EE201ADFED430A40EE010A9FED94
:10A86000421A00EE201ADFED410A10F0010F40EE0F
:10A87000010A9FED3F1A00EE201A61EE000AB0EEC9
:10A88000480A08EE200A02BF01B0BDEC028B00BDF1
:10A89000BFEE001A01B0C1EE000ABDEC028BB0EEB3
:10A8A000600A00BD334B21F00042934228D911F0D9
:10A8B000004FDFED310A20EE201ADFED300A19BF1C
:10A8C00031EE601A71EE200A31EE201A71EE600A44
:10A8D000BDEEE01A11EE100A9FED291A00F00300F8
:10A8E00000EEC10A9FED271A009000EEC10A9FED0D
:10A8F000261A00EEC10A9FED251A00EEC10A9DE757
:10A9000000F0FCF89AE718EE100A4000B0F17F4F13
:10A910000DD218EE100AFFF71BFA042808BF00F04A
:10A92000E5F8B0EE480A01B0BDEC028B00BD09D1DC
:10A930000120F5F73EFE01B0BDEC028B5DF804EBA3
:10A9400000F0CCB801B0B0EE480ABDEC028B5DF867
:10A9500004EB00F0BDB80000B61F927EBBE9223CBC
:10A960000C6D063B8A76CE3CACB5593D35A1083E10
:10A9700029AAAA3E490E494683F9223F0000004B0E
:10A980000000C93F00A0FD390020A2331A61342C19
:10A9900070B504462DED028B4D1E00EBC500B0EEE8
:10A9A000408AF0EE608A90ED000B35F0060017D07B
:10A9B00053EC182B51EC100B03F0C6FE41EC100BBE
:10A9C0006D1E04EBC50090ED001B51EC100B53EC19
:10A9D000112B03F0E9FB41EC100B35F00600E7D139
:10A9E000022D36D0042D1CD0062D1CBFBDEC028BD1
:10A9F00070BD53EC182B51EC100B03F0A5FE94ED39
:10AA00000A1B53EC112B03F0CFFB53EC182B03F074
:10AA10009BFE94ED081B53EC112B03F0C5FB41EC9E
:10AA2000100B53EC182B51EC100B03F08DFE94ED32
:10AA3000061B53EC112B03F0B7FB53EC182B03F060
:10AA400083FE94ED040B53EC102B03F0ADFB41ECB3
:10AA5000100B53EC182B51EC100B03F075FE94ED1A
:10AA6000021B53EC112B03F09FFB53EC182B03F04C
:10AA70006BFE94ED001B53EC112B03F095FBBDEC2A
:10AA8000028B41EC100B70BD10B553EC102B51EC48
:10AA9000100B03F089FB41EC100B10BD10B553EC0B
:10AAA000112B51EC100B03F07FFB41EC100B10BD90
:10AAB0009FED050B10B553EC102B51EC100B03F070
:10AAC00043FE41EC100B10BD000000000000001020
:10AAD00030EE000A704730EE200A7047DFED020AC0
:10AAE00080EEA00A70470000000000009FED020AFF
:10AAF00020EE000A70470000000000102DE9F00170
:10AB00004FF07F42B2EB410F9FBF4FF0FF3101602A
:10AB1000BDE8F00170474FF0004242EA0123C1F363
:10AB2000C752783A551112F01F0C434CCCF1200655
:10AB30007C44C1F3C752A2F178024FEA621204EBDF
:10AB4000820254F8254008BFD2E9015612D0556858
:10AB500004FA0CF425FA06F73C43976805FA0CF55D
:10AB600027FA06F8D26807FA0CFCF24045EA080515
:10AB70004CEA0206A4FB034CA5FB0352A6FB0363AD
:10AB80001D449D4234BF012600261319334416B1DB
:10AB9000934202D903E0934201D2012200E0002255
:10ABA000624402F1200C9206DC0C42EA443200EED0
:10ABB000102A5B03DFED210AF8EEC01A00EE103A0E
:10ABC0004FEA9C1C11F0004FB8EE400AC0F800C0DC
:10ABD00020EE201A00EE105ADFED190AB8EE400AF6
:10ABE00020EE200A71EE810A70EE800A10EE902AA3
:10ABF00002F500626FF30B0200EE902A70EEE11A8C
:10AC000031EEC11ADFED101A30EE411A9FED0D0A38
:10AC100020EE800A01EE210A9FED0C1A00EE810A57
:10AC200004BFBDE8F0017047CCF180510160BDE880
:10AC3000F001B1EE400A7047944300000000003676
:10AC40000000802C22AAFD29DB0FC92F0000C92F8C
:10AC500010B541EC100BFFF74FF951EC100B10BD84
:10AC600070470000074800680749B0FBF1F007494A
:10AC70000870044800684FF47A71B0FBF1F00449A1
:10AC8000086070471400002040420F00B40000200C
:10AC9000B80000202DE9F04707463E4656B900BFF0
:10ACA000502080F31188BFF34F8FBFF36F8F00BF29
:10ACB00000BFFEE717480068864201D1002426E065
:10ACC00001F0DEFB75691448D0F800801348D0F815
:10ACD000009001F0FFFB454501D04D4501D1022414
:10ACE00015E00F4885420BD1B06A38B996F860007C
:10ACF000012801D102240AE0032408E0022406E02E
:10AD00000848854200D00DB9042400E00124204603
:10AD1000BDE8F087180000201C0000202000002063
:10AD2000F80A0020E40A002082B0CDE9000121F0F9
:10AD3000004001909DED000B02B051EC100B7047EC
:10AD400000207047F9F7A4FFFEF762FAFDF7C4FB95
:10AD5000FDF76EFBFDF724FBFDF746FBFDF7F0FC6E
:10AD6000FDF712FDFDF76AFDFDF7AAFDFDF730FDC9
:10AD7000FDF7AAFCFDF7C6FCFDF786FD00F064F8C0
:10AD8000FDF792FB00F092F800BFFEE770B50446B5
:10AD9000049D601AEE1A7043561A90FBF6F01844A0
:10ADA00070BD70B50546FFF70BF810B16FF00504E4
:10ADB00004E0002415B1284601F088FC204670BD4F
:10ADC000F8B50646FEF7FCFF10B16FF005050FE081
:10ADD000002502F0B9FE00900098341A34B1E00F5B
:10ADE00020B92146684601F09FFC01E06FF00305A1
:10ADF0002846F8BD10B502F097FE28B1012806D00C
:10AE0000022803D102240AE0032408E000BF054819
:10AE10000068012801D1012400E0002400BF00BF28
:10AE2000204610BD7000002010B5FEF7C9FF18B114
:10AE300002F090FE044602E002F086FE0446204640
:10AE400010BD4FF47A70704710B5FEF7B9FF10B11E
:10AE50006FF0050409E00648006820B901200449A4
:10AE60000860002401E04FF0FF34204610BD0000D0
:10AE70007000002010B5FEF7A3FF10B16FF00504BD
:10AE800012E002F051FE20B1012809D0022806D1BB
:10AE900001E0012407E001F029FE002403E000BFE7
:10AEA0004FF0FF3400BF00BF204610BD70B5FEF765
:10AEB00087FF10B16FF005041FE0114800680128FA
:10AEC00019D100BF801F0021002804DB0A07130EE0
:10AED0000C4A135406E00A07150E0B4A00F00F0344
:10AEE0001B1FD55400BF00BF02200549086001F0B8
:10AEF0009FFD002401E04FF0FF34204670BD0000AC
:10AF00007000002000E400E018ED00E010B5FEF74E
:10AF100057FF10B16FF0050418E002F005FE20B1F4
:10AF200001280FD002280CD109E0012402F0FEFF15
:10AF3000012803D002F0F8FD00B9A41E05E00024AA
:10AF400003E000BF4FF0FF3400BF00BF204610BD3C
:10AF50002DE9F84307460D4691461C463E464FF004
:10AF60000008FEF72DFFE0B10EB105B114B16FF08E
:10AF7000030828E0002000906A462946304602F087
:10AF800047FA012802D06FF002081CE00098D0B107
:10AF90004FF080500D490860BFF34F8FBFF36F8FA4
:10AFA00011E006B115B96FF003080CE022462946FE
:10AFB000304602F079F9012805D014B16FF001088C
:10AFC00001E06FF002084046BDE8F88304ED00E0C0
:10AFD0002DE9F84305460E4614464FF00009FEF7EA
:10AFE000EFFE00283ED1002D3CD0002E3AD0471E67
:10AFF000BCB1A06858B1E068502808D3206930B1CE
:10B0000005FB06F06169814201D301270AE0A068CF
:10B0100040B9E06830B9206920B9606910B90027EB
:10B0200000E00027012F09D100200090314628467A
:10B03000A368226901F005FF814606E02FB90022CE
:10B040003146284601F0D0FE8146B9F1000F09D003
:10B0500014B1D4F8008001E04FF0000841464846A2
:10B0600001F0F8FA4846BDE8F88300002DE9F843FE
:10B0700007460D4691461C463E464FF00008FEF737
:10B080009FFEE8B10EB105B114B16FF003082AE0DC
:10B090000020009000236A462946304602F062F8FC
:10B0A000012802D06FF002081DE00098D8B14FF0DF
:10B0B00080500E490860BFF34F8FBFF36F8F12E0CF
:10B0C00006B115B96FF003080DE0002322462946AA
:10B0D000304601F073FF012805D014B16FF001086C
:10B0E00001E06FF002084046BDE8F88304ED00E09F
:10B0F00070B505462E46FEF763FE10B16FF00504ED
:10B1000008E016B96FF0030404E000240021304683
:10B1100001F008FF204670BD2DE9F04104460D46C0
:10B1200024F0010604F001080027FEF749FE08B1EB
:10B13000BF1F1FE016B96FF003071BE0B8F1000F47
:10B140000CD02946304602F0A5FA012812D015B1DC
:10B150006FF001070EE06FF002070BE02946304662
:10B1600002F0BCF9012805D015B16FF0010701E02C
:10B170006FF002073846BDE8F0812DE9F04704463C
:10B180000026FEF71DFE00284DD10CB1676800E0D7
:10B19000002707F0010008B1012500E0002507F0B5
:10B1A000080008283FD04FF0FF3874B1A06828B1DC
:10B1B000E068502802D34FF0010808E0A06830B9D9
:10B1C000E06820B94FF0000801E04FF00008B8F146
:10B1D000010F0CD12DB10420A16801F0F0FD06464D
:10B1E00012E00120A16801F0EAFD06460CE0B8F18A
:10B1F000000F09D125B1042001F0D0FD064603E07F
:10B20000012001F0CBFD06464EB114B1D4F80090F8
:10B2100001E04FF000094946304601F01BFA16B133
:10B220000DB146F001063046BDE8F0872DE9F0414A
:10B23000044624F0010504F001070026FEF7C0FDD6
:10B2400008B1B61F16E015B96FF0030612E03FB162
:10B25000284602F005F801280CD06FF0020609E03C
:10B2600000231A461946284601F0A8FE012801D0FD
:10B270006FF002063046BDE8F0810000FEB50446DE
:10B280000D46264616B105F0004018B16FF00300D8
:10B2900002902EE04FF0FF300290FEF791FDE0B1FA
:10B2A0000020019001A80023012229460090304689
:10B2B00002F082FB002002AB0246014600903046BD
:10B2C00002F07AFB0198A0B14FF080500A49086063
:10B2D000BFF34F8FBFF36F8F0BE00023012229468E
:10B2E000304602F0D5FA02AB00221146304602F099
:10B2F000CFFA0298FEBD000004ED00E02DE9FC5FEE
:10B30000054689461646FEF75BFD10B16FF0050451
:10B310004AE005F0004010B16FF0030444E009F08A
:10B320000200022802D14FF0000A00E0AA460024E1
:10B33000374602F009FC009000BF3B4601AA514687
:10B34000002002F0B3FC8046B8F1010F22D12C405E
:10B350000198044309F0010040B105EA0400A84245
:10B3600000D120E056B96FF002041CE005EA0400A9
:10B3700000B118E016B96FF0020414E002F0E4FB2B
:10B380000099A0EB010BBB4501D9002708E0A7EB12
:10B390000B0705E016B96FF0020401E06FF001043D
:10B3A000B8F1000FC9D100BF2046BDE8FC9F10B521
:10B3B00002F0B4FB0446204610BD2DE9FF4780464D
:10B3C0008946144600200390FEF7FAFC00284ED16F
:10B3D000B8F1000F4BD0802618258246471E44B393
:10B3E000206808B1D4F800A0A06900B1A5692DB10A
:10B3F000382D03D8207900F0010018B1002004B0E6
:10B40000BDE8F087606908B160698608A06840B14E
:10B41000E068642805D3206918B1606908B1012784
:10B4200008E0A06830B9E06820B9206910B90027A9
:10B4300000E00027012F0CD12169A0684B4632465D
:10B44000CDE9005102905146404602F0C3F9039005
:10B450000DE067B903A8B2B24B465146CDE90050A2
:10B46000404602F085F9012801D00020039003989E
:10B47000C5E72DE9F04106463746FEF7A1FC10B1BD
:10B480006FF0050410E017B96FF003040CE03846C4
:10B49000FFF700FC0546042D04D00024384601F0D7
:10B4A000ADF901E06FF002042046BDE8F081000034
:10B4B0002DE9F04105460E46164807681648006813
:10B4C000001D00F078FF681C38B936B112480168D9
:10B4D000091D124800F0C7FF1AE07C190E480068E9
:10B4E0004460BC4207D20C480168091D0C48006842
:10B4F00000F09FFF0CE008480168091D094800683A
:10B5000000F097FF08480068844201D206480460B2
:10B51000BDE8F0812C00002018000020F80A00206F
:10B52000200000201C0000204800002010B5044628
:10B5300000F0A6FF24480068401C23490860234807
:10B54000006840B9214804600846006801280DD110
:10B5500000F018FA0AE01E48006838B91B48006875
:10B56000C06AE16A884201D8184804601948006836
:10B57000401C1849086008460068A0641649E06A43
:10B580000968884202D91449E06A0860E16A01EB5F
:10B590008101124A02EB8100211D00F064FF00F0DE
:10B5A00099FF0B48006868B108480068C06AE16A02
:10B5B000884207D24FF0805009490860BFF34F8F8F
:10B5C000BFF36F8F10BD000028000020180000207E
:10B5D00034000020440000203000002048060020F5
:10B5E00004ED00E008B500F04BFF12480068E8B930
:10B5F000114800F00EFF114800F00BFF0E481049F3
:10B6000008600E480F49086000200F4B0F4A1021B8
:10B6100000900A2001F015FC064908600846006801
:10B6200020B10BA10348006801F014F800F052FFAC
:10B6300008BD0000640000200C0B0020200B00203F
:10B640005C00002060000020340B0020840B0020F0
:10B65000546D72510000000010B516E000F010FFAC
:10B660000C48C068C468201D00F0A5FE0A480068A8
:10B67000401E0949086009480068401E07490860E3
:10B6800000F028FF204600F05FF80448006800281A
:10B69000E4D110BDE40A002028000020240000208E
:10B6A00070B504460D46206C70B1216CE068014411
:10B6B000E160D4E90210884201D32168E1602846A4
:10B6C000226CE168F4F7C7FE70BD2DE9F041044635
:10B6D0000F4615464FF00008A66B206C48B920684D
:10B6E00000282CD1A06802F031FB80460020A06029
:10B6F00025E07DB93946226C6068F4F7ACFE216C18
:10B70000606808446060D4E90101884217D320686A
:10B71000606014E03946226CE068F4F79CFE216C0E
:10B72000E068411AE1602168E068884203D2216C38
:10B73000A068411AE160022D01D106B1761E701C8D
:10B74000A0634046BDE8F08110B5044694F861005E
:10B7500030B9206B00F0DCFE204600F0D9FE1AE084
:10B7600094F86100012803D1204600F0D1FE12E0D8
:10B7700094F86100022801D1012000E0002050B9B6
:10B7800000BF502080F31188BFF34F8FBFF36F8F3E
:10B7900000BF00BFFEE710BD01464A6A22B10A6B36
:10B7A0001268C2F1380000E0002070470146084AE4
:10B7B000126812680AB9012200E000220A600A68D1
:10B7C00022B9034A1268D268106800E0002070476E
:10B7D0005C00002030B54FF4C043174800F0070468
:10B7E0002CB1C01D20F00700134C041B1B1B02468C
:10B7F000124C22600024114D6C60D018083820F0E3
:10B8000007000F4C206000240D4D2D686C600C4D1E
:10B810002D682C601146441A4C60094C24680C6059
:10B82000084D4C682C60084D4C682C604FF000446B
:10B83000064D2C6030BD0000EC120020740000208A
:10B840007C00002084000020800000209000002068
:10B8500000BFFFF701FF064800680128F9D94FF043
:10B86000805004490860BFF34F8FBFF36F8FF0E73C
:10B870004806002004ED00E010B5044654B1002055
:10B88000A06020600021E16000231A46194620468E
:10B8900001F094FB10BD2DE9F04106460D46174618
:10B8A0009846069C0DB9246000E02760E663256495
:10B8B0000121204601F036FB84F84C80BDE8F08180
:10B8C0002DE9F05F82460E4691469B460A9F0C9CEE
:10B8D0004FEA8901A522206BF4F734FEA9F101009B
:10B8E000216B01EB800828F0070808F0070008B971
:10B8F000012000E0002050B900BF502080F31188E3
:10B90000BFF34F8FBFF36F8F00BF00BFFEE7C4F8D8
:10B91000448086B1002507E0715D04F13400415593
:10B92000705D00B902E06D1C102DF5D300BF002141
:10B930004320015502E0002084F83400382F00D362
:10B940003727E762276500206065201D00F06EFD47
:10B9500004F1180000F06AFD2461C7F13800A0610D
:10B9600064620020A065E06584F860005A46514694
:10B97000404600F081FB20600B9808B10B980460F2
:10B98000BDE8F09F10B5002407E004EB84010F4AE6
:10B9900002EB810000F03DFD641C382CF5D30C480F
:10B9A00000F037FD0B4800F034FD0B4800F031FD8E
:10B9B0000A4800F02EFD0A4800F02BFD0448094912
:10B9C000086004480849086010BD000048060020CF
:10B9D000A80A0020BC0A0020D00A0020E40A0020A7
:10B9E000F80A00201C0000202000002010B50146AD
:10B9F000164800E0006803688B42FBD302464368A8
:10BA000013448B4204D143684C682344436001468D
:10BA10000A464B6813440468A34211D10C4C0368D6
:10BA20002468A34208D04B680468646823444B60D0
:10BA300003681B680B6005E0054B1B680B6001E0A9
:10BA400003680B60884200D0016010BD74000020C4
:10BA50007C0000202DE9F04104460D4616461F46A5
:10BA60004FF0000865602461B5420CD8F01BA16955
:10BA7000884202D34FF0010811E0211D09480068F7
:10BA800000F0D7FC0BE0BE4204D2BD4202D34FF01F
:10BA9000010804E0211D0448006800F0CAFC40468B
:10BAA000BDE8F081600000205C00002070B5054614
:10BAB00000F0E6FCA86B08B9012400E0002400F0C7
:10BAC00009FD204670BD70B5054600F0D9FCA86B95
:10BAD000E96B884201D1012400E0002400F0FAFC67
:10BAE000204670BDF8B505460F461A480068C06884
:10BAF000C468201D00F05FFC94F8280000F00400EA
:10BB0000E8B1A06941192B463A462046FFF7A2FF4B
:10BB1000D8B1002003462A4601460090204602F094
:10BB2000C3FA064656B900BF502080F31188BFF310
:10BB30004F8FBFF36F8F00BF00BFFEE705E094F8A3
:10BB4000280020F0010084F828002046216A884758
:10BB5000F8BD00005C000020F0B587B0A0E00398BD
:10BB6000002811DA04AE56B900BF502080F31188C6
:10BB7000BFF34F8FBFF36F8F00BF00BFFEE7D6E963
:10BB80000020B168904700BF03980028E6DB059CC1
:10BB9000606908B9012000E0002010B9201D00F004
:10BBA0000AFC02A800F0DEF8054603980A2875D2C0
:10BBB000DFE800F009050739416306083A4200BF93
:10BBC00000BF00BF00BF94F8280040F0010084F8D7
:10BBD00028000498A269811803462A462046FFF7E8
:10BBE00039FFF8B12046216A884794F8280000F010
:10BBF0000400B8B1002000900498A1694218002305
:10BC00001946204602F050FA074657B900BF5020A7
:10BC100080F31188BFF34F8FBFF36F8F00BF00BF5A
:10BC2000FEE700BF3BE000BF94F8280020F00100D1
:10BC300084F8280033E000BF94F8280040F00100A9
:10BC400084F828000498A061A06908B1012000E0F0
:10BC5000002050B900BF502080F31188BFF34F8FF0
:10BC6000BFF36F8F00BF00BFFEE7A06941192B46ED
:10BC70002A462046FFF7EEFE11E094F8280000F077
:10BC8000020018B9204600F043FC05E094F82800B3
:10BC900020F0010084F8280001E0FFE700BF00BFAA
:10BCA000002203A90448006801F0FEFA00287FF48E
:10BCB00056AF07B0F0BD000064000020F8B505469F
:10BCC0000C4600F013FF684600F04CF8064600985A
:10BCD00020BB44B9B54206D802F028F931462846BF
:10BCE000FFF700FF1CE03CB10E480068006808B98F
:10BCF000012000E000200446A91B22460A480068F3
:10BD000000F0BEFC02F012F950B94FF08050074924
:10BD10000860BFF34F8FBFF36F8F01E002F006F9A9
:10BD2000F8BD0000600000206400002004ED00E089
:10BD30000A490968096809B9012100E0002121B117
:10BD40004FF0FF31064A116006E004490968C968EE
:10BD5000C868034A41681160704700001C00002059
:10BD60004800002070B5044601F0EEFE0546074885
:10BD70000068854204D200F00BF80120206001E049
:10BD80000020206001480560284670BD6C0000203E
:10BD90002DE9F84334E025480068C0680568234869
:10BDA0000068C068C468201D00F005FB2046216AB9
:10BDB000884794F8280000F0040008B3A0694619E9
:10BDC000AE4207D966602461211D1848006800F062
:10BDD00030FB15E0002003462A460146009020462D
:10BDE00002F062F9074657B900BF502080F311886E
:10BDF000BFF34F8FBFF36F8F00BF00BFFEE700BFE1
:10BE00000A480068006808B9012000E00020002806
:10BE1000C1D00648D0F80080054800680349086092
:10BE20000348C0F80080BDE8F88300005C000020F3
:10BE3000600000200E480068401C08B9012000E0A6
:10BE4000002050B900BF502080F31188BFF34F8FFE
:10BE5000BFF36F8F00BF00BFFEE700BF502080F32D
:10BE60001188BFF34F8FBFF36F8F00BF00BFFEE796
:10BE70009400002008B500BF6846FFF797FC044611
:10BE800020460099FFF71AFFFFF766FEF4E770B54A
:10BE9000044600F0F5FA94F9455010E0606A08B9DC
:10BEA000012000E0002038B904F1240001F0F2FF85
:10BEB00018B100F013FD00E003E0681E45B2002D4C
:10BEC000ECDC00BFFF2084F8450000F003FB00F02D
:10BED000D7FA94F9445010E0206908B9012000E035
:10BEE000002048B904F1100001F0D4FF08B100F0BF
:10BEF000F5FC681E45B200E001E0002DECDC00BF5F
:10BF0000FF2084F8440000F0E5FA70BD2DE9F0410F
:10BF100004464FF0000800F0E9FD4948006808B900
:10BF2000FFF758FC474800682040002870D1D4B182
:10BF3000083404F00700B0B104F00700C0F10800B5
:10BF4000044404F0070008B9012000E0002050B9C3
:10BF500000BF502080F31188BFF34F8FBFF36F8F66
:10BF600000BF00BFFEE7002C52D037480068844273
:10BF70004ED8364E3046056801E02E462D6868687A
:10BF8000A04202D228680028F7D12D4800688542D7
:10BF90003ED0306800F10808286830606868001BEF
:10BFA000102819D92F1907F0070008B9012000E05F
:10BFB000002050B900BF502080F31188BFF34F8F8D
:10BFC000BFF36F8F00BF00BFFEE76868001B78609B
:10BFD0006C603846FFF70AFD1B4968680968081A53
:10BFE000194908600846006819490968884203D25F
:10BFF00015480068164908601249686809680843CE
:10C0000068600020286013480068401C11490860DF
:10C0100001F08CFF08F0070008B9012000E00020C3
:10C0200050B900BF502080F31188BFF34F8FBFF38A
:10C030006F8F00BF00BFFEE74046BDE8F081000003
:10C040007C00002090000020800000207400002070
:10C0500084000020880000200648006830B10549AF
:10C06000096801F15400496D491C016001480068EC
:10C070007047000018000020001F4FF0807303601D
:10C08000001F21F001030360001F054B03601438FB
:10C090000260001F6FF00203036020387047000049
:10C0A00035BE000870B52DED048B04460D461646CE
:10C0B000B5F90C00B0F5E16F26D101202070B5F97B
:10C0C0000410A1F5437002F014FB41EC190B9FED35
:10C0D000130B53EC102B02F037FB41EC180B02F062
:10C0E00031F8A060B5F9000002F003FB41EC190B38
:10C0F0009FED0C0B53EC102B02F026FB41EC180BC0
:10C1000002F020F8606005E0B5F90C00C82801D104
:10C1100000202070BDEC048B70BD0000EE42B24ADE
:10C120000ADB483FFC90728EDF3F623F10B5192159
:10C130000148FCF709FE10BD7B7C002030B52DEDD9
:10C14000048B81B005460C4605B11CB901B0BDECAD
:10C15000048B30BD6878A97840EA0120C0F30A005A
:10C160002080A878C010E97840EA4110C0F30A00A6
:10C170006080E8788011297940EA8100697940EA95
:10C180008120C0F30A00A08068794010A97940EAB4
:10C19000C110C0F30A00E080A8790011E97940EAF3
:10C1A0000110C0F30A002081E879C011297A40EA21
:10C1B0004100697A40EA4120C0F30A0104F1080015
:10C1C0006181687A8010A97A40EA8110C0F30A017F
:10C1D00004F10800A181A87A4011E97A40EAC1007F
:10C1E00004F10801E081287B697B40EA0120C0F36B
:10C1F0000A0104F108002182687BC010A97B40EA93
:10C200004110C0F30A0104F108006182A87B80118B
:10C21000E97B40EA8100297C40EA8120C0F30A01E1
:10C2200004F10800A182287C4010697C40EAC1101A
:10C23000C0F30A0104F10800E1822088A0F58060C3
:10C2400000B220806088A0F5806000B26080A08885
:10C25000A0F5806000B2A080E088A0F5806000B208
:10C26000E0802088183000B2208060884042183872
:10C2700000B26080A088C0F53F7000B2A080E08866
:10C28000183000B2E0804FF42F700090B4F9020033
:10C290002A4B40F2B622D91DFEF778FD00B260802D
:10C2A0004FF42F700090B4F90000244B40F2B522F7
:10C2B000991DFEF76BFD00B22080B4F9060002F074
:10C2C00018FA41EC190B9FED1E0B53EC102B02F0EA
:10C2D0003BFA41EC180B02F0AFF900B2E080B4F980
:10C2E000000010F11E0F05DDB4F900001E2801DA70
:10C2F00000202080B4F9020010F11E0F05DDB4F912
:10C3000002001E2801DA00206080B4F9040010F158
:10C310001E0F05DDB4F904001E2801DA0020A080FC
:10C32000B4F9060010F11E0F05DDB4F906001E2851
:10C3300001DA0020E08000BF08E7000044FDFFFFB5
:10C34000000000000000E03F10B500EE100A2DEDE7
:10C35000028BB1EEC08A18EE100A20F00040C0F146
:10C36000FF40C00F0AD010EE100A20F00040C0F1CC
:10C37000FF40C00F04BF0120F4F71BF918EE100AAC
:10C38000BDEC028B10BD00B5034605E04FF47A709A
:10C3900000F005F8581E83B2002BF7DC00BD07E063
:10C3A000322101E04A1ED1B20029FBDC411E88B2D5
:10C3B0000028F5DC704701460A69D1E90130986030
:10C3C000D1E9010358605068884201D18868506003
:10C3D000002008611068401E10601068704700005F
:10C3E000034B0360034B0B60802313607047000016
:10C3F000240C0020880C0020034B0360034B0B60CF
:10C400004FF4807313607047880E0020EC0E0020FC
:10C41000704700F1080141604FF0FF31816000F189
:10C420000801C160016100210160704700210161C4
:10C43000704710B502460B685C1C0CB9106907E028
:10C4400002F1080000E04068446824689C42FAD980
:10C4500044684C604C68A160886041600A6114685F
:10C46000641C146010BD42684A6093688B609368D6
:10C4700059609160086103685B1C036070470000AD
:10C4800000BF502080F31188BFF34F8FBFF36F8F31
:10C4900000BF0E480068401C0C4908600846006850
:10C4A000012812D10A480068C0B208B9012000E092
:10C4B000002050B900BF502080F31188BFF34F8F88
:10C4C000BFF36F8F00BF00BFFEE7704794000020EE
:10C4D00004ED00E00D48006850B900BF502080F323
:10C4E0001188BFF34F8FBFF36F8F00BF00BFFEE710
:10C4F00006480068401E054908600846006820B9E3
:10C50000002080F3118800BF00BF70479400002016
:10C5100070B506463546002E44D0083D2C462249CB
:10C5200060680968084008B1012000E0002050B9A7
:10C5300000BF502080F31188BFF34F8FBFF36F8F80
:10C5400000BF00BFFEE7206808B9012000E000201E
:10C5500050B900BF502080F31188BFF34F8FBFF355
:10C560006F8F00BF00BFFEE70F4960680968084091
:10C57000C0B12068B0B90C49606809688843606040
:10C5800000F0B4FA0949606809680844074908607E
:10C590002046FFF72BFA06480068401C0449086053
:10C5A00001F0C4FC70BD000090000020800000205D
:10C5B0008C00002000204FF0E021086188610648CF
:10C5C00000684FF47A71B0FBF1F0401E4FF0E021AB
:10C5D00048610720086170471400002070B5F3F728
:10C5E0009FFE0446102C16D304F1E02090F8F0537F
:10C5F00015480078854201DB012000E0002050B999
:10C6000000BF502080F31188BFF34F8FBFF36F8FAF
:10C6100000BF00BFFEE70D48006800F4E0600C4971
:10C620000968884201D8012000E0002050B900BF0D
:10C63000502080F31188BFF34F8FBFF36F8F00BF7F
:10C6400000BFFEE770BD0000980000200CED00E088
:10C650009C000020024600200BE0084B53F83030CD
:10C6600033B9064B43F8301003EBC0035A6002E0C5
:10C67000401C0828F1D300BF7047000008060020C6
:10C680002DE9F04105460E4617462C46FFF7F8FE09
:10C6900094F94400401C10B9002084F8440094F937
:10C6A0004500401C10B9002084F84500FFF712FF38
:10C6B000A06B28B93A46314604F1240000F030F965
:10C6C0002046FFF7E4FBBDE8F081000070B50446AA
:10C6D0000025D4B11248006808B9012000E000200C
:10C6E00050B900BF502080F31188BFF34F8FBFF3C4
:10C6F0006F8F00BF00BFFEE700F0F8F90021204671
:10C70000FEF7D6FE01F012FC05463DB94FF0805011
:10C7100004490860BFF34F8FBFF36F8F70BD0000F7
:10C720005000002004ED00E02DE9F04704460F46DC
:10C730004FF0000954B900BF502080F31188BFF3B7
:10C740004F8FBFF36F8F00BF00BFFEE70FB1012017
:10C7500000E0002050B900BF502080F31188BFF3E3
:10C760004F8FBFF36F8F00BF00BFFEE72048006808
:10C7700008B9012000E0002050B900BF502080F32C
:10C780001188BFF34F8FBFF36F8F00BF00BFFEE76D
:10C7900000F0ACF9174806682068C5192068B04257
:10C7A00007D92068A8420BD9B54209D94FF0010931
:10C7B00006E02068A84201D8B54201D94FF001092E
:10C7C0002560B9F1000F03D0A81B0021FEF770FE11
:10C7D00001F0ACFB8046B8F1000F07D14FF080505C
:10C7E00005490860BFF34F8FBFF36F8FBDE8F08737
:10C7F000500000202C00002004ED00E070B505463C
:10C80000FFF73EFE15B92748006800E028460446B9
:10C81000201DFFF7D0FDA06A18B104F11800FFF742
:10C82000CAFD21480068401C1F4908601D48006877
:10C83000844209D1211D1D48FFF715FE1C480068E0
:10C84000401C1B49086009E01A480068401E19494D
:10C8500008602046FEF778FFFFF76AFAFFF73AFE16
:10C8600015480068E8B10F480068844219D11348A0
:10C87000006808B9012000E0002050B900BF502036
:10C8800080F31188BFF34F8FBFF36F8F00BF00BFDE
:10C89000FEE74FF080500A490860BFF34F8FBFF3A7
:10C8A0006F8F70BD1800002044000020E40A0020B3
:10C8B0002400002028000020340000205000002028
:10C8C00004ED00E00349096801600349096841601B
:10C8D00070470000400000202C000020012001498A
:10C8E000086070473C00002070B504460D4654B9FE
:10C8F00000BF502080F31188BFF34F8FBFF36F8FBD
:10C9000000BF00BFFEE70548016818312046FFF769
:10C9100090FD01212846FEF7CBFD70BD18000020D8
:10C9200070B505460E46144655B900BF502080F339
:10C930001188BFF34F8FBFF36F8F00BF00BFFEE7BB
:10C940000648016818312846FFF78DFD0CB14FF0FD
:10C95000FF3621463046FEF7ABFD70BD18000020C3
:10C960002DE9F04706460F4634464FF00109002EE8
:10C9700055D0606D50B900BF502080F31188BFF3CF
:10C980004F8FBFF36F8F00BF00BFFEE7206DB8422F
:10C9900001D23D4600E0256DE06AA8423FD0606DBF
:10C9A00001283CD11F480068844201D0012000E0EA
:10C9B000002050B900BF502080F31188BFF34F8F83
:10C9C000BFF36F8F00BF00BFFEE7D4F82C80E56295
:10C9D000A06900F0004010B9C5F13800A06108EB73
:10C9E0008801114A02EB81016069884201D101206E
:10C9F00000E0002098B1201DFFF7DDFC0B49E06A44
:10CA00000968884202D90949E06A0860E16A01EBD5
:10CA10008101054A02EB8100211DFFF724FDBDE8DD
:10CA2000F087000018000020480600203000002099
:10CA300010B586B000200590049003AA04A905A8AB
:10CA4000FFF7CEFC0022DDE904101346CDE90021FA
:10CA500002901FA12048039A00F0BCFE1F49086005
:10CA60000846006808B1012400E00024012C02D12E
:10CA700001F0DEFA0446012C17D100BF502080F3EC
:10CA80001188BFF34F8FBFF36F8F00BF4FF0FF30A0
:10CA9000134908600120134908600020124908600A
:10CAA000FEF7DEF800F0ACF810E0601C08B10120E1
:10CAB00000E0002050B900BF502080F31188BFF380
:10CAC0004F8FBFF36F8F00BF00BFFEE706B010BDF2
:10CAD00049444C450000000051B800084C000020BB
:10CAE00048000020340000202C000020024800688C
:10CAF000401C0149086070475000002070B539485B
:10CB0000006818B101203849086069E00020364902
:10CB10000860FEF715F93549086008460068344991
:10CB2000096888420BD93349096801F15800896DB9
:10CB30002E4A12682E4B1B68D21A114401602B48F2
:10CB400000682B4908602B480068046B4FF0A5353E
:10CB50002068B0F1A53F0BD16068B0F1A53F07D1C7
:10CB6000A068B0F1A53F03D1E068B0F1A53F05D0C2
:10CB70002048016834310068FFF74AFC1E4801680C
:10CB80000CE051B900BF502080F31188BFF34F8FE4
:10CB9000BFF36F8F00BF00BFFEE7491E01EB8100AE
:10CBA000164A52F8200008B9012000E000200028B1
:10CBB000E7D101EB8102114B03EB8200426852681E
:10CBC000426000F108024368934202D14268526811
:10CBD00042604268D268074B1A600748016000BF94
:10CBE00070BD0000500000203C00002058000020D4
:10CBF00054000020180000203000002048060020CB
:10CC00001CB5524800685249884201D0012000E01A
:10CC1000002050B900BF502080F31188BFF34F8F20
:10CC2000BFF36F8F00BF00BFFEE748480068484968
:10CC3000491E884201D0012000E0002050B900BF09
:10CC4000502080F31188BFF34F8FBFF36F8F00BF69
:10CC500000BFFEE73F49084600780190FF200A46E2
:10CC600010700846007800909DF8000000F0F00079
:10CC70009DF80020904201D1012000E0002050B931
:10CC800000BF502080F31188BFF34F8FBFF36F8F29
:10CC900000BF00BFFEE79DF8000000F050002E4AE4
:10CCA000107007202D4A106009E02C480068401ED3
:10CCB0002A4A10609DF800004006000E00909DF882
:10CCC000000000F080008028EFD024480068C0F108
:10CCD0000700042801D1012000E0002050B900BF66
:10CCE000502080F31188BFF34F8FBFF36F8F00BFC9
:10CCF00000BFFEE7194800680002184A106010469D
:10CD0000008800F4E0601060124A019810700F482B
:10CD10002030006840F470000C492031086008465B
:10CD2000006840F070400860FFF744FC00200C49A8
:10CD30000860F3F7BDFA0B48006840F0404009492D
:10CD40000860F3F7A1FA00201CBD000000ED00E030
:10CD500071C20F4100E400E0980000209C00002018
:10CD60009400002034EF00E010B500BF502080F3A5
:10CD70001188BFF34F8FBFF36F8F00BF00F0F4FE39
:10CD800018B14FF080500449086000BF002080F3C4
:10CD9000118800BF10BD000004ED00E02DE9F04156
:10CDA00004460126002722460021012000F01CF83D
:10CDB00005462846FEF760FD2846BDE8F0812DE9CE
:10CDC000F84304460D4601274FF000082B46002289
:10CDD00011460120009400F034F806463046FEF774
:10CDE0004BFD3046BDE8F8832DE9F84305460E4675
:10CDF00017460DB1012000E0002050B900BF5020BF
:10CE000080F31188BFF34F8FBFF36F8F00BF00BF58
:10CE1000FEE705FB06F808F15000FFF777F8044637
:10CE200064B1A14609F15009002084F846003B4650
:10CE30004A46314628460094FEF72DFD2046BDE8BF
:10CE4000F8832DE9F84380460E4617461D46DDF867
:10CE50002090B8F1000F01D0012000E0002050B96F
:10CE600000BF502080F31188BFF34F8FBFF36F8F47
:10CE700000BF00BFFEE70DB1012000E0002050B967
:10CE800000BF502080F31188BFF34F8FBFF36F8F27
:10CE900000BF00BFFEE707B10EB1012000E0002097
:10CEA00050B900BF502080F31188BFF34F8FBFF3FC
:10CEB0006F8F00BF00BFFEE707B90EB9012000E089
:10CEC000002050B900BF502080F31188BFF34F8F6E
:10CED000BFF36F8F00BF00BFFEE7502000900098A7
:10CEE000502801D1012000E0002050B900BF50209F
:10CEF00080F31188BFF34F8FBFF36F8F00BF00BF68
:10CF0000FEE700BF2C464CB1012084F846004B469A
:10CF10003A46314640460094FEF7BDFC2046BDE847
:10CF2000F883000070B505460E462C4654B900BF84
:10CF3000502080F31188BFF34F8FBFF36F8F00BF76
:10CF400000BFFEE7FFF79CFAD4E90F12206801FB4F
:10CF50000200A0600020A06320686060E06B401EBB
:10CF6000226C216800FB0211E160FF2084F844007C
:10CF700084F845009EB9206908B9012000E000202E
:10CF8000A8B904F1100000F085FF80B14FF0805087
:10CF900009490860BFF34F8FBFF36F8F07E004F1BB
:10CFA0001000FFF736FA04F12400FFF732FAFFF71A
:10CFB00091FA012070BD000004ED00E02DE9FF436F
:10CFC00083B0064688461D464FF00009344654B9E2
:10CFD00000BF502080F31188BFF34F8FBFF36F8FD6
:10CFE00000BF00BFFEE7B8F1000F01D1206C08B907
:10CFF000012000E0002050B900BF502080F31188CC
:10D00000BFF34F8FBFF36F8F00BF00BFFEE7022D4E
:10D0100002D1E06B012801D1012000E0002050B9CD
:10D0200000BF502080F31188BFF34F8FBFF36F8F85
:10D0300000BF00BFFEE700F077FD08B9059808B90A
:10D04000012000E0002050B900BF502080F311887B
:10D05000BFF34F8FBFF36F8F00BF00BFFEE700BF6E
:10D06000FFF70EFAA06BE16B884201D3022D28D1A5
:10D070002A4641462046FEF728FB0746606A08B963
:10D08000012000E0002068B904F1240000F002FF54
:10D0900088B14FF0805032490860BFF34F8FBFF323
:10D0A0006F8F08E03FB14FF080502D490860BFF30B
:10D0B0004F8FBFF36F8FFFF70DFA012007B0BDE868
:10D0C000F083059818B9FFF705FA0020F6E7B9F1E3
:10D0D000000F04D101A8FFF7F5FB4FF00109FFF79E
:10D0E000F9F9FFF703FDFFF7CBF994F94400401C71
:10D0F00010B9002084F8440094F94500401C10B990
:10D10000002084F84500FFF7E5F905A901A800F023
:10D11000E9FAF0B92046FEF7D6FCA0B104F1100000
:10D120000599FFF7E1FB2046FEF7B1FE00F0FEFE99
:10D13000002895D14FF0805009490860BFF34F8F08
:10D14000BFF36F8F8CE72046FEF7A1FE00F0EEFEE6
:10D1500086E72046FEF79BFE00F0E8FE0020ADE7E4
:10D1600004ED00E02DE9F84F07468A4690461E463A
:10D170003C4654B900BF502080F31188BFF34F8F55
:10D18000BFF36F8F00BF00BFFEE7BAF1000F01D100
:10D19000206C08B9012000E0002050B900BF5020E9
:10D1A00080F31188BFF34F8FBFF36F8F00BF00BFB5
:10D1B000FEE7022E02D1E06B012801D1012000E040
:10D1C000002050B900BF502080F31188BFF34F8F6B
:10D1D000BFF36F8F00BF00BFFEE7FFF7FFF900BF8F
:10D1E0005021EFF3118081F31188BFF34F8FBFF30C
:10D1F0006F8F00BF0546A06BE16B884201D3022E02
:10D2000025D194F945B0A06B009032465146204696
:10D21000FEF75BFA0BF1010088B9606A08B90120DA
:10D2200000E0002050B904F1240000F033FE28B1E2
:10D23000B8F1000F02D00120C8F8000004E00BF1A3
:10D24000010040B284F845004FF0010901E04FF0C1
:10D25000000900BF85F3118800BF4846BDE8F88F7C
:10D2600070B505462C4654B900BF502080F3118894
:10D27000BFF34F8FBFF36F8F00BF00BFFEE700F01B
:10D280004DFCA16888420CD1E068401EE060E06877
:10D2900028B900231A4619462046FFF78FFE0126BB
:10D2A00000E00026304670BD2DE9F74183B0054609
:10D2B0000E464FF000082C4654B900BF502080F3B2
:10D2C0001188BFF34F8FBFF36F8F00BF00BFFEE722
:10D2D0000EB9206C08B9012000E0002050B900BF51
:10D2E000502080F31188BFF34F8FBFF36F8F00BFC3
:10D2F00000BFFEE700F018FC08B9059808B9012046
:10D3000000E0002050B900BF502080F31188BFF327
:10D310004F8FBFF36F8F00BF00BFFEE700BFFFF767
:10D32000AFF8A76BF7B131462046FEF7B9F9781E82
:10D33000A063206908B9012000E0002060B904F171
:10D34000100000F0A7FD38B14FF080502F49086061
:10D35000BFF34F8FBFF36F8FFFF7BCF8012006B00C
:10D36000BDE8F081059818B9FFF7B4F80020F6E79A
:10D37000B8F1000F04D101A8FFF7A4FA4FF001089B
:10D38000FFF7A8F8FFF7B2FBFFF77AF894F944002B
:10D39000401C10B9002084F8440094F94500401C5A
:10D3A00010B9002084F84500FFF794F805A901A8FA
:10D3B00000F098F9F0B92046FEF778FBA0B104F12F
:10D3C00024000599FFF790FA2046FEF760FD00F073
:10D3D000ADFD0028A3D14FF080500C490860BFF389
:10D3E0004F8FBFF36F8F9AE72046FEF750FD00F096
:10D3F0009DFD94E72046FEF74AFD00F097FD20468C
:10D40000FEF754FB00288AD00020A8E704ED00E0D6
:10D410002DE9F05F064689461746344654B900BFE9
:10D42000502080F31188BFF34F8FBFF36F8F00BF81
:10D4300000BFFEE7B9F1000F01D1206C08B901204F
:10D4400000E0002050B900BF502080F31188BFF3E6
:10D450004F8FBFF36F8F00BF00BFFEE7FFF7BEF82F
:10D4600000BF5021EFF3118081F31188BFF34F8F7C
:10D47000BFF36F8F00BF0546D4F838A0BAF1000F94
:10D4800022D094F944B049462046FEF709F9AAF1A2
:10D490000100A0630BF1010070B9206908B90120F7
:10D4A00000E0002068B904F1100000F0F3FC40B186
:10D4B0003FB10120386004E00BF1010040B284F874
:10D4C00044004FF0010801E04FF0000800BF85F371
:10D4D000118800BF4046BDE8F09F00002DE9F341F0
:10D4E00082B005464FF000082C46002654B900BF14
:10D4F000502080F31188BFF34F8FBFF36F8F00BFB1
:10D5000000BFFEE7206C08B9012000E0002050B900
:10D5100000BF502080F31188BFF34F8FBFF36F8F90
:10D5200000BF00BFFEE700F0FFFA08B9039808B992
:10D53000012000E0002050B900BF502080F3118886
:10D54000BFF34F8FBFF36F8F00BF00BFFEE700BF79
:10D55000FEF796FFA76BFFB1781EA063206810B995
:10D56000FEF77AFDA060206908B9012000E00020E4
:10D5700060B904F1100000F08DFC38B14FF080501C
:10D5800043490860BFF34F8FBFF36F8FFEF7A2FFD1
:10D59000012004B0BDE8F081039898B90EB90120CC
:10D5A00000E0002050B900BF502080F31188BFF385
:10D5B0004F8FBFF36F8F00BF00BFFEE7FEF78AFFFC
:10D5C0000020E6E7B8F1000F04D16846FFF77AF9CA
:10D5D0004FF00108FEF77EFFFFF788FAFEF750FFD5
:10D5E00094F94400401C10B9002084F8440094F9D8
:10D5F0004500401C10B9002084F84500FEF76AFF82
:10D6000003A9684600F06EF840BB2046FEF74EFACC
:10D61000F0B1206838B9FEF733FFA06800F0E8FBEE
:10D620000646FEF757FF04F124000399FFF75CF963
:10D630002046FEF72CFC00F079FC002888D14FF042
:10D64000805013490860BFF34F8FBFF36F8F7FE7A0
:10D650002046FEF71CFC00F069FC79E72046FEF747
:10D6600016FC00F063FC2046FEF720FA0028EED0FE
:10D670005EB1FEF705FF2046FEF78EF807463946F5
:10D68000A068FFF76DF9FEF725FF002081E7000095
:10D6900004ED00E02DE9F04106460F46344654B94A
:10D6A00000BF502080F31188BFF34F8FBFF36F8FFF
:10D6B00000BF00BFFEE700F031FAA168884204D144
:10D6C000E068401CE060012508E039462046FFF78D
:10D6D00005FF054615B1E068401CE0602846BDE83E
:10D6E000F081000070B505460C4655B900BF5020CA
:10D6F00080F31188BFF34F8FBFF36F8F00BF00BF60
:10D70000FEE754B900BF502080F31188BFF34F8F5C
:10D71000BFF36F8F00BF00BFFEE7FEF7B1FE1248F8
:10D7200002686868131A2068401C08B9002617E0D0
:10D730000E4928680968884204D06868904201D878
:10D7400001260DE02068984207D92068C01A2060A1
:10D750002846FFF7B7F8002602E0002020600126E7
:10D76000FEF7B8FE304670BD2C00002040000020BF
:10D770002DE9FF4F85B0804689461746DDE912AB9B
:10D78000B800FEF7C3FB064656B16420FEF7BEFBA9
:10D7900004460CB1266304E03046FEF7B9FE00E013
:10D7A00000248CB1002084F86100CDE900ABCDE904
:10D7B00002403A4649464046089BFEF781F820461B
:10D7C000FDF7B4FE012501E04FF0FF35284609B012
:10D7D000BDE8F08F2DE9F04F85B0074688469146A9
:10D7E0009A46DDE90EB6109C0EB1012000E0002043
:10D7F00050B900BF502080F31188BFF34F8FBFF3A3
:10D800006F8F00BF00BFFEE70CB1012000E00020D9
:10D8100050B900BF502080F31188BFF34F8FBFF382
:10D820006F8F00BF00BFFEE7642003900398642859
:10D8300001D1012000E0002050B900BF502080F34A
:10D840001188BFF34F8FBFF36F8F00BF00BFFEE79C
:10D8500000BFB4B1AEB125462C462E63022085F838
:10D860006100002004A953464A46CDE900B1CDE944
:10D87000025041463846FEF723F82846FDF756FE8B
:10D8800001E000200490049805B0BDE8F08F00008E
:10D890002DE9F04706460D46174698464FF0010A17
:10D8A00056B900BF502080F31188BFF34F8FBFF3EC
:10D8B0006F8F00BF00BFFEE73446FEF7E1FDB8F111
:10D8C000000F02D0E06DC8F8000094F860900220CC
:10D8D00084F86000052F17D2DFE807F01503070B67
:10D8E0000D00E06D2843E06521E0E06D401CE0653F
:10D8F0001DE0E5651BE0B9F1020F01D0E56501E02F
:10D900004FF0000A13E012E0E06D401C08B901205E
:10D9100000E0002050B900BF502080F31188BFF311
:10D920004F8FBFF36F8F00BF00BFFEE700BF00BF88
:10D93000B9F1010F32D1201DFEF73DFD1A49E06A11
:10D940000968884202D91849E06A0860E16A01EB77
:10D950008101164A02EB8100211DFEF784FDA06AB9
:10D9600008B9012000E0002050B900BF502080F32A
:10D970001188BFF34F8FBFF36F8F00BF00BFFEE76B
:10D980000B49E06A0968C96A884207D94FF080509C
:10D9900008490860BFF34F8FBFF36F8FFEF79AFD02
:10D9A0005046BDE8F0870000300000204806002007
:10D9B0001800002004ED00E02DE9F84F07460E4660
:10D9C00090469946DDF828B00120009057B900BF75
:10D9D000502080F31188BFF34F8FBFF36F8F00BFCC
:10D9E00000BFFEE7FEF7FAFD3C4600BF5021EFF313
:10D9F000118081F31188BFF34F8FBFF36F8F00BF8A
:10DA00000546B9F1000F02D0E06DC9F8000094F8A6
:10DA100060A0022084F86000B8F1050F17D2DFE89B
:10DA200008F01503070B0D00E06D3043E06521E0C1
:10DA3000E06D401CE0651DE0E6651BE0BAF1020FF9
:10DA400001D0E66501E00020009013E012E0E06DF7
:10DA5000401C08B9012000E0002050B900BF502050
:10DA600080F31188BFF34F8FBFF36F8F00BF00BFEC
:10DA7000FEE700BF00BFBAF1010F3CD1A06A08B9B0
:10DA8000012000E0002050B900BF502080F3118831
:10DA9000BFF34F8FBFF36F8F00BF00BFFEE7194882
:10DAA0000068A0B9201DFEF786FC1749E06A0968E6
:10DAB000884202D91449E06A0860E16A01EB8101F9
:10DAC000124A02EB8100211DFEF7CDFC04E004F1B7
:10DAD00018010F48FEF7C7FC0E49E06A0968C96AD9
:10DAE000884208D9BBF1000F02D00120CBF800001A
:10DAF00001200949086000BF85F3118800BF009824
:10DB0000BDE8F88F500000203000002048060020BB
:10DB1000D00A0020180000203C00002001490868BD
:10DB200070470000180000200549096809B9012064
:10DB300005E00449096809B9022000E000207047A7
:10DB400034000020500000200149086870470000A0
:10DB50002C00002070B5FEF741FD00250148046847
:10DB6000204670BD2C0000202DE9F0414FF0000848
:10DB70004348006800287BD142480068451C414862
:10DB8000056015BB40480068006808B9012000E046
:10DB9000002050B900BF502080F31188BFF34F8F91
:10DBA000BFF36F8F00BF00BFFEE7374807683748F5
:10DBB0000068354908603548076035480068401CF2
:10DBC00033490860FEF7B4F800BF32480068854268
:10DBD0003BD300BF2C480068006808B9012000E072
:10DBE000002020B14FF0FF302A4908602CE0264881
:10DBF0000068C068C4686668B54202D225480660FD
:10DC000022E0201DFEF7D7FBA06A18B104F118002E
:10DC1000FEF7D1FB2049E06A0968884202D91E4913
:10DC2000E06A0860E16A01EB81011C4A02EB8100B5
:10DC3000211DFEF718FC1A49E06A0968C96A884282
:10DC4000C8D34FF00108C5E700BF15480068C06A97
:10DC500000EB8000114951F82000012801D94FF054
:10DC600001081048006808B14FF0010805E0FFE71F
:10DC70000D480068401C0C4908604046BDE8F08132
:10DC8000500000202C0000201C000020200000205C
:10DC900040000020480000203000002048060020FE
:10DCA000180000203C000020380000202DE9F04141
:10DCB0000746884614461D46FEF7E2FB21480068E9
:10DCC00090F86000022818D01E49096801F15C0034
:10DCD000C96DB943016001201A49096881F86000E3
:10DCE0005DB101212846FDF7E3FB4FF08050164956
:10DCF0000860BFF34F8FBFF36F8FFEF7EBFBFEF7AC
:10DD0000BFFB1CB10F480068C06D20600D48006863
:10DD100090F86000022801D0002608E0094909684F
:10DD200001F15C00C96D21EA0801016001260020B3
:10DD30000449096881F86000FEF7CCFB3046BDE875
:10DD4000F08100001800002004ED00E070B50546E9
:10DD50002C460026002D43D022480068844201D181
:10DD6000012000E0002050B900BF502080F311884E
:10DD7000BFF34F8FBFF36F8F00BF00BFFEE7606D33
:10DD800050B900BF502080F31188BFF34F8FBFF30D
:10DD90006F8F00BF00BFFEE7606D401E6065216DA4
:10DDA000E06A88421CD0606DD0B9201DFEF703FBED
:10DDB000206DE062E06AC0F13800A0610A49E06AC3
:10DDC0000968884202D90849E06A0860E16A01EB03
:10DDD0008101064A02EB8100211DFEF744FB01266A
:10DDE000304670BD1800002030000020480600209A
:10DDF00070B505462C460026002D42D02249E06A27
:10DE00000968C96A884235D2A06900F0004028B983
:10DE10001D480068C06AC0F13800A061E16A01EBEA
:10DE200081011A4A02EB81016069884201D1012017
:10DE300000E00020C0B1201DFEF7BDFA12480068C6
:10DE4000C06AE0621249E06A0968884202D9104952
:10DE5000E06A0860E16A01EB81010C4A02EB810093
:10DE6000211DFEF700FB03E007480068C06AE0627E
:10DE7000012606E00449206D0968C96A884200D27B
:10DE80000126304670BD0000180000204806002022
:10DE90003000002070B50646F068C46854B900BF71
:10DEA000502080F31188BFF34F8FBFF36F8F00BFF7
:10DEB00000BFFEE704F11800FEF77DFA1548006880
:10DEC000A0B9201DFEF777FA1349E06A0968884275
:10DED00002D91149E06A0860E16A01EB81010F4A49
:10DEE00002EB8100211DFEF7BEFA04E004F11801E7
:10DEF0000B48FEF7B8FA0B49E06A0968C96A88421C
:10DF000004D9012501200849086000E000252846C1
:10DF100070BD0000500000203000002048060020A6
:10DF2000D00A0020180000203C00002070B500241A
:10DF300000263648006850B900BF502080F3118891
:10DF4000BFF34F8FBFF36F8F00BF00BFFEE7FEF739
:10DF500097FA2E480068401E2C4908600846006861
:10DF600000284ED12A48006800284AD023E02948DA
:10DF7000C068C46804F11800FEF71DFA201DFEF702
:10DF80001AFA2549E06A0968884202D92249E06AFA
:10DF90000860E16A01EB8101204A02EB8100211D4A
:10DFA000FEF761FA1E49E06A0968C96A884202D32D
:10DFB00001201C4908601748006808B9012000E0EA
:10DFC00000200028D3D00CB1FDF7B2FE164805683A
:10DFD00065B100BFFFF7C8FD10B10120114908600D
:10DFE0006D1E002DF6D100200F4908600D48006815
:10DFF00038B1012630070D490860BFF34F8FBFF3DA
:10E000006F8FFEF767FA304670BD000050000020A9
:10E0100028000020D00A0020300000204806002000
:10E02000180000203C0000203800002004ED00E033
:10E0300010B586B00024FDF7D5FA16480068D0B1B7
:10E0400000200590049003AA04A905A8FEF7D4F9BE
:10E050000222DDE904100023CDE9002102900EA187
:10E060000F48039AFFF7B6FB0E49086008460068A0
:10E0700000B1012400BF54B900BF502080F31188C3
:10E08000BFF34F8FBFF36F8F00BF00BFFEE7204687
:10E0900006B010BD64000020546D722053766300FA
:10E0A00075BE0008680000202DE9FF4704460D46B4
:10E0B00016461F46DDF830804FF0000954B900BF06
:10E0C000502080F31188BFF34F8FBFF36F8F00BFD5
:10E0D00000BFFEE71448006810B300950196029453
:10E0E000062D15DAFFF720FD022808D1002342464D
:10E0F00069460D480068FEF761FF814610E0002385
:10E100001A46694608480068FEF758FF814607E04E
:10E1100000233A46694604480068FFF723F8814621
:10E12000484604B0BDE8F0876400002081F000415B
:10E13000704780F00040704721F00041704720F0A8
:10E140000040704721F00042A2F16052B2F5801FFA
:10E1500001F0004328BFD2F17F6C0BD95FEA001CAD
:10E1600043EAC20242EB507018BF704728BF20F04C
:10E1700001007047B2F5801FBCBF184670474FEAD8
:10E18000410C1CF5001F02D2084600F0ADBD70B571
:10E1900000F084FB00000089FFF7F6BF4FF000405D
:10E1A000A0F580007047000010B591EA030F48BF4A
:10E1B00083F0004300F1DA83841A71EB030C05D27B
:10E1C000121943EB0C03001B61EB0C01DFF824E197
:10E1D0004FEA1154A4EB135C1EEA430F18BF9EEAEA
:10E1E000445F73D023EA0E03DCF1200E21EA0451D0
:10E1F00043F4801332D322FA0CFE10EB0E0023FA04
:10E200000CFE41EB0E01CCF1200E03FA0EFE10EBDA
:10E210000E0051F10001B1F5801FCCF1200E32D279
:10E2200001EB045112FA0EF2BDE8104058BF7047DE
:10E23000401C38BF5FEA420218BF7047002814BF75
:10E2400020F0010041F100014FEA410313F5001FE6
:10E2500038BF7047A1F1C04100F06EBB012A43EB0B
:10E260000302ACF1200CDCF11F0E32BF4FF0000EA8
:10E2700023FA0CF310EB030041EB0451B4EB115FF4
:10E28000D0D0A1EB045101F5801149085FEA3000BC
:10E2900001EB04510ED350F1000038BF12FA0EFE0C
:10E2A00008D1BDE81040C9E7401C38BF5FEA420210
:10E2B000CAD1C3E7BDE810404FEA410313F5001F80
:10E2C00038BF7047A1F1C04100F036BB9EEA445F01
:10E2D00008D011EA5E0FBDE8104004BF01F0004114
:10E2E00000207047BDE8104070B500F0D7FA00BFBD
:10E2F00064FBBE3E0000E0FF491058BFC1F1404141
:10E300005B1058BFC3F140438B42EFF3008070476E
:10E310002DE9C04130B4DFF8A0C23CEA111418BFA7
:10E320003CEA131400F0EC8081EA03051CEA1114A6
:10E3300044EAD57418BF1CEA131500F0C780A4EB9B
:10E3400005044FF0004545EAC12145EAC32341EAEF
:10E35000505143EA525304F17F74994204F500345A
:10E360004FEAC0204FEAC22208BF904200F09C80D2
:10E370004FEA13650FF24016765D4FEA134506FB30
:10E3800005F7C7F1807706FB07F74FEAD737A7FBFA
:10E3900003687642C8F58038A7FB06CE38BFA8F1DF
:10E3A000010807FB08E64FF0000EA6FB028CE6FB17
:10E3B00003CEDCF1000CCEF1004E38BFAEF1010E01
:10E3C000A6FB0C584FF000074FF00005E6FB0E8748
:10E3D000A1FB08C6A0FB07CE16EB0E0645F1000513
:10E3E000E1FB076515F1E04E7EBFA4F580345FEADE
:10E3F00046066D4116F1800745F100054FEA1727E3
:10E400004FEA066647EA0567A6F1DE46B6F1805F89
:10E410004FEA15251FD9384624F0010C05EBC471CD
:10E42000BCF1FE6F01EB0C1102D8F0BCBDE800811D
:10E4300024425CBF01F5801E9EEAC47F02D4F0BC7A
:10E44000BDE80081244238D4F0BCA1F1C041BDE850
:10E45000004100F071BA4FEAD22242EA43524FEA39
:10E46000D323A7FB02864FEAD02040EA415007FBA6
:10E4700003661EEA0E0F4FEAD12105FB026658BF64
:10E48000A6EB0056B6EB00564FEA520E4EEAC37E9C
:10E4900018EB0E0E56EB530EBDD518EB02085E417D
:10E4A0007F1C55F10005B6E74FF480154FF00007CB
:10E4B0004FF000064FF00008ADE7F0BC4FF0000051
:10E4C00001F1C04101F00041BDE8008111EA0C1FDB
:10E4D0000CEA131500D00CE013EA0C1F00F02580A5
:10E4E0004FF00000F0BC81EA030101F00041BDE8FB
:10E4F0000081F0BCBDE8004181EA030100F01CBAD4
:10E50000F0BCBDE8004170B500F0C8F9097EFC3EE2
:10E5100000F007B881EA03014FF0000001F000416C
:10E52000704781EA030100F007BAF0BCBDE8004182
:10E530004FF0000021497047FFFDFBF9F7F5F4F2B9
:10E54000F0EEEDEBE9E8E6E4E3E1E0DEDDDBDAD88E
:10E55000D7D5D4D3D1D0CFCDCCCBCAC8C7C6C5C4EC
:10E56000C2C1C0BFBEBDBCBBBAB9B8B7B6B5B4B303
:10E57000B2B1B0AFAEADACABAAA9A8A8A7A6A5A4EE
:10E58000A3A3A2A1A09F9F9E9D9C9C9B9A999998B2
:10E590009797969595949393929191908F8F8E8E55
:10E5A0008D8C8C8B8B8A89898888878786858584E2
:10E5B00084838382828181800000FF070000F87FCE
:10E5C00051EA030C17D41CF5801F58BFBCF5801FFF
:10E5D00000F10680994218BF704708BF904270470B
:10E5E00007D711F5801F58BF13F5801F19D4994222
:10E5F0007047894270471CF5801F08D5BCF5801F05
:10E60000F7D58B4218BF704708BF824270474FF45E
:10E61000001C1CEB410F38BF1CEB430F01D28B4297
:10E62000704770B500F03AF9922449004FF000515C
:10E630004FF08053FFF760BE4FEA41034FEA535358
:10E64000A3F58063D3F11E03C8BFD3F1210C0CDD09
:10E650004FF0004242EAC12242EA505232FA03FC31
:10E660008CEAE17CACEBE1707047102BC4BF00205A
:10E67000704703F5787CBCF1FF3F04D06FF0004297
:10E6800082EA2100704770B500F008F949922480B1
:10E6900000207047F2E700004FEA1153A3F58063B2
:10E6A000D3F11E03A8BFD3F1200C08DB4FF00042CA
:10E6B00042EAC12252EA505232FA03F0704709424C
:10E6C0000BD4102BC4BF0020704703F5787CBCF13D
:10E6D000FF3F05D04FF0FF3070474FF0000070470C
:10E6E00070B500F0DBF800BF49922480002070472D
:10E6F000F0E710F0004248BF4042B0FA80F310FA51
:10E7000003F10AD0C3F11D0303F580634FEA4150C2
:10E7100002EB035202EBD12170474FF0000070472B
:10E72000B0FA80F310FA03F10AD0C3F11D0303F528
:10E7300080634FEA41504FEA035202EBD121704708
:10E740004FF0000070470000DFF848C170B51CEAC8
:10E75000111E1EBF1CEA13159EEA0C0F95EA0C0F42
:10E7600000F06F8081EA030423EA4C134EEAD47E62
:10E7700021EA4C1141F4801143F48013AE44A1FB13
:10E78000024CA0FB0365AEF17F7E361955EB0C05FC
:10E79000A1FB034C4CF10003A0FB021C16EB0C0682
:10E7A000654153F10003094218BF46F0010613F416
:10E7B000007F0BD14FEA03314FEA0530340341EAC1
:10E7C000155140EA16506FF003020AE04FEAC321E8
:10E7D0004FEAC520F40241EA555140EA56506FF025
:10E7E000020202EB2E4201EB025585EACE710AD0FD
:10E7F0005FEA440C18BF24F0004450F1000041F1DE
:10E80000000120EAD47040F2FE7C624500D270BD67
:10E81000A84214BF4FF080444FF04044002E08BF80
:10E820000024BEF1806FA8BFA1F1C041BDE87040D7
:10E8300080F282804FF0000001F1C04101F0004100
:10E8400070479EEA0C0F0CEA131518BF95EA0C0FDF
:10E8500006D04FF0000081EA030E0EF0004170BDBB
:10E8600000F01CF88900013E00F007B800F009B87C
:10E870004FEA430C5FEA5C5C08D081EA030100F0D8
:10E880005BB84FEA410C5FEA5C5CF6D14FF00000E8
:10E89000014970470000FF070000F87F0EF1020EEB
:10E8A0002EF0030E5EF8046B364205D4012A43EBCA
:10E8B000030515F5001F12D8012841EB010C1CF5CA
:10E8C000001F0CD80ED14FEAD17C15F5001F0CEBC0
:10E8D0004C0C0CF1020C08BF4CEBD37C04E04FF065
:10E8E000080C01E04FEAD37C0CEB4C0526FA05F648
:10E8F00006F00706B6F1040C06D20EEB860CBDE856
:10E9000070404CF0010C6047DFE80CF0090B02028C
:10E910004FF000414FF00000A1F5002170BD1946F5
:10E920001046012851EB010418BFD4F5001484BF30
:10E93000002001F0004170BD0808A0F500114FEA69
:10E940003101704791EA030F10B581F000413FF5A6
:10E9500033AC83F0004300F009B8000010B591EA31
:10E96000030F48BF83F000433FF526AC841A71EBD8
:10E97000030C07D212198CF0004C43EB0C03001B64
:10E9800061EB0C01DFF8A4E14FEA1154A4EB135C36
:10E990001EEA430F18BF9EEA445F00F0B08023EAEE
:10E9A0006E03524221EA0451C3EB6E0338BF5B1E73
:10E9B000DCF1200E25D322FA0CFE10EB0E0043FAF8
:10E9C0000CFE41EB0E01CCF1200E03FA0EFE10EB13
:10E9D0000E0051F10001CCF1200E29D412FA0EF2F2
:10E9E00001EB0451BDE8104058BF7047401C1CBFEC
:10E9F000B2F1004F704700280CBF491C20F0010005
:10EA0000704712EB020E43EB030218BF4FF0010EEA
:10EA10004EEA4202ACF1200CDCF11E0E54D943FA4E
:10EA20000CFE10EB0E0051F1FF31CCF11E0ED5D5CE
:10EA30000EF1010E12FA0EFE404141EB010101EB15
:10EA4000445C5FEA5C5C10D910EBDE7001EB0451B2
:10EA500038BFBEF1004FBDE8104018BF7047002816
:10EA60000CBF491C20F00100704730D24FEAD42C73
:10EA700011F5001124F400641BD0B1FA81F20B3AB5
:10EA8000A41AA41ED2F12003914030FA03F31943D3
:10EA9000904001EBCC71002C01EB0451BDE810401B
:10EAA000A8BF704701F1C0414FF0000001F00041E4
:10EAB0007047B0FA80F310FA03F100D110BDE41AE8
:10EAC000173C4805C90AE4E701EB045110BD4910A1
:10EAD00001EB0451BDE810404FEA300002E04FF076
:10EAE000000170474A0008BF0042F8D0B2F5001F8D
:10EAF00028BF704701F000414FF0000070479EEAC8
:10EB0000445F07D011EA5E0FBDE8104004BF00214A
:10EB100000207047BDE8104070B5FFF7BFFE00BF92
:10EB200040DFF63E83F00041104670470000E0FFF2
:10EB300043004FEAD30C4FEA3C0C43401FBF400751
:10EB40000CF1605113F0FE4F70471CF0006F03D1C1
:10EB500000200CF0004170470CF0004343EA507075
:10EB600010B540EACC0000F074F800BF000000923D
:10EB70004FEA0001FFF7E0BE4FF000414FF0000008
:10EB8000A1F500217047000000EE100A00EE901A77
:10EB9000B4EE600AF1EE10FA78BF704700F00DB8DD
:10EBA00010B5FFF7F1FFEFF3008020F0104038BF01
:10EBB00040F0004080F3008810BDBDE8104010B563
:10EBC00000F047F80000000900F007B84FF040409F
:10EBD00010F1004FEFF300807047401058BFC0F1B4
:10EBE0004040491058BFC1F140418142EFF30080DD
:10EBF00070474FF07E5209E011F0004204D54042C8
:10EC0000C1F1000138BF491E42F07E520B0002F1F3
:10EC1000706212BF20235FEA00017047B1FA81FCE5
:10EC2000A3EB0C0301FA0CF120FA03FC02EBC35234
:10EC3000C3F1200341EA0C0110FA03FC5CEA416CC9
:10EC400042EB112018BF5FF0806C28BF20F001005C
:10EC500070470EF1020E2EF0030E5EF8044B2442B4
:10EC600004D44FEA4102B2F17F4F11D84FEA40037A
:10EC7000B3F17F4F0CD80ED14FEAD07CB2F17F4F69
:10EC80000CEB4C0C0CF1020C08BF4CEBD17C04E0FB
:10EC90004FF0080C01E04FEAD17C0CEB4C0324FA56
:10ECA00003F404F00704B4F1040C06D20EEB840C58
:10ECB000BDE810404CF0010C6047DFE80CF007089D
:10ECC00002024FF00040A0F5800010BD084642004F
:10ECD00018BFD2F1807288BF00F0004010BD4FF025
:10ECE0004070E1EE100A7047FF2141EAD050C005A4
:10ECF00070470000E8EE000800000000000000007F
:10ED000000000000000000000002000018000000E9
:10ED1000000000000000000000061016000610169B
:10ED200000000000000000000102030406070809BB
:10ED30000000000001020304010000000000024086
:10ED4000100000000000024001000000000402402A
:10ED500010000000000802402000000000080240EF
:10ED600008000000001802404000000000180240A7
:10ED7000D0040020000000009A99193E0000803F56
:10ED800000000000000000000000803F0000803F05
:10ED9000000000000000000014EF00080000000068
:10EDA000000000000000000000000000000400005F
:10EDB000300000000000000000000000FCEE000831
:10EDC0000000000000000000000000000000000043
:10EDD0000004000018000000000000000000000017
:10EDE00008EF000800000000000000000000000024
:10EDF00000000000000400001800000000000000F7
:10EE000000000000F4EE0008000000000000000018
:10EE100000000000000000000004000018000000D6
:10EE200000000000000000004FBB610567ACDD3F43
:10EE3000182D4454FB21E93F9BF681D20B73EF3F21
:10EE4000182D4454FB21F93FE2652F227F2B7A3C99
:10EE5000075C143326A6813CBDCBF07A8807703C52
:10EE6000075C143326A6913CC4EB98999999C9BFC5
:10EE7000711623FEC671BCBF6D9A74AFF2B0B3BFFA
:10EE80009AFDDE522DDEADBF2F6C6A2C44B4A2BFBA
:10EE90000D5555555555D53FFF8300922449C23F26
:10EEA0006E204CC5CD45B73F513DD0A0660DB13F5A
:10EEB000EB0D76244B7BA93F11DA22E33AAD903F6C
:10EEC0000000000000000000000000006E83F9A2B6
:10EED0002915444ED15727FCC0DD34F5999562DBE6
:10EEE0004190433CAB6351FE64656661756C74543C
:10EEF00061736B0072656D6F746500006174746995
:10EF00005F6573746900000067696D62616C5F63BF
:10EF100074726C005461736B5F496E697400000019
:10EF200040EF00080000002020020000C40100089B
:10EF3000B0EF000820020020108500002002000829
:10EF4000C132104201037D24F41AAA010118051CE4
:10EF5000022B073D12013C0A0202083A0908256605
:10EF600066E63E23803F4FC04017B7513A0C390444
:10EF70004ABF04332041E24029141E80BFDB0FC981
:10EF8000185A8040210C11FA2AF9400E19404166A6
:10EF90006606400110E9400114094A4029249B7A81
:10EFA0004440293869401D3FD7A330040318F0BE00
:040000050800018965
:00000001FF
